:020000040800F2
:100000000004002011360008D1380008D13800085B
:10001000D1380008D1380008D1380008D13800089C
:10002000D1380008D1380008D1380008413900081B
:10003000D1380008D1380008D1380008613A0008EA
:10004000D1380008D1380008D1380008D13800086C
:10005000D1380008D1380008D1380008D13800085C
:10006000D1380008D1380008D1380008C14701084C
:10007000014801084148010881480108C1480108B8
:100080000149010841490108C1530108B15801085B
:10009000D1580108F158010811590108D138000858
:1000A00051750108D1740108D1380008F1740108B4
:1000B0001175010831750108D1790108415C010809
:1000C000B15D0108D1380008D1380008D1380008E6
:1000D000D1380008017E0108217E0108417E010817
:1000E000D1380008D1380008D1380008D1380008CC
:1000F000D1380008D1380008D138000881490108FA
:10010000D1380008D1380008F1790108D138000849
:10011000D1380008D1380008D1380008D13800089B
:10012000C1490108014A0108414A0108814A010800
:10013000C14A0108D1380008D138000831590108F6
:1001400051590108715901089159010821680108A4
:10015000014B0108414B0108814B0108D1380008CF
:10016000D1380008D1380008D1380008D13800084B
:10017000D1380008D1380008D1380008D13800083B
:08018000D1380008D138000855
:0C0188009D070008351100084513000811
:08019400B10700084911000841
:1001A00080B584B000AF7860396041F27823C2F244
:1001B00000031B68B3F848311AB23B689A420BDA65
:1001C00043F62840C2F200004EF6C001C0F601011D
:1001D0003A6808F065F95CE0386811F0D1FB024636
:1001E00041F27823C2F200031B68D3F8883C104622
:1001F000194602F065FC034618464FF00001C4F2B0
:10020000C82102F05DFC0346184602F021FE0346B9
:10021000FB60FB68002B0BDA43F62840C2F20000BB
:100220004EF6D801C0F60101FA6808F039F930E05D
:10023000386813F01DFD02467B689B68104619461E
:1002400002F03EFC0346184602F002FE0346BB6085
:100250001AF0F6FD0346002B0CBF00230123DBB28E
:10026000002B0AD043F62840C2F200004EF6FC01F3
:10027000C0F60101FA6808F013F97B685A6840F289
:10028000B413C1F20003DB681046B968FA6812F0D3
:100290001FFB07F11007BD4680BD00BF80B586B0CB
:1002A00000AF03463960FB710FF01AF90346002BCB
:1002B00014BF00230123DBB2002B65D141F274236C
:1002C000C2F200031B68D3F830273B689A420BDC6C
:1002D0004EF60C10C0F601004EF61C11C0F60101DE
:1002E0004FF05D0203F004FD1AF0AAFD0346002B57
:1002F00007D041F27423C2F200031B6803F5E763E1
:1003000006E041F27423C2F200031B6803F61C13DB
:100310003B613868396943F62C52C2F2000212F090
:10032000CFFD43F62C53C2F200031B68002B2DD0E7
:100330001AF076FDF8604FF000037B6116E07A69F1
:1003400013464FEA43039B184FEA830343F62C52AC
:10035000C2F200029B1803F10403BB60B868F9689D
:10036000FFF71EFF7B6903F101037B6143F62C530A
:10037000C2F200031A687B699A42D4BF00230123AA
:10038000DBB2002BDBD102E000BF00E000BF07F1D1
:100390001807BD4680BD00BFB0B58AB002AF786017
:1003A00039603B68002B00F0AD8041F27823C2F247
:1003B00000031B68184613F0A3FC0346386819466F
:1003C00011F056FBB861386813F042FC034618463A
:1003D000B96902F075FB03467B6141F27823C2F2F2
:1003E00000031B681846396813F0C2FC386138698D
:1003F0004FF0000102F002FD0346002B0CD03869DB
:1004000001F0E2FE02460B46396800914EF64C10B0
:10041000C0F6010001F020FD38694FF0000102F044
:10042000F7FC0346002B6FD1386813F011FC02462D
:100430007B689B681046194602F042FB034618464B
:10044000796902F033FA03461846396902F02CFA4A
:100450000346184602F0FCFC0346184602F0DAFA9E
:100460000346FB614FF001031C46F8694FF00001A1
:1004700002F0C4FC0346002B02D14FF000031C46DF
:10048000E3B2FB6043F6E030C2F20000F96801F02D
:100490003DFBFB68002B11D0F86901F095FE024688
:1004A0000B4643F62840C2F200004EF66411C0F637
:1004B000010107F0F5FF4FF00003FB617B685D6809
:1004C000F8694FF00001C4F2C82102F0F9FA0346BE
:1004D000184602F0BDFC044638694FF00001C4F232
:1004E000C82102F0EDFA0346184602F0B1FC0246BC
:1004F00040F2B413C1F20003DB682846214612F033
:10050000E7F902E000BF00E000BF07F12007BD46A9
:10051000B0BD00BF80B586B000AF03463960FB7147
:100520001AF07EFC386141F27423C2F200031B68AA
:1005300003F530633868194643F62C52C2F20002C4
:1005400012F0BEFC43F62C53C2F200031B68002BD2
:1005500028D04FF000037B6116E07A6913464FEA1A
:1005600043039B184FEA830343F62C52C2F2000266
:100570009B1803F10403FB60F8683969FFF70CFF6F
:100580007B6903F101037B6143F62C53C2F2000344
:100590001A687B699A42D4BF00230123DBB2002B87
:1005A000DBD100E000BF07F11807BD4680BD00BFEA
:1005B00080B500AF43F62840C2F2000043F6107148
:1005C000C2F2000108F0ECF880BD00BF80B586B033
:1005D00000AF03463960FB7141F27423C2F200039D
:1005E0001B68D3F830273B689A420BDC4EF60C10A0
:1005F000C0F601004EF61C11C0F601014FF0A50235
:1006000003F076FB1AF00CFC78617B69B3F1FF3FD5
:100610000AD143F62840C2F200004EF67C11C0F623
:10062000010107F03DFF24E04FF48053CEF20003B8
:100630005B683B61FB7918463968FFF72FFEFB7951
:1006400018463968FFF766FF4FF48053CEF2000377
:100650005A683B69D31AFB60FB68002B09DDF96817
:100660000A464FEAE27343F61070C2F2000005F04A
:10067000AFFC07F11807BD4680BD00BF80B500AFD5
:100680001AF05EFBFFF794FF80BD00BF80B500AF9E
:100690004EF68C10C0F6010040F27D61C0F60001FC
:1006A00005F096FE43F62840C2F200004EF69C117B
:1006B000C0F6010107F03CFD40F2B413C1F20003A3
:1006C000DB6843F62840C2F200004EF6B011C0F6D7
:1006D00001011A4607F02CFF43F61070C2F2000029
:1006E0004EF6C411C0F6010105F04AFC0EF0F8FE0A
:1006F0000346002B14BF00230123DBB2002B09D0DB
:1007000043F62840C2F200004EF6D411C0F60101B3
:1007100007F00EFF40F2CD50C0F600004EF6FC117F
:10072000C0F601011AF01CFA80BD00BF80B500AF11
:1007300043F6E030C2F200004FF0060101F010FA7B
:100740000346042BD4BF00230123DBB2184680BD2F
:1007500080B582B000AF786039607B68012B0AD128
:100760003A684FF6FF739A4205D143F6E030C2F281
:10077000000001F04DF97B68002B0AD13A684FF672
:10078000FF739A4205D143F6E030C2F2000001F057
:1007900085F907F10807BD4680BD00BF80B500AFF1
:1007A0004FF001004FF6FF71FFF7D2FF80BD00BF91
:1007B00080B500AF4FF000004FF6FF71FFF7C8FFA4
:1007C00080BD00BF0000000000000000000000002D
:1007D00080B500AF41F27823C2F200031B681846CF
:1007E00010F056F803464EF61020C0F601001946E8
:1007F00006F056FB43F2D813C2F200034FF00A0290
:100800001A7043F2D813C2F200034FF00B025A7071
:1008100043F2D813C2F200031B784EF62020C0F634
:10082000010019464FF44062C4F202024FF0010386
:100830000CF046FE43F2D813C2F200035B784EF68A
:100840003020C0F6010019464FF44062C4F20202A3
:100850004FF002030CF034FE4EF6D160C0F60000FB
:1008600000F00AFD80BD00BF000000000000000095
:1008700080B582B000AF78604EF64020C0F601002F
:10088000796806F00DFB4FF44063C4F202037A6806
:1008900002F00102002A02D14FF4803201E04FF051
:1008A0000002796801F001010A439A6107F1080723
:1008B000BD4680BD80B582B000AF4EF65420C0F674
:1008C000010006F0EDFA4FF00100FFF7D1FF4FF005
:1008D000010003F015FE4FF0010006F039FD4FF462
:1008E000C8737B6021E07A6848F21F53C5F2EB13AE
:1008F00083FB02134FEA23114FEAE273CB1A4FF046
:10090000320101FB03F3D31A002B09D1786800F000
:1009100027FC49F2E030C0F2040003F0F1FD00E0F2
:1009200000BF7B6803F101037B607A6840F21453D7
:100930009A42CCBF00230123DBB2002BD3D14FF06E
:10094000000000F00DFC4FF0000006F001FD4FF03C
:100950000000FFF78DFF4FF0010003F0D1FD4EF6D0
:100960006420C0F6010006F09BFA07F10807BD46B7
:1009700080BD00BF80B582B000AF786040F29813B0
:10098000C1F200039A694EF67823C0F60103936121
:1009900003E04FF47A7003F0B3FD44F6E873C2F25B
:1009A00000031B68002B14BF00230123DBB2002BC4
:1009B000EFD144F6E873C2F200034FF000021A6070
:1009C000FFF778FF00BFE8E780B400AF44F6E873B4
:1009D000C2F200034FF001021A60BD4680BC7047AE
:1009E00080B586B002AF78603960386801F0DAFB14
:1009F00002460B46104619464FF000024FF0000326
:100A0000C4F2590301F05EFD02460B46104619463A
:100A100001F0F6FE03467868194611F029F8F860EF
:100A2000F86801F0D1FB02460B46CDE900234EF6F3
:100A30008020C0F6010079683A6806F031FA07F1C3
:100A40001007BD4680BD00BF80B582B002AF4EF634
:100A5000A420C0F601004FF44061C4F202014FF03F
:100A600000024FF001030CF05BFB4EF6A820C0F62D
:100A7000010040F67101C0F6000105F0B1FC4EF630
:100A8000B020C0F6010040F6C911C0F6000105F023
:100A90009FFC4EF6B420C0F6010040F6E111C0F60E
:100AA000000105F0A5FC4FF00100FFF7E1FE4FF05B
:100AB0000003009344F63050C2F200004FF42E7150
:100AC0004FF0400240F67513C0F6000303F0F0FC4F
:100AD000BD4680BD80B500AF0BF072F8FFF778FE21
:100AE00080BD00BF0000000000000000000000000A
:100AF00080B500AF45F2F400C2F200004FF00601ED
:100B000001F02EF80346042BD4BF00230123DBB2EF
:100B1000184680BD90B585B000AFF860B9607A60C6
:100B20003B607B685B68002B02D14FF0000334E030
:100B3000386801F06FFF0446FB689B68184601F0B7
:100B400069FF02467B681B691046194601F0B8FF31
:100B500003462046194602F06FF90346002B1AD0CF
:100B6000386801F057FF0446FB689B68184601F09F
:100B700051FF02467B685B691046194601F0A0FFF1
:100B800003462046194602F039F90346002B02D0ED
:100B90004FF0010301E04FF00003184607F114077E
:100BA000BD4690BD80B485B000AFF860B9607A6092
:100BB0007B685B68002B02D04FF0000312E0FB68FB
:100BC0001B78002B02D14FF001030BE0FB685A6841
:100BD000BB68D3F8143703F1FF339A42B4BF002344
:100BE0000123DBB2184607F11407BD4680BC7047ED
:100BF00080B588B000AFF860B9607A60FB707B6840
:100C00009B69002B02D0FB78002B06D17B689B6987
:100C1000002B05D1FB78012B02D04FF0010301E03E
:100C20004FF00003FB61FB69002B06D0FB685B689B
:100C300003F10102FB685A6045E0FB68DB68BA6AB1
:100C4000D31ABB61F868B9687A68FFF7ABFF03464F
:100C5000002B08D1F868B9687A68BB69FFF75AFFBA
:100C60000346002B02D04FF0010301E04FF00003D8
:100C7000002B1CD0FB685A68BB68D3F8143703F10B
:100C8000FF339A420CBF00230123DBB27B6145F2A4
:100C9000F400C2F20000796900F038FFFB684FF001
:100CA00001021A70FB684FF000025A6005E0FB6811
:100CB0005B6803F10102FB685A60FB68BA699A60DD
:100CC000FB68BA6ADA6007F12007BD4680BD00BF45
:100CD000B0B58AB000AFF860B9607A60F86812F019
:100CE00047FB4FF07C533B624FF000037B6263E0B5
:100CF000B86801F057FA02460B464FF000004FF477
:100D00000041C4F2860101F0DDFB02460B461446A9
:100D10001D46786A01F07EFE03461846396A01F0E6
:100D2000C5FD0346184601F04FFA02460B46204621
:100D3000294601F09DFA02460B461046194601F07D
:100D40005FFD0346FB61B86801F02CFA02460B46D2
:100D50004FF000004FF40041C4F2860101F0B2FBF5
:100D600002460B4614461D467B6A03F101031846F2
:100D700001F018FA02460B462046294601F078FA9F
:100D800002460B461046194601F03AFD0346BB6188
:100D9000F868F9694FF000024FF0010312F0F0FA21
:100DA000F868B9694FF000024FF0000312F0E8FA5A
:100DB0007B6A03F101037B62BA687B68D31A03F193
:100DC000FF327B6A9A42D4BF00230123DBB2002B9F
:100DD0008ED1B86801F0E6F902460B464FF00000EC
:100DE0004FF40041C4F2860101F06CFB02460B4651
:100DF00014461D46BA687B68D31A03F1FF331846C0
:100E000001F008FE03461846396A01F04FFD03461B
:100E1000184601F0D9F902460B462046294601F052
:100E200027FA02460B461046194601F0E9FC034634
:100E30007B61F86879694FF000024FF0010312F00E
:100E40009FFAF8684FF00001C4F234414FF00002FD
:100E50004FF0000312F094FA07F12807BD46B0BD29
:100E600080B586B000AFF860B9607A60FB6803F1C6
:100E70001C037B617869B9687A68FFF729FFBA6853
:100E80007B68D31A4FEA4302FB68C3F830277B69BB
:100E9000D3F810277B6903F597631046194612F0C3
:100EA000B7FA07F11807BD4680BD00BF80B582B014
:100EB00000AF7860786812F05BFA78684FF0000154
:100EC000C4F270214FF000024FF0010312F058FA03
:100ED00078684FF00001C4F252314FF000024FF039
:100EE000000312F04DFA78684FF00001C4F2D231DD
:100EF0004FF000024FF0010312F042FA78684FF40D
:100F00000041C4F21D414FF000024FF0000312F007
:100F100037FA78684FF00001C4F234414FF0000214
:100F20004FF0000312F02CFA7B684FF00402C3F874
:100F3000142707F10807BD4680BD00BF80B582B009
:100F400000AF7860786812F013FA7B684FF00A02FD
:100F5000C3F8142778684FF6EE41C4F256214FF0DB
:100F600001024FF0010312F00BFA78684CF6CD4104
:100F7000C4F2F3214FF001024FF0000312F000FA27
:100F800078684CF28F21C4F268314FF001024FF0C3
:100F9000010312F0F5F9786844F21F51C4F296315A
:100FA0004FF001024FF0000312F0EAF978684FF0B9
:100FB0000001C4F2B4314FF000024FF0010312F00F
:100FC000DFF978684EF6AC31C4F2CC314FF0010253
:100FD0004FF0010312F0D4F9786845F24431C4F2BD
:100FE000EF314FF001024FF0000312F0C9F97868B9
:100FF00040F2E121C4F213414FF001024FF001032E
:1010000012F0BEF9786844F2EC11C4F224414FF0BA
:1010100001024FF0000312F0B3F978684FF00001BD
:10102000C4F234414FF000024FF0000312F0A8F96F
:1010300007F10807BD4680BD80B584B000AF786079
:1010400039607B6803F62C43FB60FB681B68042B4C
:101050002BD801A252F823F06D1000089D10000853
:101060008F100008AB10000881100008FB689A6818
:10107000FB68DB68386811461A46FFF7F1FE20E08E
:101080003B6803F11C03184611F05AFF19E03B6856
:1010900003F11C031846FFF709FF12E03B6803F158
:1010A0001C031846FFF74AFF0BE04EF6C020C0F6BF
:1010B00001004EF6D021C0F601014FF0C10205F04B
:1010C000C7FE07F11007BD4680BD00BF80B500AF69
:1010D00044F6F070C2F200004EF6F821C0F60101AD
:1010E00007F026F880BD00BF80B582B000AF786001
:1010F00039607B68012B0AD13A684FF6FF739A4238
:1011000005D145F2F400C2F2000000F081FC7B68DA
:10111000002B0AD13A684FF6FF739A4205D145F287
:10112000F400C2F2000000F0B9FC07F10807BD4668
:1011300080BD00BF80B500AF4FF001004FF6FF71DA
:10114000FFF7D2FF80BD00BF80B500AF4FF00000B9
:101150004FF6FF71FFF7C8FF80BD00BF0000000021
:1011600080B584B000AF78607B68002B0AD143F271
:10117000D813C2F200034FF00002C7F6C072C3F8E2
:10118000182727E0786801F045FC024641F27823F1
:10119000C2F200031B68D3F8E03B1046194601F089
:1011A0008FFC034618464FF00001C4F2702101F095
:1011B0003BFD0346FB604FF4A040C4F2C370F968E6
:1011C00001F032FD03461A4643F2D813C2F200037F
:1011D000C3F8182745F23C10C2F200004EF6103159
:1011E000C0F601017A6807F05BF907F11007BD4608
:1011F00080BD00BF80B588B002AF786045F2402066
:10120000C2F2000000F004FD0346002B30D045F28E
:101210003C10C2F200004EF63831C0F6010107F072
:101220003FF941F27423C2F200031B6803F11C036F
:101230007B617B6903F10803FB607B6903F518732D
:101240003B617B69D3F810277B6903F5976307F14E
:101250000C010091786811461A464FF0020319F00C
:10126000EFFF7B684FF00002CBF68072C3F8EC29E9
:1012700007F11807BD4680BD90B58BB004AF78600C
:1012800045F23C10C2F200004EF65C31C0F601019E
:1012900006F04EFF41F27423C2F200031B6803F113
:1012A0001C037B614FF49660FFF75AFF7B6903F1E3
:1012B0000803FB607B6903F518733B617B69D3F816
:1012C00010277B6903F597644FF00203009307F141
:1012D0000C03019341F2F513C0F6000302937B68FF
:1012E00003934EF67830C0F6010043F2D811C2F2F3
:1012F000000123461AF00CF84EF68830C0F60100C3
:1013000041F26111C0F6000105F06AF807F11C070F
:10131000BD4690BD80B582B000AF786039607B6813
:10132000012B0AD13A684FF6FF739A4205D145F274
:101330004020C2F2000000F05BFC07F10807BD4648
:1013400080BD00BF80B500AF4FF001004FF6FF71C8
:10135000FFF7E0FF80BD00BF0000000000000000BC
:10136000B0B588B002AFF860B9607A607B681846A3
:1013700011F07EFD7C684FF0120011F051FA034627
:1013800020464FF001011A464FF0000311F078FD9E
:101390007C684FF0130011F043FA034620464FF0EB
:1013A00001011A464FF0000311F06AFD7C684FF00E
:1013B000140011F035FA034620464FF001011A4699
:1013C0004FF0000311F05CFD7C684FF0150011F048
:1013D00027FA034620464FF001011A464FF000035A
:1013E00011F04EFD7C684FF0120011F019FA03461F
:1013F00020464FF003011A464FF0000311F040FD64
:101400007C684FF0130011F00BFA034620464FF0B2
:1014100003011A464FF0000311F032FD7C684FF0D3
:10142000140011F0FDF9034620464FF003011A465F
:101430004FF0000311F024FD7C684FF0150011F00F
:10144000EFF9034620464FF003011A464FF0000320
:1014500011F016FD7C684FF0120011F0E1F903461F
:1014600020464FF006011A464FF0000311F008FD28
:101470007C684FF0130011F0D3F9034620464FF07B
:1014800006011A464FF0000311F0FAFC7C684FF099
:10149000140011F0C5F9034620464FF006011A4624
:1014A0004FF0000311F0ECFC7C684FF0150011F0D8
:1014B000B7F9034620464FF006011A464FF00003E5
:1014C00011F0DEFC7C684FF0120011F0A9F9034620
:1014D00020464FF008011A464FF0000311F0D0FCEF
:1014E0007C684FF0130011F09BF9034620464FF043
:1014F00008011A464FF0000311F0C2FC7C684FF05F
:10150000140011F08DF9034620464FF008011A46E9
:101510004FF0000311F0B4FC7C684FF0150011F09F
:101520007FF9034620464FF008011A464FF00003AA
:1015300011F0A6FCF868B9687A6812F069FD4FF0FE
:101540000003C4F27E337B614FF00003C4F29423A6
:101550003B617B6803F57273184611F089FC7B6868
:1015600003F572744FF00C0011F05AF903463A6912
:101570000092F868B968224612F032FC7B6803F5E5
:1015800072754FF00C0011F04BF9044638694FF0BA
:101590000001C4F2343101F089F903460093F86880
:1015A000B9682A46234612F01BFC7B6803F5727566
:1015B0004FF00C0011F034F9044638694FF0000187
:1015C000C4F2B43101F072F903460093F868B968C7
:1015D0002A46234612F004FC7B6803F572754FF02F
:1015E0000C0011F01DF9044638694FF00001C4F2F7
:1015F000074101F05BF903460093F868B9682A4691
:10160000234612F0EDFB07F11807BD46B0BD00BF41
:1016100080B48BB000AF78604FF000037B6210E0C5
:1016200040F60003C2F200037A6A53F822107B6886
:101630007A6A02F2C62243F822107B6A03F10103A0
:101640007B627B6A0F2BCCBF00230123DBB2002B14
:10165000E6D14FF000033B6210E040F64003C2F2D7
:1016600000033A6A53F822107B683A6A02F2D622E3
:1016700043F822103B6A03F101033B623B6A0F2BE4
:10168000CCBF00230123DBB2002BE6D14FF00003D7
:10169000FB6128E04FF00003BB6118E040F68003D7
:1016A000C2F20003FA694FEA0211BA698A1853F8C4
:1016B00022107B68FA694FEA0210BA69821802F5B3
:1016C000E37243F82210BB6903F10103BB61BB69FC
:1016D0000F2BCCBF00230123DBB2002BDED1FB6933
:1016E00003F10103FB61FB690F2BCCBF0023012336
:1016F000DBB2002BCED14FF000037B6112E040F64D
:101700008043C2F200037A6953F8222079687B692A
:1017100003F5D0734FEA8303CB185A607B6903F15A
:1017200001037B617B690F2BCCBF00230123DBB25C
:10173000002BE4D14FF000033B6112E040F6C043C0
:10174000C2F200033A6953F8222079683B6903F535
:10175000D8734FEA8303CB185A603B6903F1010346
:101760003B613B690F2BCCBF00230123DBB2002B75
:10177000E4D14FF00003FB602AE04FF00003BB60B0
:101780001AE040F60053C2F20003FA684FEA021171
:10179000BA688A1853F822207968FB684FEA031068
:1017A000BB68C31803F1A0034FEA8303CB185A6048
:1017B000BB6803F10103BB60BB680F2BCCBF0023E8
:1017C0000123DBB2002BDCD1FB6803F10103FB60DA
:1017D000FB680F2BCCBF00230123DBB2002BCCD145
:1017E00007F12C07BD4680BC704700BF80B588B0AC
:1017F00004AF78607B684FF00102A3F84A217B6850
:101800004FF47A72A3F84C217B6841F65832A3F862
:1018100048217B6803F5FA734FF48042C4F2035207
:10182000009248F63C62C4F2432201924FF000025B
:10183000C4F27A42029218464FF00001CCF2A01195
:101840004FF42042C4F28C6241F67843C4F2BF13D5
:1018500012F0CEFE7B684FF48042C4F24E52C3F8C1
:101860000C227B684FF00002C4F28222C3F854219C
:101870007B684FF08242C3F85C217B684FF0000226
:10188000C3F850217B684FF00002C4F2A012C3F8E5
:1018900058217B684FF00402C3F8D42B7B684FF0CB
:1018A0000202C3F8DC2B7B684FF00002C4F22F3237
:1018B000C3F8AC2B7B684FF00002C4F20C22C3F8D3
:1018C00004277B684FF00002C4F27E32C3F8AC2CD0
:1018D0007868FFF79DFE7B6840F22622A3F860211E
:1018E0007B684FF00002C4F28222C3F808274FF051
:1018F0000003FB6019E07A68FB6803F190034FEA8C
:101900008303D3184FF000025A607A68FB6803F132
:1019100098034FEA8303D3184FF00002CBF680728E
:101920005A60FB6803F10103FB60FB68072BCCBF27
:1019300000230123DBB2002BDDD17B684FF07E5208
:10194000C3F858227B684FF08142C3F878227B6845
:101950004FF42042C4F28C52C3F85C227B684FF0F3
:101960008142C3F87C227B684FF4A042C4F24362F8
:10197000C3F860227B684FF00002C3F880227B68C6
:101980004FF00102C3F82C2C7B684FF00002C3F823
:10199000302C7B684FF01402C3F8F02B7B684FF0BB
:1019A0000402C3F8F42B7B684FF00302C3F8F82B52
:1019B0007B684FF00002C3F8842C7B684FF0010273
:1019C000C3F8942C7B684FF00B02C3F88C2C7B6817
:1019D0004FF00102C3F8EC2107F11007BD4680BDAE
:1019E00080B582B000AF786039603B6803F11C02BB
:1019F0003B6803F5E763786811461A46FFF7B0FCC9
:101A000007F10807BD4680BD00000000000000008F
:101A100080B582B000AF78607B6818464FF0000157
:101A20004FF040021BF0E4FA7B684FF000021A64AA
:101A30007B684FF000025A647B68184607F108077C
:101A4000BD4680BD80B485B000AF786039603B682A
:101A50001A6C7B681A643B685A6C7B685A644FF056
:101A60000003FB600BE03B68FA6853F822107B68C8
:101A7000FA6843F82210FB6803F10103FB60FB687E
:101A80000F2BCCBF00230123DBB2002BEBD17B68F3
:101A9000184607F11407BD4680BC704780B483B078
:101AA00000AF78607B68184607F10C07BD4680BC24
:101AB000704700BF80B485B000AF786039603B6884
:101AC0001A6C7B681A643B685A6C7B685A644FF0E6
:101AD0000003FB600BE03B68FA6853F822107B6858
:101AE000FA6843F82210FB6803F10103FB60FB680E
:101AF0000F2BCCBF00230123DBB2002BEBD17B6883
:101B0000184607F11407BD4680BC704780B483B007
:101B100000AF786039607B681B6C03F101027B6861
:101B20001A647B681B6C102B14BF00230123DBB2EB
:101B3000002B03D07B684FF000021A647B681A6C9C
:101B40007B68396843F822107B685B6C03F1010203
:101B50007B685A6407F10C07BD4680BC704700BF24
:101B600080B487B000AF786039607B685A6C3B689E
:101B70009A42ACBF00230123DBB2002B02D07B686A
:101B80005B6C3B607B681B6CBB604FF000037B6150
:101B90004FF000033B6119E0BA683B69D31AFB6060
:101BA00003E0FB6803F11003FB60FB684FEAD373AB
:101BB000DBB2002BF5D17B68FA6853F822307A69E2
:101BC000D3187B613B6903F101033B613A693B68D0
:101BD0009A42ACBF00230123DBB2002BDCD17B692E
:101BE000184607F11C07BD4680BC70470000000086
:101BF00080B483B000AF78607B684FF000021A7049
:101C00007B68184607F10C07BD4680BC704700BFD3
:101C100080B584B000AF78600FF0A2FFF8607B68F9
:101C20001B781A46FB689A420ADAFB68002B0CBF45
:101C300000230123DAB27B681A704FF0010301E040
:101C40004FF00003184607F11007BD4680BD00BFE6
:101C500080B400AFBFF34F8F4FF46D42CEF200025D
:101C60004FF46D43CEF20003DB6803F4E0614FF004
:101C70000403C0F2FA530B43D360BFF34F8FFEE768
:101C800080B500AF45F24C30C2F2000045F2603141
:101C9000C2F200014FF0C8024FF0000303F020FD34
:101CA0000BF0FEF905F02CFA45F24420C2F20000D8
:101CB0004EF69031C0F6010106F03AFA4EF6983031
:101CC000C0F6010041F64551C0F6000104F080FB6A
:101CD0000AF096FA05F0ACFE0DF0D2FAFEF7FAFE25
:101CE00005F0EEFE4EF6A030C0F6010005F0D8F883
:101CF00045F24833C2F200034FF001021A6005F0CA
:101D0000DFFC4FF4FA7002F0FBFBF8E780B483B01D
:101D100000AF78607A6848F21F53C5F2EB1383FB7B
:101D200002134FEA63114FEAE273CB1A184607F128
:101D30000C07BD4680BC704780B500AFFFF788FF39
:101D400080BD00BF80B500AF45F24420C2F2000064
:101D50004EF6B431C0F6010106F0A2FB05F0B0FA70
:101D600045F22C40C2F200004AF22011C0F20701F5
:101D700041F63952C0F600024FF0000302F048F974
:101D800005F0BEFA80BD00BF80B584B000AFF8603A
:101D9000B9607A6005F07CFCF8680BF041FF45F211
:101DA0004833C2F200031B68002B10D14EF6D0302E
:101DB000C0F60100F968BA687B6805F071F848F26E
:101DC000A060C0F2010002F09BFB01F0A9FD07F149
:101DD0001007BD4680BD00BF80B500AF4EF6E430B1
:101DE000C0F601004EF6F831C0F601014FF0C20214
:101DF00001F07EFFFEE700BF80B500AF4EF6044065
:101E0000C0F601004EF6F831C0F601014FF0CA02EB
:101E100001F06EFFFEE700BF80B500AF4EF6184040
:101E2000C0F601004EF6F831C0F601014FF0D202C3
:101E300001F05EFFFEE700BF80B500AF4EF6284020
:101E4000C0F601004EF6F831C0F601014FF0DA029B
:101E500001F04EFFFEE700BF0FB480B582B000AFC7
:101E600045F22843C2F200031B78002B26D145F22D
:101E70002843C2F200034FF001021A7045F24C33BE
:101E8000C2F200034FF00002DA6007F114037B6036
:101E900045F24C30C2F2000039697A6803F090F9DB
:101EA00045F24C33C2F200035A6845F24C33C2F299
:101EB0000003DB68D3184FF000021A7007F108071F
:101EC000BD46BDE8804004B0704700BF80B400AF9D
:101ED00045F22013C0F233131846BD4680BC70474C
:101EE00080B500AF06F0BCFC01F07AFEFFF7C8FE3B
:101EF0004FF00003184680BD000000000000000005
:101F000081F0004102E000BF83F0004330B54FEAAA
:101F100041044FEA430594EA050F08BF90EA020F17
:101F20001FBF54EA000C55EA020C7FEA645C7FEAAA
:101F3000655C00F0E2804FEA5454D4EB5555B8BFCD
:101F40006D420CDD2C4480EA020281EA030382EA3E
:101F5000000083EA010180EA020281EA0303362DD0
:101F600088BF30BD11F0004F4FEA01314FF4801CA3
:101F70004CEA113102D0404261EB410113F0004FB5
:101F80004FEA03334CEA133302D0524263EB43036C
:101F900094EA050F00F0A780A4F10104D5F1200E0A
:101FA0000DDB02FA0EFC22FA05F2801841F1000165
:101FB00003FA0EF2801843FA05F359410EE0A5F139
:101FC00020050EF1200E012A03FA0EFC28BF4CF06A
:101FD000020C43FA05F3C01851EBE37101F0004520
:101FE00007D54FF0000EDCF1000C7EEB00006EEB2D
:101FF0000101B1F5801F1BD3B1F5001F0CD34908B7
:102000005FEA30004FEA3C0C04F101044FEA44520D
:1020100012F5800F80F09A80BCF1004F08BF5FEA94
:10202000500C50F1000041EB045141EA050130BD74
:102030005FEA4C0C404141EB010111F4801FA4F117
:102040000104E9D191F0000F04BF01460020B1FA6C
:1020500081F308BF2033A3F10B03B3F120020CDAA4
:102060000C3208DD02F1140CC2F10C0201FA0CF082
:1020700021FA02F10CE002F11402D8BFC2F1200CE7
:1020800001FA02F120FA0CFCDCBF41EA0C0190409D
:10209000E41AA2BF01EB0451294330BD6FEA0404E6
:1020A0001F3C1CDA0C340EDC04F11404C4F12002D1
:1020B00020FA04F001FA02F340EA030021FA04F3E3
:1020C00045EA030130BDC4F10C04C4F1200220FA3A
:1020D00002F001FA04F340EA0300294630BD21FA78
:1020E00004F0294630BD94F0000F83F4801306BF3E
:1020F00081F480110134013D4EE77FEA645C18BF32
:102100007FEA655C29D094EA050F08BF90EA020FC8
:1021100005D054EA000C04BF1946104630BD91EAC0
:10212000030F1EBF0021002030BD5FEA545C05D1C3
:102130004000494128BF41F0004130BD14F5800402
:102140003CBF01F5801130BD01F0004545F0FE4176
:1021500041F470014FF0000030BD7FEA645C1ABFAB
:10216000194610467FEA655C1CBF0B46024650EAE2
:10217000013406BF52EA033591EA030F41F400210E
:1021800030BD00BF90F0000F04BF0021704730B594
:102190004FF4806404F132044FF000054FF0000169
:1021A00050E700BF90F0000F04BF0021704730B52A
:1021B0004FF4806404F1320410F0004548BF4042FF
:1021C0004FF000013EE700BF42004FEAE2014FEA54
:1021D00031014FEA02701FBF12F07F4393F07F4F2F
:1021E00081F06051704792F0000F14BF93F07F4F61
:1021F000704730B54FF4607401F0004521F00041A4
:1022000020E700BF50EA010208BF704730B54FF029
:1022100000050AE050EA010208BF704730B511F02E
:10222000004502D5404261EB41014FF4806404F166
:1022300032045FEA915C3FF4DCAE4FF003025FEAE8
:10224000DC0C18BF03325FEADC0C18BF033202EB70
:10225000DC02C2F1200300FA03FC20FA02F001FACA
:1022600003FE40EA0E0021FA02F11444C1E600BF69
:1022700070B54FF0FF0C4CF4E06C1CEA11541DBF1C
:102280001CEA135594EA0C0F95EA0C0F00F0DEF8E7
:102290002C4481EA030621EA4C5123EA4C5350EACC
:1022A000013518BF52EA033541F4801143F480131D
:1022B00038D0A0FB02CE4FF00005E1FB02E506F0AE
:1022C0000042E0FB03E54FF00006E1FB03569CF003
:1022D000000F18BF4EF0010EA4F1FF04B6F5007F09
:1022E00064F5407404D25FEA4E0E6D4146EB06067B
:1022F00042EAC62141EA55514FEAC52040EA5E5004
:102300004FEACE2EB4F1FD0C88BFBCF5E06F1ED8AD
:10231000BEF1004F08BF5FEA500E50F1000041EBE4
:10232000045170BD06F0004646EA010140EA020091
:1023300081EA0301B4EB5C04C2BFD4EB0C0541EAB3
:10234000045170BD41F480114FF0000E013C00F3C8
:10235000AB8014F1360FDEBF002001F0004170BDEC
:10236000C4F10004203C35DA0C341BDC04F1140405
:10237000C4F1200500FA05F320FA04F001FA05F291
:1023800040EA020001F0004221F0004110EBD3705E
:1023900021FA04F642EB06015EEA430E08BF20EA8A
:1023A000D37070BDC4F10C04C4F1200500FA04F32D
:1023B00020FA05F001FA04F240EA020001F00041BF
:1023C00010EBD37041F100015EEA430E08BF20EA32
:1023D000D37070BDC4F1200500FA05F24EEA020E7A
:1023E00020FA04F301FA05F243EA020321FA04F0A9
:1023F00001F0004121FA04F220EA020000EBD37060
:102400005EEA430E08BF20EAD37070BD94F0000F5F
:102410000FD101F00046400041EB010111F4801F93
:1024200008BF013CF7D041EA060195F0000F18BF44
:10243000704703F00046520043EB030313F4801F80
:1024400008BF013DF7D043EA0603704794EA0C0F3A
:102450000CEA135518BF95EA0C0F0CD050EA410650
:1024600018BF52EA4306D1D181EA030101F00041CD
:102470004FF0000070BD50EA410606BF10461946F5
:1024800052EA430619D094EA0C0F02D150EA013601
:1024900013D195EA0C0F05D152EA03361CBF104642
:1024A00019460AD181EA030101F0004141F0FE41E1
:1024B00041F470014FF0000070BD41F0FE4141F465
:1024C000780170BD70B54FF0FF0C4CF4E06C1CEA65
:1024D00011541DBF1CEA135594EA0C0F95EA0C0F1A
:1024E00000F0A7F8A4EB050481EA030E52EA0335D5
:1024F0004FEA013100F088804FEA03334FF08055F6
:1025000045EA131343EA12634FEA022245EA111522
:1025100045EA10654FEA00260EF000419D4208BFD3
:10252000964244F1FD0404F5407402D25B084FEA80
:102530003202B61A65EB03055B084FEA32024FF42C
:1025400080104FF4002CB6EB020E75EB030E22BF89
:10255000B61A754640EA0C005B084FEA3202B6EB49
:10256000020E75EB030E22BFB61A754640EA5C00F8
:102570005B084FEA3202B6EB020E75EB030E22BF88
:10258000B61A754640EA9C005B084FEA3202B6EB89
:10259000020E75EB030E22BFB61A754640EADC0048
:1025A00055EA060E18D04FEA051545EA16754FEAAA
:1025B00006164FEAC30343EA52734FEAC2025FEAC8
:1025C0001C1CC0D111F4801F0BD141EA00014FF057
:1025D00000004FF0004CB6E711F4801F04BF014328
:1025E0000020B4F1FD0C88BFBCF5E06F3FF6AFAE44
:1025F000B5EB030C04BFB6EB020C5FEA500C50F1D4
:10260000000041EB045170BD0EF0004E4EEA113156
:1026100014EB5C04C2BFD4EB0C0541EA045170BD5D
:1026200041F480114FF0000E013C90E645EA060EA1
:102630008DE60CEA135594EA0C0F08BF95EA0C0FCF
:102640003FF43BAF94EA0C0F0AD150EA01347FF417
:1026500034AF95EA0C0F7FF425AF104619462CE7EE
:1026600095EA0C0F06D152EA03353FF4FDAE104651
:10267000194622E750EA410618BF52EA43067FF4A2
:10268000C5AE50EA41047FF40DAF52EA43057FF432
:10269000EBAE12E7000000000000000000000000A8
:1026A0004FF0FF3C06E000BF4FF0010C02E000BF1E
:1026B0004FF0010C4DF804CD4FEA410C7FEA6C5C01
:1026C0004FEA430C18BF7FEA6C5C1BD001B050EAA4
:1026D000410C0CBF52EA430C91EA030F02BF90EA8F
:1026E000020F0020704710F1000F91EA030F58BF4E
:1026F000994208BF90422CBFD8176FEAE37040F0B0
:10270000010070474FEA410C7FEA6C5C02D150EA4D
:10271000013C07D14FEA430C7FEA6C5CD6D152EA08
:10272000033CD3D05DF8040B704700BF84461046CD
:1027300062468C461946634600E000BF01B5FFF7CC
:10274000B7FF002848BF10F1000F01BD4DF808ED9C
:10275000FFF7F4FF0CBF012000205DF808FB00BF6D
:102760004DF808EDFFF7EAFF34BF012000205DF8C7
:1027700008FB00BF4DF808EDFFF7E0FF94BF012014
:1027800000205DF808FB00BF4DF808EDFFF7CEFF15
:1027900094BF012000205DF808FB00BF4DF808ED54
:1027A000FFF7C4FF34BF012000205DF808FB00BF25
:1027B0004FEA410212F5001215D211D56FF4787369
:1027C000B3EB625212D94FEAC12343F0004343EA0C
:1027D000505311F0004F23FA02F018BF40427047E7
:1027E0004FF00000704750EA013005D111F0004071
:1027F00008BF6FF0004070474FF00000704700BF07
:102800004FEA4102B2F1E04324BFB3F5001CDCF112
:10281000FE5C0DD901F0004C4FEAC0024CEA50704A
:10282000B2F1004F40EB830008BF20F00100704779
:1028300011F0804F21D113F13872BCBF01F000407C
:10284000704741F480114FEA5252C2F11802C2F1AE
:10285000200C10FA0CF320FA02F018BF40F001002F
:102860004FEAC1234FEAD32303FA0CFC40EA0C00E1
:1028700023FA02F34FEA4303CCE77FEA625307D11E
:1028800050EA01331EBF4FF0FE4040F44000704755
:1028900001F0004040F0FE4040F40000704700BFEF
:1028A00080F0004002E000BF81F0004142001FBF05
:1028B0005FEA410392EA030F7FEA226C7FEA236C0E
:1028C0006AD04FEA1262D2EB1363C1BFD218414003
:1028D00048404140B8BF5B42192B88BF704710F099
:1028E000004F40F4000020F07F4018BF404211F03C
:1028F000004F41F4000121F07F4118BF494292EAA4
:10290000030F3FD0A2F1010241FA03FC10EB0C00CF
:10291000C3F1200301FA03F100F0004302D549425C
:1029200060EB4000B0F5000F13D3B0F1807F06D309
:1029300040084FEA310102F10102FE2A51D2B1F101
:10294000004F40EBC25008BF20F0010040EA0300F6
:102950007047490040EB000010F4000FA2F10102A3
:10296000EDD1B0FA80FCACF1080CB2EB0C0200FA2D
:102970000CF0AABF00EBC25052421843BCBFD0407B
:102980001843704792F0000F81F4000106BF80F4F5
:1029900000000132013BB5E74FEA41037FEA226CB8
:1029A00018BF7FEA236C21D092EA030F04D092F083
:1029B000000F08BF0846704790EA010F1CBF0020B7
:1029C000704712F07F4F04D1400028BF40F0004014
:1029D000704712F100723CBF00F50000704700F034
:1029E000004343F0FE4040F4000070477FEA22625B
:1029F00016BF08467FEA23630146420206BF5FEA2C
:102A0000412390EA010F40F4800070474FF000032B
:102A100004E000BF10F0004348BF40425FEA000CF2
:102A200008BF704743F0964301464FF000001CE09A
:102A300050EA010208BF70474FF000030AE000BFF0
:102A400050EA010208BF704711F0004302D540422E
:102A500061EB41015FEA010C02BF844601460020A0
:102A600043F0B64308BFA3F18053A3F50003BCFABB
:102A70008CF2083AA3EBC25310DB01FA02FC634468
:102A800000FA02FCC2F12002BCF1004F20FA02F26F
:102A900043EB020008BF20F00100704702F1200262
:102AA00001FA02FCC2F1200250EA4C0021FA02F2C3
:102AB00043EB020008BF20EADC7070470000000012
:102AC0004FF0FF0C1CEAD0521EBF1CEAD15392EA11
:102AD0000C0F93EA0C0F6FD01A4480EA010C4002ED
:102AE00018BF5FEA41211ED04FF0006343EA501047
:102AF00043EA5111A0FB01310CF00040B1F5000F89
:102B00003EBF490041EAD3715B0040EA010062F137
:102B10007F02FD2A1DD8B3F1004F40EBC25008BF21
:102B200020F00100704790F0000F0CF0004C08BF3F
:102B300049024CEA502040EA51207F3AC2BFD2F10C
:102B4000FF0340EAC250704740F400004FF000031A
:102B5000013A5DDC12F1190FDCBF00F00040704754
:102B6000C2F10002410021FA02F1C2F1200200FA92
:102B700002FC5FEA310040F1000053EA4C0308BF59
:102B800020EADC70704792F0000F00F0004C02BFAA
:102B9000400010F4000F013AF9D040EA0C0093F025
:102BA000000F01F0004C02BF490011F4000F013B7F
:102BB000F9D041EA0C018FE70CEAD15392EA0C0FED
:102BC00018BF93EA0C0F0AD030F0004C18BF31F058
:102BD000004CD8D180EA010000F00040704790F02E
:102BE000000F17BF90F0004F084691F0000F91F0D2
:102BF000004F14D092EA0C0F01D142020FD193EA98
:102C00000C0F03D14B0218BF084608D180EA01001F
:102C100000F0004040F0FE4040F40000704740F0FB
:102C2000FE4040F4400070474FF0FF0C1CEAD052C9
:102C30001EBF1CEAD15392EA0C0F93EA0C0F69D025
:102C4000A2EB030280EA010C49024FEA402037D090
:102C50004FF0805343EA111143EA10130CF0004087
:102C60008B4238BF5B0042F17D024FF4000C8B4277
:102C700024BF5B1A40EA0C00B3EB510F24BFA3EB57
:102C8000510340EA5C00B3EB910F24BFA3EB910327
:102C900040EA9C00B3EBD10F24BFA3EBD10340EA81
:102CA000DC001B0118BF5FEA1C1CE0D1FD2A3FF6C7
:102CB00050AF8B4240EBC25008BF20F0010070477C
:102CC0000CF0004C4CEA50207F32C2BFD2F1FF031F
:102CD00040EAC250704740F400004FF00003013A50
:102CE00037E792F0000F00F0004C02BF400010F4F4
:102CF000000F013AF9D040EA0C0093F0000F01F008
:102D0000004C02BF490011F4000F013BF9D041EA29
:102D10000C0195E70CEAD15392EA0C0F08D142025C
:102D20007FF47DAF93EA0C0F7FF470AF084676E72F
:102D300093EA0C0F04D14B023FF44CAF08466EE708
:102D400030F0004C18BF31F0004CCAD130F00042D6
:102D50007FF45CAF31F000437FF43CAF5FE700BF2E
:102D60004FF0FF3C06E000BF4FF0010C02E000BF57
:102D70004FF0010C4DF804CD4FEA40024FEA4103F9
:102D80007FEA226C18BF7FEA236C11D001B052EAAF
:102D9000530C18BF90EA010F58BFB2EB030088BF75
:102DA000C81738BF6FEAE17018BF40F001007047E4
:102DB0007FEA226C02D15FEA402C05D17FEA236CC6
:102DC000E4D15FEA412CE1D05DF8040B704700BF0D
:102DD000844608466146FFE70FB5FFF7C9FF0028A4
:102DE00048BF10F1000F0FBD4DF808EDFFF7F4FFDD
:102DF0000CBF012000205DF808FB00BF4DF808ED76
:102E0000FFF7EAFF34BF012000205DF808FB00BF98
:102E10004DF808EDFFF7E0FF94BF012000205DF8BA
:102E200008FB00BF4DF808EDFFF7D2FF94BF01206B
:102E300000205DF808FB00BF4DF808EDFFF7C8FF64
:102E400034BF012000205DF808FB00BF0000000037
:102E50004FEA4002B2F1FE4F0FD34FF09E03B3EBA7
:102E600012620DD94FEA002343F0004310F0004FE7
:102E700023FA02F018BF404270474FF0000070473D
:102E800012F1610F01D1420205D110F0004008BFDC
:102E90006FF0004070474FF00000704700000000E6
:102EA00073B96AB9002908BF0028BCBF00204FF0E1
:102EB0000041C4BF6FF000414FF0FF3000F0C8B8D0
:102EC00082B0EC462DE9005000F092F8DDF804E005
:102ED00002B00CBC704700BF000000000000000002
:102EE00010B500210446FFF789FF20B92046BDE850
:102EF000104000F02DB804F1004000F029F84242E3
:102F000061EB41031046194610BD00BF00000000F0
:102F100038B50022002305460C46FFF721FC28B9EE
:102F200028462146BDE8384000F03AB8284604F16A
:102F3000004100F035F8424261EB4103104619466A
:102F400038BD00BF000000000000000000000000CD
:102F500070B5FFF739F900230022C3F6F053044699
:102F60000D46FFF785F900F07BF80646FFF70AF9F2
:102F700000230022C4F2F013FFF77AF902460B4651
:102F800020462946FEF7C0FF00F06AF800220243FF
:102F90001046314670BD00BF000000000000000078
:102FA000002370B50022C3F6F05304460D46FFF728
:102FB0005FF900F055F80646FFF7E4F80023002219
:102FC000C4F2F013FFF754F902460B462046294697
:102FD000FEF79AFF00F044F8002202431046314603
:102FE00070BD00BF000000000000000000000000F5
:102FF000F8B5164604460D461F4600F051F806FB8C
:1030000001F300FB0737A6FB0023FB18A21A65EBB0
:103010000303069CC4E90023F8BD00BFF8B51646BB
:1030200004460D461F4600F09BF900FB07F7A0FB86
:10303000062306FB0177FB18A21A65EB0303069C27
:10304000C4E90023F8BD00BF00000000000000003C
:10305000704700BF000000000000000000000000FA
:103060004A0011D212F5001211D20DD56FF4787307
:10307000B3EB62520ED44FEAC12343F0004343EA5C
:10308000505323FA02F070474FF00000704750EAA7
:10309000013002D14FF0FF3070474FF00000704711
:1030A00000292DE9F00F1D46C0F29D800024002D5F
:1030B000C0F2948080460F4694461E46E3BB8A4287
:1030C00055D9B2FA82F747B1C7F1200520FA05F6C3
:1030D00001FA07F1BA403143B840170CB1FBF7F6DB
:1030E000030C1FFA82FC07FB16110CFB06F543EAE2
:1030F00001439D4208D9711E9B1880F013819D42A7
:1031000040F21081023E9B18591BB1FBF7F507FBFB
:10311000151380B20CFB05FC40EA03418C4507D92E
:103120006B1E8A1880F00081944540F2FD80023DBC
:1031300045EA0641002503E08B420CD900252946CB
:103140000A462B4614B1524263EB4303104619461C
:10315000BDE8F00F7047B3FA83F5002D40F087808B
:103160008B4201D38242EAD800250121E8E712B957
:103170000126B6FBF2F2B2FA82F6002E39D18E1A8F
:10318000130C1FFA82FC0125B6FBF3F703FB176152
:103190004FEA10490CFB07F849EA0146B04506D949
:1031A000791EB61802D2B04500F2D3800F46C8EBA4
:1031B0000606B6FBF3F103FB116380B20CFB01FCC6
:1031C00040EA03439C4506D94E1E9A1802D2944504
:1031D00000F2C280314641EA0741B1E7E44352427E
:1031E00063EB430366E7404261EB41014FF0FF347C
:1031F0005DE7B240C6F1200921FA09F720FA09F586
:10320000130C01FA06F1B7FBF3F845EA01091FFABE
:1032100082FC03FB18774FEA19410CFB08F541EAE1
:103220000747B040BD420AD9BF1808F1FF3680F009
:103230008E80BD4240F28B80A8F10208BF18791B36
:10324000B1FBF3F503FB15171FFA89F90CFB05F623
:1032500049EA07418E4206D96F1E891871D28E4203
:103260006FD9023D89188E1B45EA08458CE7C5F1E8
:10327000200122FA01F306FA05F61E4327FA01F2AD
:103280004FEA164907FA05F720FA01F1B2FBF9F8FF
:103290000F433B0C1FFA86FA09FB18220AFB08FBB6
:1032A00043EA024293450CFA05FC08D9921908F149
:1032B000FF314AD2934548D9A8F102089219CBEBC5
:1032C0000203B3FBF9F109FB1132BFB20AFB01FAA9
:1032D00047EA02439A4506D94A1E9B1933D29A45BA
:1032E00031D902399B1941EA08410F0C1FFA8CF8B9
:1032F00008FB07F68AB24FEA1C4C08FB02F80CFBED
:10330000026202EB18420CFB07FC964288BF0CF5E8
:10331000803CCAEB03030CEB124C63450ED305D083
:1033200000250DE70E46EFE61D4601E71FFA88F877
:1033300000FA05F008EB0245A842F1D20139002558
:10334000FEE63D468FE71146CDE78846B7E7B04633
:1033500075E7023FB6182AE702393CE70000000093
:103360002DE9F007144605460E46002B3DD18A4252
:1033700049D9B2FA82F747B1C7F1200120FA01F228
:1033800006FA07F6BC401643BD40220CB6FBF2F02D
:103390002F0CA1B202FB106601FB00F347EA0646C0
:1033A000B34208D9471E361980F0F880B34240F284
:1033B000F58002383619F61AB6FBF2F302FB1362F7
:1033C000ADB201FB03F145EA0242914207D95E1E0C
:1033D000121980F0E580914240F2E280023B43EA1C
:1033E00000400021BDE8F00770478B4243D8B3FA94
:1033F00083F4002C42D18B4202D3824200F2DF8060
:1034000000210120EEE712B90127B7FBF2F4B4FA6C
:1034100084F2002A40F088800A1B230CA7B2012105
:10342000B2FBF3F603FB16224FEA154C07FB06F03E
:103430004CEA0242904207D9121906F1FF3C02D22F
:10344000904200F2CE806646121AB2FBF3F003FB04
:103450001023ADB207FB00F745EA03439F4207D9AB
:10346000421E1B1980F09E809F4240F29B800238D2
:1034700040EA0640B6E700210846B3E7C4F120065B
:1034800022FA06F503FA04F32B434FEA134C21FA10
:1034900006F501FA04F120FA06F6B5FBFCF746EA58
:1034A000010A1FFA83F80CFB17554FEA1A4108FB73
:1034B00007F941EA0545A94502FA04F203D97E1E3F
:1034C000ED187FD33746C9EB0501B1FBFCF60CFBC9
:1034D00016151FFA8AFA08FB06F84AEA05418845DC
:1034E00003D9751EC91873D32E4646EA0746370C12
:1034F0001FFA82FC0CFB07F5120CB3B20CFB03FCA9
:1035000002FB035303EB1C4302FB07F29D4288BFFF
:1035100002F58032C8EB010102EB134291424BD31A
:1035200042D0304600215DE79440C2F1200521FAE7
:1035300005F6230C20FA05F701FA02F1B6FBF3FCBD
:1035400039430D0CA7B203FB1C6645EA064607FB90
:103550000CF8B04500FA02F508D936190CF1FF3025
:103560003DD2B0453BD9ACF1020C3619C8EB06028E
:10357000B2FBF3F003FB10268AB242EA064207FBD5
:1035800000F1914206D9461E121926D2914224D941
:1035900002381219521A40EA0C4141E738460AE74C
:1035A00033461CE7104663E71FFA8CFC00FA04F070
:1035B0000CEB03439842B4D2701E002112E721465F
:1035C00020460FE7A9457FF67DAF023FED187AE769
:1035D000884589D9023EC91887E73046DAE784462C
:1035E000C4E7023E12192FE70000000000000000AF
:1035F000704700BFAFF30080AFF30080AFF30080EF
:10360000FEE700BFAFF30080AFF30080AFF30080B0
:1036100072B640F60004C2F2000484F309884EF644
:103620003473CEF200034FF040421A604EF68850D9
:10363000CEF20000016841F4700303604FF0000215
:10364000E1EE102A4EF63C70CEF2000002604FF020
:10365000060181F31488BFF36F8F8E4B8E4A9A4216
:103660001FD2A2F104038D48C11A21F0030240F2D7
:103670000000C2F2000010184FF05531C21AA2F13A
:103680000402C2F3800243F8041F834240F0F88032
:1036900007E003F10402596003F10803516083421B
:1036A000F7D17F4B7F48984220D2A0F10403E41A5F
:1036B000A4F1050424F0030440F20041C2F2000129
:1036C00060184FF05531C21AA2F10402C2F3800211
:1036D00043F8041F834240F0CA8007E003F104026C
:1036E000596003F1080351608342F7D114F070FC74
:1036F0006D4B6E48984225D200F104056C4C611B5D
:1037000021F003004FF0000340F60002C2F2000275
:1037100043F2E071C0F6020100F10404C0F380003E
:103720005D589D5003F10403A34240F0958009E0E9
:103730005858985003F104035858985003F1040363
:10374000A342F5D15B4B5C4A9A421ED2A2F104031C
:103750005A49C81A20F0030243F6E031C2F20001D0
:1037600050184FF00001C21AA2F10402C2F3800205
:1037700043F8041F834268D107E003F10402596053
:1037800003F1080351608342F7D1FFF731FF4C4B3F
:103790004C4898421ED2A0F10404A3F105031E1B5D
:1037A0004FEA960505F1010705F0010654F8041FDC
:1037B00088474FF00105BD423DD10BE004F10406FE
:1037C0006368984704F108047068804705F10205B2
:1037D000BD42F3D1FEF784FB3B493C4A8A421ED2EC
:1037E000A2F10404A1F105010F1B4FEA970606F1AF
:1037F000010706F0010654F8045FA8474FF00105E1
:10380000BD420ED10BE004F104066068804704F16C
:1038100008047168884705F10205BD42F3D1FFF73E
:10382000EFFE002EEFD054F8043F984705F1010554
:10383000BD42E8D1F3E7002EC0D054F8042F9047E2
:1038400005F10105BD42B9D1C4E7002A95D043F87E
:10385000041F834291D198E700283FF469AF58587C
:10386000985003F10403A3427FF462AF6AE7002A91
:103870003FF434AF43F8041F83427FF42FAF35E7A2
:10388000002A3FF406AF43F8041F83427FF401AFE0
:1038900007E700BF0004002000000020FB03002019
:1038A0000008002000040020FC1600200008002072
:1038B000FF160020B4A50120E03B0020AFA50120A9
:1038C00094010008880100089C0100089401000888
:1038D000FEE700BFAFF30080AFF30080AFF30080DE
:1038E000F8B5074645F24046C2F2000634464EF6A9
:1038F0004045C0F601050FCD0FC42B68237030463C
:10390000B9691AF05DF930464EF65441C0F601012E
:103910004FF02E0200F0ECF9F8BD00BFAFF30080CD
:1039200072B6FEE7AFF30080AFF30080AFF3008024
:1039300000F016FB00F04CFD00F0EAFA00DF00BFDB
:10394000EFF30982D2F8CC104EF63073CEF20003BA
:103950005960986800F16800986002F1680282F38B
:1039600009884FF0000383F311887047AFF300809C
:1039700008B54FF46D43CEF200034FF000029A6099
:103980004FF44070C0F2FA50D8604FF007004FF08B
:10399000100100F0F5F84FF00A004FF4007100F04C
:1039A000EFF84FF00B004FF0800100F0E9F808BD90
:1039B0004FF0200383F311884FF46D43CEF20003E0
:1039C000586810F4006F42D0EFF30983A3F1680246
:1039D00082F309884FF0807143F84C1C40F2981034
:1039E000C1F20000826992F8231059B140F2981197
:1039F000C1F20001086881689268914294BF002278
:103A000001220AE040F29810C1F2000001688868C3
:103A10009268904234BF0022012242B143F6311035
:103A2000C0F6000043F8500CF1EE10FA05E043F642
:103A30003C12C0F6000243F8502C4EF63072CEF223
:103A400000025168596641F00103536070474FF01E
:103A5000000383F311887047AFF30080AFF3008059
:103A600008B500F0D5F94FF0200383F3118800F07A
:103A700027FA00F0F5F800F0FBF94FF0000383F3AC
:103A8000118800F095F9FFF793FF08BDAFF30080B0
:103A90002DE9F04F2DED108AC1F80CD0D0F80CD0E4
:103AA000BDEC108ABDE8F08FAFF30080AFF300806B
:103AB00008B500F02DFA4FF0000383F31188284673
:103AC000A04700F075FD08BDAFF30080AFF30080A4
:103AD00070B44FEA90024FF46143CEF2000302F15A
:103AE000C00253F8226000F003044FEAC4044FF010
:103AF000FF0505FA04F526EA050501FA04F10D4370
:103B000043F822504FEA501200F01F004FF001011D
:103B100001FA00F002F1600143F8210043F82200AD
:103B200070BC7047AFF30080AFF30080AFF300804C
:103B300010B44FEA501200F01F034FF0010101FAD8
:103B400003F14FF46143CEF2000302F1200243F887
:103B500022104FEA900202F1C00253F8221000F046
:103B600003004FEAC0004FF0FF0404FA00F021EA1E
:103B7000000143F8221010BC704700BFAFF3008073
:103B800030B44FEA90024FF46D43CEF2000302F1DD
:103B9000060253F8225000F003004FEAC0004FF035
:103BA000FF0404FA00F425EA040401FA00F10C43CE
:103BB00043F8224030BC7047AFF30080AFF3008081
:103BC00040F29813C1F2000398694EF68042C0F6A5
:103BD00001028261FEE700BFAFF30080AFF3008017
:103BE00030B583B0FFF7C4FE00F082FA00F000FAAF
:103BF00001F04EF901F09CF940F20000C1F2000022
:103C00004FF0400100F0F4FB40F29815C1F20005BE
:103C1000A8614FF0010480F8204040F20043C2F256
:103C20000003C36100F0C4F94FF0000383F311886F
:103C300062B6AA694EF62071C0F601019161009347
:103C400040F25000C1F200004FF4A471224643F646
:103C5000C133C0F6000300F02BFC03B030BD00BF41
:103C60002DE9F04100F084F840F29813C1F200030E
:103C7000986990F823201AB102F1FF3180F82310DF
:103C8000436A03F10103436240F2B410C1F2000041
:103C9000C26802F10102C2600168814224D08C68CE
:103CA00004F1FF338B600C468A68EAB94FF00006D6
:103CB00040F2B415C1F200054FF02008E768E66055
:103CC00021684D6023682B6000F0D2F8334683F3FF
:103CD00011882069B847434683F3118800F0F0F853
:103CE0002C68A0680028E9D0BDE8F081AFF300801F
:103CF00070B506460D46144603F0D2FC98B945F25D
:103D00000853C2F200031D6045F21050C2F20000D9
:103D1000046045F21851C2F200010E603046294697
:103D20002246FEF731F870BDAFF30080AFF300809C
:103D300008B545F20C53C2F20003186830B945F2D9
:103D40001451C2F200010A68002A0BDC4EF69040C2
:103D5000C0F601004EF69841C0F601014FF0D202C4
:103D6000FFF7C6FF08BD00BFAFF30080AFF30080D0
:103D700008B545F20C53C2F200031868002806DBB0
:103D800045F21451C2F200010A68002A0BDC4EF61B
:103D9000B840C0F601004EF69841C0F601014FF060
:103DA000C402FFF7A5FF08BDAFF30080AFF30080AA
:103DB00008B54FF0200383F3118845F20C53C2F28B
:103DC00000031868002805DD45F21451C2F2000115
:103DD0000A685AB14EF6DC40C0F601004EF6984132
:103DE000C0F601014FF0B402FFF782FF45F20C5319
:103DF000C2F20003186800F1FF3119604FF00003B0
:103E000083F3118808BD00BFAFF30080AFF30080DB
:103E100008B54FF0200383F3118845F20C53C2F22A
:103E200000031868002805DB45F21451C2F20001B6
:103E30000A685AB14EF6E440C0F601004EF69841C9
:103E4000C0F601014FF0A602FFF752FF45F20C53F6
:103E5000C2F20003186800F1010018604FF000037F
:103E600083F3118808BD00BFAFF30080AFF300807B
:103E700008B545F20C53C2F200031868002806DDAD
:103E800045F21451C2F200010A68002A0BDC4EF61A
:103E9000EC40C0F601004EF69841C0F601014FF02B
:103EA0009902FFF725FF45F21453C2F200034FF0C9
:103EB0000000186008BD00BFAFF30080AFF30080C2
:103EC00008B545F20C53C2F200031868002805DD5E
:103ED00045F21451C2F200010A685AB14EF6F4409C
:103EE000C0F601004EF69841C0F601014FF08D0278
:103EF000FFF7FEFE45F21453C2F200034FF001003B
:103F0000186008BDAFF30080AFF30080AFF300800E
:103F100008B545F20C53C2F20003186830B945F2F7
:103F20001451C2F200010A68002A0BDC4EF614504C
:103F3000C0F601004EF69841C0F601014FF0810233
:103F4000FFF7D6FE45F21453C2F200034FF0000013
:103F5000186008BDAFF30080AFF30080AFF30080BE
:103F600008B545F20C53C2F20003186828B945F2AF
:103F70001451C2F200010A685AB14EF61C50C0F644
:103F800001004EF69841C0F601014FF07502FFF7AF
:103F9000AFFE45F21453C2F200034FF00100186067
:103FA00008BD00BFAFF30080AFF30080AFF3008027
:103FB00008B545F20C53C2F20003186828B945F25F
:103FC0001451C2F200010A685AB14EF63850C0F6D8
:103FD00001004EF69841C0F601014FF06A02FFF76A
:103FE00087FE08BDAFF30080AFF30080AFF3008021
:103FF00040F2B413C1F200035B601B604FF0FF326C
:104000009A604FF00000D860704700BFAFF30080A7
:10401000F8B505460C4616461F46FFF7A9FE0DB13A
:1040200006B15CB94EF65050C0F601004EF6605134
:10403000C0F601014FF05102FFF75AFE2F61EE600A
:1040400040F2B413C1F2000318688268944204D9A4
:10405000A41A00688268A242FAD3286041686960A5
:1040600045600D60AC6040F2B413C1F200039842A9
:1040700002D08268141B8460F8BD00BFAFF30080DB
:1040800010B50446FFF774FE5CB94EF68050C0F6DA
:1040900001004EF66051C0F601014FF06D02FFF7CE
:1040A00027FEE3685BB94EF69050C0F601004EF66D
:1040B0006051C0F601014FF07002FFF719FE206851
:1040C00040F2B412C1F20002904203D08168A368AA
:1040D000CA188260606821680160236862685A605B
:1040E0004FF00000E06010BDAFF30080AFF3008040
:1040F00040F29813C1F200035B601B604FF00002B6
:104100009A605B611B617047AFF30080AFF3008082
:1041100010B50446FFF72CFE94F820300BB10E2B9F
:104120000BD14EF6B050C0F601004EF6C451C0F6A9
:1041300001014FF05A02FFF7DBFD4FF0000084F859
:104140002000A16840F29813C1F200031B689A682E
:104150008A42FBD22360586860605C60046020463D
:1041600010BD00BFAFF30080AFF30080AFF300805D
:1041700010B504464FF0200383F31188FFF7A0FE2B
:1041800094F820300D2B1AD8DFE803F00719190E28
:1041900019131919191919191913FFF769FE4FF095
:1041A000000383F3118810BDA06A826802F1010246
:1041B0008260616823680B602068626842604FF02B
:1041C000FF31A1622046FFF7A3FFFFF751FE4FF03A
:1041D000000383F3118810BDAFF30080AFF30080BC
:1041E00038B50546FFF7A4FD40F29813C1F200036D
:1041F0009C6984F820504FF0140284F8232018683A
:10420000016819604B6098614FF0010380F820301D
:10421000ADF16402E069904202D92046FFF760FBED
:1042200040F29811C1F2000188692146FFF730FC85
:1042300038BD00BFAFF30080AFF30080AFF3008064
:1042400030B587B005460C46FFF772FDB4F1FF3F6D
:1042500015D001A8214644F27112C0F6000240F2C6
:104260009813C1F200039B69FFF7D2FE2846FFF7BF
:10427000B7FF049830B101A8FFF702FF02E028461B
:10428000FFF7AEFF40F29811C1F200018A69906A0F
:1042900007B030BDAFF30080AFF30080AFF3008014
:1042A00038B504460D46FFF743FDA56240F298136A
:1042B000C1F200039869A26881688A4203D8204647
:1042C000FFF726FF38BDFFF723FF054640F29810A1
:1042D000C1F2000084614FF0010384F82030ADF199
:1042E0006402E969914202D92846FFF7F9FA2046AB
:1042F0002946FFF7CDFB38BDAFF30080AFF3008058
:1043000010B540F29813C1F200039C691A68116855
:1043100019604B609A614FF0010082F820004FF065
:10432000140384F823302046FFF7F2FEADF1640257
:10433000E169914202D92046FFF7D2FA40F2981083
:10434000C1F2000080692146FFF7A2FB10BD00BF4B
:1043500010B540F29813C1F200039C691A68116805
:1043600019604B609A614FF0010082F820004FF015
:10437000000284F82020A1681B6898688842FBD856
:1043800023605A6862605C601460ADF16401E369A7
:104390008B4202D92046FFF7A3FA40F29810C1F2EF
:1043A000000080692146FFF773FB10BDAFF300806A
:1043B00008B5FFF7BDFC40F29813C1F200031A687C
:1043C000986991688368994201D9FFF7C1FF08BDD8
:1043D00008B540F29813C1F20003986990F82310D1
:1043E00011B9FFF78DFF08BDFFF7B2FF08BD00BF91
:1043F00010B481604FF0020280F820204FF00002DC
:1044000080F821204FF0140480F8234041640264B6
:10441000C26342624FF0010180F82210826140F2D3
:104420009812C1F200020261516941615061086154
:1044300000F12C02C26200F130014163016300F11E
:104440004C02C26110BC7047AFF30080AFF3008034
:10445000F8B504460D4616461F46FFF789FC2CB1F9
:10446000B5F59C7F02D37F2E00D85FB94EF6F05091
:10447000C0F601004EF60461C0F601014FF0A6023D
:10448000FFF736FCA5F164002118E1600F64E368D2
:10449000069A5A64E06843F6B121C0F6000101664D
:1044A00020463146FFF7A4FFF8BD00BFAFF3008000
:1044B000F0B583B007460E4615461C464FF0200364
:1044C00083F31188FFF74CFD089B00933846314673
:1044D0002A462346FFF7BCFF04464FF00001FFF7D2
:1044E000DFFEFFF715FD4FF0000383F31188204630
:1044F00003B0F0BDAFF30080AFF30080AFF30080F6
:1045000010B5044658B94EF65460C0F601004EF698
:104510000461C0F601014FF49372FFF7E9FB4FF01D
:10452000200383F31188FFF71BFD4FF0060021469F
:10453000FFF786FEFFF7ECFC4FF0000383F31188D2
:1045400010BD00BFAFF30080AFF30080AFF3008079
:1045500038B540F29813C1F200039C69A062254669
:1045600055F82C0FA84206D00168E162FFF7D0FD94
:10457000E06AA842F8D194F8210010F0030F05D1A9
:10458000636922691A612169606948614FF00E0010
:10459000FFF726FE4EF66460C0F601004EF6046199
:1045A000C0F6010140F28112FFF7A2FB38BD00BF47
:1045B00010B504464FF0200383F31188FFF7D0FCB9
:1045C0002046FFF7C5FF10BDAFF30080AFF30080BA
:1045D00038B504464FF0200383F31188FFF7C0FC81
:1045E00094F822305BB94EF6E860C0F601004EF652
:1045F000C461C0F601014FF04E02FFF779FB94F859
:10460000225005F1FF30C5B284F82250FFF780FC3C
:104610004FF0000383F3118805BB94F820100E2996
:104620001CD194F8212002F00303012B02D0022BAD
:1046300014D109E0606921690161236962695A61E5
:10464000204600F0D5FC38BD60692169016123690D
:1046500062695A61A06C214600F04AFD38BD00BF76
:1046600010B54FF0200383F31188FFF779FC40F277
:104670009813C1F200031C6994F8220000F10100B4
:1046800084F82200FFF744FC4FF0000383F3118805
:10469000204610BDAFF30080AFF30080AFF3008081
:1046A00038B505464FF0200383F31188FFF758FC17
:1046B0002C6940F29813C1F200039C4216D094F882
:1046C0002200FF280BD14EF64070C0F601004EF6D6
:1046D0005871C0F601014FF09602FFF709FB94F8FC
:1046E000221001F1010184F8221001E04FF00004D2
:1046F000FFF70EFC4FF0000383F311882846FFF705
:1047000067FF204638BD00BFAFF30080AFF30080E5
:1047100038B50D46044608B100290BDA4EF6807014
:10472000C0F601004EF69071C0F601014FF058023C
:10473000FFF7DEFA64602460A56038BDAFF3008047
:1047400010B50446FFF714FB5CB94FF24C00C0F6FD
:1047500001004EF69071C0F601014FF49972FFF717
:10476000C7FAA368002B03DB2068A04203D10EE048
:104770002168A1420BD14FF26000C0F601004EF655
:104780009071C0F601014FF49B72FFF7B1FAA26875
:1047900002F10102A260002A08DC2068036823609D
:1047A0005C604FF000018162FFF7B2FC10BD00BFFA
:1047B00010B5044658B94FF2F000C0F601004FF2B0
:1047C0000011C0F601014FF05802FFF791FA646042
:1047D00024604FF00003A36010BD00BFAFF3008062
:1047E00070B5054640F29813C1F200039C69FFF7CB
:1047F0009FFA5DB94FF22010C0F601004FF2001190
:10480000C0F601014FF07D02FFF772FAA868002898
:1048100000F08280A2688168914249D2826090F85B
:104820002020042A04D0052A1FD0002A34D03FE0DB
:10483000466802683260036841685960866A324699
:104840001268964204D0936881688B42F8D200E0E7
:10485000324602605368436050601860806A806826
:10486000A26881689142D9D322E04668016831602C
:10487000036842685A60866A32461268964204D0DB
:10488000936881688B42F8D200E032460260536838
:104890004360506018600BE04FF0010380F8203057
:1048A000426801681160036842685A60FFF730FC93
:1048B00028462B461B68984204D09968A26891420A
:1048C000F8D200E02B462360586860605C600460AA
:1048D000A5624FF00400FFF783FCAB68A3420BD046
:1048E0004FF23010C0F601004FF20011C0F6010186
:1048F0004FF0B202FFF7FCF9216CA94210D04FF241
:104900004410C0F601004FF20011C0F601014FF053
:10491000B302FFF7EDF970BDAC60206CE860256470
:1049200070BD00BFAFF30080AFF30080AFF3008035
:1049300010B504464FF0200383F31188FFF710FBF6
:104940002046FFF74DFFFFF7E3FA4FF0000383F334
:10495000118810BDAFF30080AFF30080AFF300808B
:1049600038B540F29813C1F200039D694FF020035F
:1049700083F31188FFF7F4FA286C58B94FF26C10E2
:10498000C0F601004FF20011C0F601014FF484722D
:10499000FFF7AEF9296C8A68AA420BD04FF280105B
:1049A000C0F601004FF20011C0F6010140F20B12F7
:1049B000FFF79EF92C6CE3682B642068A04219D0A5
:1049C000696C4BB11A689A4203D09068814238BF33
:1049D0000146DB68002BF5D1A960206801682160E1
:1049E0004C60A060026CE26004644FF00001FFF7CD
:1049F00057FC02E04FF00003A360FFF789FA4FF085
:104A0000000383F31188204638BD00BFAFF3008058
:104A100038B504460D46FFF7ABF95CB94FF21020EC
:104A2000C0F601004FF2D811C0F601014FF0FE02AE
:104A3000FFF75EF9E36B45EA0301E16394F82000B8
:104A4000082803D1A36A194206D138BD092809D123
:104A5000A26A11408A4205D12046FFF759FB4FF068
:104A60000001816238BD00BFAFF30080AFF300806A
:104A700070B505460E46FFF77BF95DB94FF234205D
:104A8000C0F601004FF2D811C0F601014FF0BC0290
:104A9000FFF72EF92C68A54209D0E3683343E360A1
:104AA0006068A168FFF7B4FF2468A542F5D170BD26
:104AB00010B50C4681B140F29813C1F20003996918
:104AC0008862086042684A60416011604FF00D00E2
:104AD0002146FFF7B5FB10BD4FF0FF3010BD00BF02
:104AE00010B4406000604FF0000484604161816157
:104AF000C1608A180261C361019B036210BC7047E8
:104B000070B50446FFF734F9E3686361A3614FF0C1
:104B10000000A06020682546A0420AD06FF0010680
:104B2000016821604D60FFF7F3FA86622068A842B1
:104B3000F6D170BDAFF30080AFF30080AFF300801B
:104B400038B504460D46FFF713F96369A26993422D
:104B500017D1A06878B914E0E36863612068A042C7
:104B60000CD0016821604C60FFF7D2FA4FF00002D0
:104B70008262104638BD6FF0030038BD4FF0000070
:104B800038BDA16801F10101A16003F8015B636117
:104B900022699342E0D2E1E7AFF30080AFF30080F7
:104BA00070B504460E464FF0200383F31188FFF7DB
:104BB000D7F9E3697BB1204698470CE0204631469F
:104BC000FFF776FF051E06DAFFF7A2F94FF00003A4
:104BD00083F3118814E0A0680028EFD000F1FF31C2
:104BE000A160A36913F8015BA3612269934224BF0A
:104BF000E368A361FFF78CF94FF0000383F311889A
:104C0000284670BDAFF30080AFF30080AFF30080A3
:104C10002DE9F84F04460F461D46C66992465AB91B
:104C20004FF28020C0F601004FF29421C0F601013E
:104C30004FF0E702FFF75CF84FF0200383F3118891
:104C4000FFF78EF907F10108BA444FF00007B946A3
:104C50004FF0200B76B12046B0470BE020462946A6
:104C6000FFF726FF30B1FFF753F94FF0000383F34E
:104C7000118821E0A368002BF0D003F1FF30A06081
:104C8000A16911F8012B08F8012CA161236999424F
:104C900024BFE168A161FFF73BF94B4683F311881C
:104CA00007F10107D04507D05B4683F31188FFF772
:104CB00057F908F10108CDE73846BDE8F88F00BF85
:104CC00040600060826041618161C160891801615A
:104CD000C361009B03627047AFF30080AFF30080B5
:104CE00070B50446FFF744F8E3686361A361226985
:104CF000D01AA06020682546A0420AD06FF00106B5
:104D0000016821604D60FFF703FA86622068A842BF
:104D1000F6D170BDAFF30080AFF30080AFF3008039
:104D2000F8B504460F4616464FF0200383F311886A
:104D3000FFF716F90CE020463146FFF7B9FE051ED5
:104D400006DAFFF7E5F84FF0000383F3118819E066
:104D5000A368002BEFD003F1FF30A060616901F878
:104D6000017B61612269914224BFE1686161E5696B
:104D70000DB12046A847FFF7CBF84FF0000383F3AF
:104D800011881D462846F8BDAFF30080AFF30080C0
:104D900038B50446FEF7ECFFA36962699A4214D164
:104DA000A06878B911E0E368A3612068A04207D049
:104DB000016821604C60FFF7ABF94FF0000282629E
:104DC000284638BD6FF0020038BDA16801F101012D
:104DD000A16013F8015BA36122699342E3D2E4E787
:104DE0002DE9F84F04460F469B46D0F81C80154627
:104DF0005AB94FF2B820C0F601004FF29421C0F624
:104E0000010140F29B12FEF773FF4FF0200383F382
:104E10001188FFF7A5F84FF00006B1464FF0200AC1
:104E20000BE020465946FFF743FE30B1FFF770F81C
:104E30004FF0000383F3118824E0A368002BF0D027
:104E400003F1FF30A06017F8012B616901F8012B15
:104E500061612369994224BFE1686161B8F1000F83
:104E600001D02046C047FFF753F84B4683F3118823
:104E700006F10106013D05D0534683F31188FFF783
:104E80006FF8DAE73046BDE8F88F00BFAFF3008077
:104E9000094A22F0070040F2C813C1F2000318606B
:104EA0004CF20001C2F2010121F0070240F2C410ED
:104EB000C1F2000002607047BBA50120AFF3008083
:104EC00010B50446FEF754FF04F1070323F0070171
:104ED00040F2C812C1F20002106840F2C413C1F2DD
:104EE00000031A68131A994206D8411840F2C812F2
:104EF000C1F20002116010BD4FF0000010BD00BFF4
:104F000010B504464FF0200383F31188FFF728F80B
:104F10002046FFF7D5FF0446FEF7FAFF4FF00003E7
:104F200083F31188204610BDAFF30080AFF30080FB
:104F300008B540F2D010C1F2000044F60173C0F68B
:104F4000000303604FF000018160C16000F11000B8
:104F5000FFF72EFC08BD00BFAFF30080AFF3008069
:104F600070B5064618B940F2D016C1F2000601F13C
:104F7000070525F0070506F1080406F11000FFF704
:104F8000D7FC1AE05A68954216D805F108019142FB
:104F900002D91A68226009E05A18186858505968EE
:104FA000A1F10801481B506022605D601C4644F876
:104FB000086BFFF7D5FC13E01C462368002BE1D1FA
:104FC000FFF7CEFC316849B105F108008847044677
:104FD00030B10660456004F1080401E04FF00004C0
:104FE000204670BDAFF30080AFF30080AFF30080C8
:104FF0002DE9F047074658B94FF20030C0F60100DE
:105000004FF2E021C0F601014FF0C602FEF770FE3C
:10501000A7F1080557F8080C00F1080600F1100088
:10502000FFF786FC34464FF2103AC0F6010A4FF201
:10503000E029C0F601094FF0D008AC420AD86368F5
:1050400003F10803E018854204D25046494642461F
:10505000FEF74EFEB44201D0AC4228D2216809B11D
:105060008D4224D247F8081C256057F8042C02F121
:105070000803E91857F8080C814208D1496852180A
:1050800002F1080247F8042CEB5847F8083C606826
:1050900000F10801621895420BD157F8043CC01882
:1050A00000F10800606057F8081C216001E02468E6
:1050B000C3E7FFF755FCBDE8F08700BFAFF3008002
:1050C00038B504460D46FEF753FE04B15DB94FF204
:1050D0007830C0F601004FF24031C0F601014FF0C8
:1050E0009902FEF705FE23682B60256038BD00BFDE
:1050F00038B505460C464FF0200383F31188FEF7C0
:105100002FFF28462146FFF7DBFFFEF701FF4FF098
:10511000000383F3118838BDAFF30080AFF3008044
:10512000F0B40746002B08BF0B4600F10B0007F157
:105130000A050E46B1FBF2F402FB141101F1300432
:10514000392CC8BF01F13704AC4605F80149B6FB5C
:10515000F2F1B3FBF2F3002BEBD1CCEB0002B81869
:105160006FEA0703C11801F001042A4612F8011F73
:105170003B4603F8011B834210D10DE002F101040C
:105180005278194601F8012B04F1010264785C7031
:1051900001F101038342F1D1F0BC7047002CEDD046
:1051A00012F8011F03F8011B8342E7D1F4E700BFA7
:1051B00008B54FF00003FFF7B3FF08BDAFF3008061
:1051C0002DE9F04F2DED048B8BB007460E461546AA
:1051D0004FF0000BDFED9A9A4CF6CD40CCF6CC4068
:1051E00002904FF2A033C0F601030393B04618F8C3
:1051F000011B002900F0ED81252905D03A6893684C
:10520000384698474646F1E771782D2903BF06F1E5
:10521000020801220192CDF804B098F800202E2A4D
:1052200001D0302A04D108F101084FF0300401E028
:105230004FF020044046D84610F8012B0646A2F154
:105240003003D9B2092904D92A2A07D1297805F1CE
:10525000040508EB880A01EB4A08EDE72E2A13D172
:105260000146DA4611F8012B0E46A2F13000C0B219
:10527000092804D92A2A08D1287805F104050AEB5F
:105280008A0600EB460AEDE7DA466C2A01D04C2A82
:1052900005D1307820B106F10106024600E0FFE7B3
:1052A000A2F14403342B00F21781DFE813F08100F0
:1052B00015011501150115018100150115011501D3
:1052C000150115010701150115011501150115013C
:1052D0000A0115011501350015011501150115010A
:1052E0001501150115011501150115013800810081
:1052F0001501970015011501810015011501150112
:1053000015011501070115011501150144001501CD
:105310000A011501150135004FF01002D3E02C6889
:105320000DF1280909F8184D05F104054FF0200486
:105330000DF11100E4E005F10404D5F80090B9F195
:10534000000F039D08BFA94647F6FF72BAF1000F90
:1053500008BF924699F80010002900F0C480BAF105
:10536000010F00F1C5804B4609EB0A056FEA090001
:10537000421902F0010103F10103184699F80120D6
:10538000002A40F04381B8E002F101031846527848
:10539000002A00F0B2801A4603F1010108465B784A
:1053A000002B40F04681A8E025464FF02004A7E0FE
:1053B000296805F10405002908DA4FF02D008DF861
:1053C0001000C1F100010DF1110000E004A84FF040
:1053D0000A02FFF7EDFE0DF1100991E005F1070556
:1053E00025F0070000F10805D0E90001FDF708FAF3
:1053F00009EE100AB4EEE99AF1EE10FA08D54FF072
:105400002D028DF81020B1EE499A0DF1110901E03D
:105410000DF1100919EE100AFCF7D6FE41EC180B3D
:1054200016F05EF870B94FF04E0189F800104FF099
:10543000610289F8012089F8021009F103003AE0BD
:105440000000000048F2A061C0F20101BAF1000FB3
:1054500008BF8A46BDEEC99A484619EE101A4FF0A9
:105460000A025B46FFF75CFE81464FF02E0309F807
:10547000013B19EE100AFCF795FE02460B4651EC73
:10548000180BFCF741FD41EC180B5046FCF77AFE77
:1054900002460B4651EC180BFCF7EAFEFDF788F9C3
:1054A00001460298A0FB0A2348464FF00A024FEA41
:1054B000D303FFF735FE0DF1100921E04FF008028C
:1054C00001E04FF00A02296805F1040504A8FFF77E
:1054D0006FFE0DF1100913E00DF1280909F8182DE0
:1054E0000DF111000CE0254648464FF0200407E07E
:1054F000254648464FF0200402E025464FF02004A0
:10550000C9EB000ACAEB080C2CEAEC78019B0BB93A
:10551000C8F10008B8F1000F2DDA99F800102D2914
:105520000BD1302C09D109F101093B689A68384642
:105530004FF02D0190470AF1FF3A6FEA080000F0A2
:10554000010101913B689A6838462146904718F15D
:10555000010843D136E03A689368384621469847B7
:1055600008F101083868826838462146904718F1EA
:105570000108F0D126E039680B68384649465246A2
:105580009847B8F1000F3FF431AE08F1FF3E0EF03E
:1055900001093A689368384621469847B8F10108EE
:1055A00028D123E639688B6838462146984708F1A8
:1055B000FF3838688268384621469047B8F10108BC
:1055C000F0D113E639680B68384649465246984789
:1055D0000CE60BB0BDEC048BBDE8F08F0198002801
:1055E000B9D039688B6838462146984718F10108C8
:1055F000B1D1E7E7B9F1000FD4D0386882683846F6
:1056000021469047B8F10108CCD1EFE51A46AB42EC
:105610003FF4CAAE00293FF4B7AE03F101010846DA
:105620005B78002B3FF469AF0A46A9427FF4ACAE29
:10563000BAE602F10102A9427FF4A6AEB4E600BFC9
:10564000C36882689A4208D04268D154C16801F1A7
:105650000101C1604FF0000070476FF0010070471A
:105660000369C2689A4206D04168CA5C03F101032B
:105670000361104670476FF001007047AFF3008080
:1056800038B504460369C568ED1AAA4238BF154605
:1056900042680846D1182A4617F002FC20694119D1
:1056A0002161284638BD00BFAFF30080AFF3008012
:1056B00038B50446C3688568ED1AAA4238BF154656
:1056C0004068C0182A4617F0EBFBE1684A19E2600F
:1056D000284638BDAFF30080AFF30080AFF3008001
:1056E00010B44FF2B034C0F601040460416082602F
:1056F000C3604FF00003036110BC7047AFF300803C
:1057000010B44B680A684FF00001C160C1610161CB
:1057100041610160416081604FF0FF340462C2F377
:105720004231072908BF00218161C2F3011404EB53
:10573000840102F00F0404EB4101C160C2F30031A7
:105740004FEA81046118C2F3032404EB410101F123
:10575000FF340461C2F3035101EB8104C2F303423D
:1057600002EB440101F164014161C3F3021404EB53
:10577000840203F00F0101EB42040460C3F3023220
:1057800002EB8204C3F3032101EB44024260C3F342
:10579000015404EB8404C3F380524FEA42018A1897
:1057A0004FEA820101EB4402C3F30343D118816045
:1057B00010BC7047AFF30080AFF30080AFF3008000
:1057C000F0B44FF000030B604B604269A2F1640239
:1057D0004CF6CD44CCF6CC44A4FB02454FEAD507A9
:1057E0004FEA075606F4700407EB8703A2EB430267
:1057F00044EA02470F608569002D08BF07254FEA7C
:10580000457647EA16450D60066906F101064CF635
:10581000CD43CCF6CC43A3FB06424FEAD2044FEA79
:10582000043707F4805704EB8402A6EB420647EAEC
:1058300006242C430C60C568A3FB05624FEAD20224
:105840004FEA021606F0300602EB8202A5EB420593
:105850002E4334430C608568A3FB05424FEAD20413
:105860004FEA045606F4401604EB8402A5EB420509
:1058700046EA05444C604568A3FB05624FEAD20244
:105880004FEA023606F4E04602EB8202A5EB420242
:1058900046EA022222434A600068A3FB00434FEA23
:1058A000D3034FEA031404F0700403EB8303A0EB6B
:1058B000430044EA00031A434A60F0BC704700BF4B
:1058C00010B584B00C464FF00003009301938DF89F
:1058D00008300393694604F083FA20466946FFF7CF
:1058E0000FFF04B010BD00BFAFF30080AFF3008026
:1058F00010B584B004464FF00003009301938DF877
:105900000830039308466946FFF75AFF2046694668
:1059100004F03EFA04B010BDAFF30080AFF3008096
:1059200000B58FB04FF000030A930B938DF8303021
:105930000D930AA904F054FA01A80AA9FFF7E0FEA2
:1059400001A817F0F5FC0FB000BD00BFAFF3008059
:1059500010B590B0044601914FF000030C930D93E5
:105960008DF838300F9301A803A917F091FA03A816
:105970000CA9FFF725FF20460CA904F009FA10B086
:1059800010BD00BFAFF30080AFF30080AFF3008025
:1059900070B504460E46154603680F2B0BD14FF227
:1059A000C030C0F601004FF2D431C0F601014FF013
:1059B0000D0201F04DFA206800F10102226004EBB3
:1059C00080014E6000F1100044F8205070BD00BF0F
:1059D00070B506460368002B0DDDA0F104044FF0FE
:1059E000000504F104046168206C884705F1010595
:1059F0003068A842F5DC70BDAFF30080AFF30080E3
:105A00002DE9F04106460F4690460368002B0EDD57
:105A1000A0F104054FF0000405F104056A6838465A
:105A20004146904704F101043068A042F4DCBDE82F
:105A3000F08100BFAFF30080AFF30080AFF30080D0
:105A400010B4002943DD034644184FF000006FF006
:105A5000270113F8012B504010F0800F0CBF4000BD
:105A600081EA4000C2B212F0800F0CBF520081EAFE
:105A70004202D0B210F0800F0CBF400081EA40001B
:105A8000C2B212F0800F0CBF520081EA4202D0B2C3
:105A900010F0800F0CBF400081EA4000C2B212F04B
:105AA000800F0CBF520081EA4202D0B210F0800F8A
:105AB0000CBF400081EA4000C2B212F0800F14BF58
:105AC00081EA42025200D0B2A342C2D101E04FF0BB
:105AD000000010BC704700BFAFF30080AFF3008040
:105AE00070B506460C4618F073F90546002816DD19
:105AF0003378A34216D033464FF0000015F0010F63
:105B000005D112E013F8011FA14215D170BD00F1BB
:105B1000010210469542F5D14FF0FF3070BD4FF0B5
:105B2000FF3070BD4FF0000070BD00F1010013F8B0
:105B3000012FA242EBD170BD02F1010013F8012F39
:105B4000A242E4D170BD00BFAFF30080AFF300808C
:105B500038B5044618F03CF9054658B322782D2A8A
:105B60000ED000282BDDA2F13003D8B2092829D8A5
:105B700023464FF00001084615F0010F0FD12BE02E
:105B800004F10100FFF7E4FFC0F1000038BD13F895
:105B9000014FA4F13002D2B2092A2DD917E000EB4F
:105BA0008000A2F1300202EB400001F101018D42C0
:105BB000EDD138BD44F23010C0F2AB0038BD4FF02B
:105BC000000038BD4BF6D060CFF6547038BD4BF6B0
:105BD000D060CFF6547038BD01EB8104A2F13002E1
:105BE00002EB440001F1010113F8012FA2F130048E
:105BF000E4B2092CD3D9EAE700EB8000A4F1300429
:105C000004EB400001F1010113F8012FA2F130046F
:105C1000E4B2092CC3D9DAE7AFF30080AFF3008018
:105C2000F8B5044618F0D4F8632855D845F21C5549
:105C3000C2F200052846214618F06AF828464FF0BF
:105C40002E01FFF74DFF0446B0F1FF3F07D1284674
:105C5000FFF77EFF02EE100AF8EEC22A3EE045F2A0
:105C60001C55C2F200054FF000032B542846FFF7E5
:105C70006FFF074604F101042D19284618F0A8F813
:105C8000064604462846FFF763FF002E15DDB2EEF8
:105C9000047A06F1FF3101F00102F0EE477A4FF08D
:105CA00001039E421DD10AE027EE870A60EE077AC3
:105CB00003F102039C42F7D101E0F7EE007A06EE11
:105CC000907AF8EEE60A06EE100AB8EEC61AC1EEB1
:105CD000271A70EEA12A01E0DFED062A12EE900AE3
:105CE000F8BD002AE0D067EE077A03F101039E4277
:105CF000DAD1E4E70000C07FAFF30080AFF30080AB
:105D00002DE9F84F2DED028B46F22055C2F2000529
:105D10002C464FF000024FF00003E4E8022305F5A3
:105D2000DF5505F11805A2469FED638B4FF0FF3854
:105D30006FF00049D3465AE9026730463946FCF70E
:105D400069FA53EC182BFCF793FAFDF7E1F8801988
:105D500041EB0701B94208BFB04206D14FF0010242
:105D60004FF00003801841EB0301B04271EB0703D1
:105D7000BCBF40464946CBE900010AF1080A5AE98E
:105D8000026730463946FCF745FA53EC182BFCF70E
:105D90006FFAFDF7BDF8801941EB0701B94208BF62
:105DA000B0427DD175E04FF0FF326FF000434449BF
:105DB000C1E904234FF00006354640F2E73845F2CA
:105DC0008059C2F200091CE007F1040B7E6005F166
:105DD000010A554652464FEAEA73824273EB0107C5
:105DE0000CDA0BF10407CBF804600AF101052A462E
:105DF0004FEAE573824273EB010A46DB664645458E
:105E000023DC06F1010CF4E802012A464FEAE573AF
:105E1000824273EB010BF1DA454516DC54E90201CD
:105E200005F1FF3709EB87036FEA050202F0010A6B
:105E300003F104075E6005F101052A464FEAE573A8
:105E4000824273EB010B0BDBD8E748F21811C2F268
:105E500000014FF001000860BDEC028BBDE8F88F37
:105E6000B5F57A7FF1D0BAF1000FADD047F8046FE5
:105E700005F101052A464FEAE573824273EB010AF8
:105E8000BCDAB5F57A7F9FD1DFE7B5F57A7F9BD194
:105E9000DBE74FF001024FF00003801841EB0301F4
:105EA000B04271EB0703BCBF40464946EAE8020135
:105EB000AA457FF43FAF76E7000000A09999A93F7B
:105EC00000810020AFF30080AFF30080AFF30080CB
:105ED000F8B504460D4648F21813C2F200031868DC
:105EE00058B94FF20040C0F601004FF21841C0F619
:105EF00001014FF03C02FDF7FBFE002C75F10003A1
:105F000037DBB4F57A7F75F1000C06DA45F2805084
:105F1000C2F2000050F82400F8BD45F28051C2F2F0
:105F20000001D1F89C1F40F27D32914224DC40F206
:105F30007E3646F22057C2F200078B194FEA630003
:105F400007EBC002D2E90023944275EB030C02DA9E
:105F500000F1FF3609E000F1010107EBC103D3E9CD
:105F60000023944275EB030C07DBB142E5DB0846E6
:105F7000F8BD4FF00000F8BD0846F8BDAFF3008053
:105F800038B504460D46084617F022FF0F2806D9FB
:105F90004FF22C40C0F601002946FBF75DFF20467A
:105FA000294617F0B5FE4FF000024FF00003C4E998
:105FB0000423C4E9062304F120004FF0000140F659
:105FC000FC5217F015F838BDAFF30080AFF3008036
:105FD000F8B5064614461D4610461946FFF778FFE9
:105FE0000746D6E90423A41845EB0305C6E9044592
:105FF000D6E906234FF001004FF00001121843EBE1
:106000000103C6E9062340F27E339F420BDD4FF2C7
:106010004C40C0F601004FF21841C0F601014FF0AC
:106020006302FDF765FE07F1080756F8272002F125
:10603000010246F82720F8BDAFF30080AFF30080DF
:106040002DE9F04F2DED028B85B081460391D0E90B
:106050000623062A73F100000EDA09F1200C46F23D
:106060002058C2F2000808F1080608F5E0584FF081
:10607000000081468A4623E0D9F820304FF000081E
:1060800093BB27E056E90245D6E90023121943EBFA
:1060900005034FEAD374121943F100035B104FEA72
:1060A000320247F8042F00F1010001F101015CF810
:1060B000042C8A42E6DC06F10806464500F0008121
:1060C0005CF8043B002BF6DD00F1FF340AEB84079B
:1060D0004946D7E709F120004FF0000808F1010810
:1060E00050F8043F002BF9D003990B604FF2F034C5
:1060F000C0F60104A4F10405019502914FF0000AD5
:106100004FF0000BD9E9066730463946FCF798FC9A
:10611000019A02F10402D2ED007A019207EE100A10
:1061200027EE270A10EE100AFCF7DAFE04460D46A9
:1061300054EA050004BF01240025BD4208BFB44253
:1061400006D14FF0FF304FF0FF31241845EB010529
:1061500008F1080259F822001AEB00024BEBE07339
:10616000A24273EB050014DA08F1080109EB810182
:1061700092469B4601E092469B4608F1010851F881
:10618000040F1AEB00024BEBE073A24273EB050025
:10619000F1DB4FEAD773F21847F100035B104FEAC7
:1061A0003202944275EB030120DA08F1080659F82F
:1061B00026701AEB07024BEBE773944275EB030072
:1061C00014DB08F1080109EB810692469B4601E0C9
:1061D00092469B4608F1010856F8040F1AEB00029C
:1061E0004BEBE073944275EB0300F1DA46F2205278
:1061F000C2F2000202EBC803D3E900673046394619
:10620000FCF71EFC08EE100AAB4508BFA2452BD0D8
:1062100046F22052C2F2000202EBC803D3E90201A7
:106220004FF0FF324FF0FF33801841EB0301801B2A
:1062300061EB0701B4EB0A0465EB0B0500FB05F30A
:1062400004FB0133A0FB0401591808F1080359F8B5
:10625000234022464FEAE473FCF722FEFCF7F0FBF2
:1062600007EE100A38EE078ABDEEC88A029918EECA
:10627000100A41F8040F0291019A144B9A427FF4DC
:1062800041AFD9F8181E51B909F6186940F27E30AD
:1062900000F1FF3059F8042D002AF9D001E040F256
:1062A0007E3046F22053C2F2000303EBC001D1E975
:1062B00002014FF0FF321218039802614FF00500FF
:1062C00005B0BDEC028BBDE8F08F00BFF8F301080C
:1062D00008B501464FF26040C0F6010000F0E0FD55
:1062E00008BD00BFAFF30080AFF30080AFF30080C4
:1062F0002DE9F84348F21C14C2F2000448F2E810F9
:10630000C2F200004FF27041C0F60101226802F0B3
:10631000C7F82368002B21DD4FF0000448F2EC257C
:10632000C2F2000548F2E819C2F200094FF28848AB
:10633000C0F6010848F21C17C2F2000704EB440241
:1063400005EB82064846414655F82220736802F064
:10635000A7F804F101043868A042EFDCBDE8F88337
:10636000F8B548F21C13C2F200031B68402B0CD195
:106370004FF29C40C0F601004FF2B841C0F6010157
:106380004FF0230200F064FDF8BD48F2EC26C2F2A3
:10639000000603EB43054FEA8505741903F1010379
:1063A00048F21C17C2F200073B6070516160A260A6
:1063B000F8BD00BFAFF30080AFF30080AFF3008003
:1063C00048F21C13C2F200034FF000021A6070473B
:1063D00008B50A464FF00001FFF7C2FF08BD00BF35
:1063E00008B50A464FF00101FFF7BAFF08BD00BF2C
:1063F00008B50A464FF00501FFF7B2FF08BD00BF20
:1064000008B50A464FF00301FFF7AAFF08BD00BF19
:1064100008B50A464FF00401FFF7A2FF08BD00BF10
:1064200008B50A464FF00201FFF79AFF08BD00BF0A
:10643000F8B504460D464368032B03D1816828460E
:106440008847F8BD042B20D108464FF02001FFF704
:1064500047FBB0F1FF3F4FD04FF000062E5400F144
:1064600001002E1830464FF02001FFF739FBB0F144
:10647000FF3F41D04FF00003335400F10102A36805
:1064800028463146B2189847F8BD052B19D1084661
:106490004FF02001FFF724FB0646B0F1FF3F2BD061
:1064A0004FF00000A8552846FFF752FB074606F1BB
:1064B00001016818FFF74CFB0146A2683846904777
:1064C000F8BD022B05D10846FFF7AAFBA368984741
:1064D000F8BD0846FFF73CFB4BF6D061CFF6547190
:1064E000884207D14FF2D440C0F60100294600F09F
:1064F000D7FCF8BDA2689047F8BD00BFAFF300809D
:10650000037863B1202B0DD04FF0000101E0202A69
:106510000AD001F10101425C002AF8D104E04FF0F9
:10652000000101E04FF0000108467047AFF3008022
:10653000F8B507460E4617F04BFC054604463046B4
:1065400017F046FC85421BD1002D1CDD3A783378CC
:106550009A421BD13B4631464FF0000215F0010F25
:1065600007D119E013F8015F11F8010F85421CD023
:106570000FE002F101029442F4D14FF00100F8BDA6
:106580004FF00000F8BD4FF00100F8BD4FF00000E3
:10659000F8BD4FF00000F8BD02F1010213F8015FF1
:1065A00011F8010F8542E4D0F3E702F1010213F87C
:1065B000015F11F8010F8542DBD0EAE7AFF30080FD
:1065C00008B548F2E810C2F200004FF2EC41C0F604
:1065D000010101F0ADFDFFF7F3FE4FF2F840C0F608
:1065E000010046F2F121C0F60001FFF7F1FE4FF283
:1065F0000050C0F6010046F2D121C0F60001FFF7BD
:10660000EFFE08BDAFF30080AFF30080AFF3008072
:1066100038B5044600283BD04FF20850C0F60100C0
:1066200021464FF0040217F003FC88BB04F104017B
:106630002379212B13D053B900E052B94FF21050F7
:10664000C0F6010000F02CFC4FF0000420E004F143
:106650000500044610F8012B212AEED100E00C467B
:106660004FF0000504F8015B0846FFF771FA054694
:10667000204617F0ADFB0246854209D04FF22C5060
:10668000C0F601002946234600F00AFC4FF0000442
:10669000204638BDAFF30080AFF30080AFF3008039
:1066A0002DE9F84FFFF7B4FF0546002800F0AC8055
:1066B00017F08EFB8146642807DD4FF26050C0F66C
:1066C000010000F0EDFBBDE8F88F48F22016C2F2A1
:1066D00000064FF27053C0F6010334460FCB07C4D7
:1066E00023803046294617F06BFA304617F070FBCE
:1066F0004FF66451C0F601010A8832522846FFF76E
:10670000FFFE814532D148F21C10C2F2000007683A
:10671000002F67DD48F2EC26C2F2000607F1FF32D7
:1067200002F0010AB04628463168FFF701FF002851
:106730006CD009E004EB440306EB8308284656F8C6
:106740002310FFF7F5FE18B1D8F80800804754E091
:1067500004F1010404EB440206EB8208284656F8D3
:106760002210FFF7E5FE00286AD0EDE705EB000AEE
:106770004FF000032B5448F21C10C2F20000D0F876
:106780000080B8F1000F2DDD48F2EC26C2F20006C1
:1067900008F1FF3707F0010B374628463168FFF74D
:1067A000C7FE002852D009E004EB440206EB820742
:1067B000284656F82210FFF7BBFE28B138460AF1EA
:1067C0000101FFF735FE18E004F1010404EB440178
:1067D00006EB8107284656F82110FFF7A9FE00288E
:1067E0004CD0EBE748F22010C2F20000494600F01E
:1067F00047FBFFF77DFDBDE8F88F48F22010C2F29D
:106800000000494600F03CFBBDE8F88F4FF0000463
:1068100004F10104BC42E5D0BAF1000F8AD004EBC8
:10682000440806EB88082846D8F80010FFF780FED9
:10683000002889D104F10104BC427FF47BAFD1E789
:1068400004F10104BC427FF475AFCBE74FF00004C4
:1068500004F101044445C5D0BBF1000FA4D004EB02
:10686000440106EB810728463968FFF761FE0028DE
:10687000A4D104F10104444596D1B3E704F1010425
:10688000444591D1AEE700BFAFF30080AFF3008085
:1068900030B585B0044641F65833A0F848314FF082
:1068A0000205C0F89C5B4FF47040C4F2EB500090BE
:1068B0004FF00001C4F2C82101914FF00002C4F270
:1068C0002F42029204F5FA704FF000014FF4684233
:1068D000C4F2FD624FF00003C4F2F0130DF088FE25
:1068E0004FF40043C4F20953C4F80C324CF6CD40C7
:1068F000C4F21620C4F854014FF00001C4F2A00104
:10690000C4F85C114FF00002CCF22022C4F85021F0
:106910004FF00003C4F2D013C4F8583104F63C40E1
:1069200047F2BD41C3F61371016004F5446349F6B3
:10693000B252C3F66F721A604FF00100C4F8300C07
:106940004FF00001C4F8441CC4F82C5CC4F8D80B08
:10695000C4F8DC5B05B030BDAFF30080AFF300805E
:106960002DE9F8430C4601F5E7600CF081FA04F6D6
:106970001C1528460CF07CFA4FF015000BF050FF68
:1069800002464FF00009C4F24C2928464FF000019E
:106990004B460CF075FA4FF013000BF041FF024626
:1069A0004FF00008C4F2673828464FF00001434614
:1069B0000CF066FA4FF012000BF032FF02464FF473
:1069C0000047C4F2CD3728464FF000013B460CF09B
:1069D00057FA4FF014000BF023FF02464FF44046E5
:1069E000C4F2134628464FF0000133460CF048FA33
:1069F00004F5306420460CF03BFA4FF00C000BF02D
:106A00000FFF024620464FF000014B460CF038FACB
:106A10004FF00D000BF004FF024620464FF000013E
:106A200043460CF02DFA4FF00E000BF0F9FE024633
:106A300020464FF000013B460CF022FA4FF00F00C9
:106A40000BF0EEFE024620464FF0000133460CF0FC
:106A500017FABDE8F88300BFAFF30080AFF3008002
:106A600041F65833A0F8483100F53E614FF07E52B0
:106A70000A604FF02403C0F8343C4FF00101C0F825
:106A8000381C4FF00202C0F8D82BC0F8DC2B70473E
:106A90002DE9F04180460C4601F5E7664FF0120003
:106AA0000BF0BEFE02464FF0000530464FF00001ED
:106AB0002B460CF0E5F94FF013000BF0B1FE024647
:106AC0004FF00007C4F2B43730464FF000013B46A8
:106AD0000CF0D6F904F61C164FF012000BF0A0FED5
:106AE000024630464FF000012B460CF0C9F94FF03A
:106AF00013000BF095FE024630464FF000014FF0B8
:106B00000003C4F234330CF0BBF904F530664FF0E7
:106B10000D000BF085FE024630464FF000012B467B
:106B20000CF0AEF94FF00D000BF07AFE0246304645
:106B30004FF000013B460CF0A3F9404621460DF012
:106B4000D7F9BDE8F08100BFAFF30080AFF300805C
:106B50002DE9F04F85B004464FF00606C0F8D46B1F
:106B600000F53E634FF07C5119604FF00005C0F80E
:106B7000D85B4FF00502C0F8DC2B0BF009F8C4F825
:106B8000346CC4F8385CC4F8305C4FF00100C4F8D1
:106B9000440CC4F8485C48F68058C4F61C084FF012
:106BA0000007C4F270274FF4204BC4F2F05BCDF81D
:106BB00000B04FF0000AC4F2F02ACDF804A04FF460
:106BC0000049C4F29349CDF8089004F5FA704FF0EB
:106BD0000001CCF2201142463B460DF009FD4FF476
:106BE0004046C4F22856C4F80C62CDF800B0CDF887
:106BF00004A0CDF8089004F507704FF00001CCF226
:106C0000201142463B460DF0F3FCC4F834624FF0CD
:106C10000701C4F8F81BC4F88C5C4FF00B03C4F8F0
:106C2000903C4FF0C102A4F84A214FF43070A4F810
:106C30004C014FF00201C4F8EC11C4F8F01105B09A
:106C4000BDE8F08FAFF30080AFF30080AFF30080BA
:106C500008B50DF04DF908BDAFF30080AFF300802B
:106C6000704700BFAFF30080AFF30080AFF3008048
:106C70004FF00403C0F82C3C4FF00101C0F8301C69
:106C800000F63C434BF22D22C3F69D521A6000F5EC
:106C9000446146F69763C3F612630B604FF000023F
:106CA000C0F8442C00F6AC304FF00001C4F2A03123
:106CB00001607047AFF30080AFF30080AFF3008056
:106CC000704700BFAFF30080AFF30080AFF30080E8
:106CD0004FF01803C0F8343C4FF00201C0F8381CE4
:106CE000704700BFAFF30080AFF30080AFF30080C8
:106CF00010B501F5306420460CF0BAF84FF00C00E6
:106D00000BF08EFD024620464FF000014FF00003CD
:106D1000C4F220130CF0B4F84FF00C000BF080FD1F
:106D2000024620464FF000014FF00003C4F23E330C
:106D30000CF0A6F84FF00C000BF072FD0246204656
:106D40004FF000014FF00003C4F2B9330CF098F893
:106D50004FF00F000BF064FD024620464FF000019B
:106D60004FF40043C4F209430CF08AF810BD00BF91
:106D700042F22833A0F848314FF44871A0F860116E
:106D800000F53B6348F65C72C3F6C2721A604FF0BE
:106D90000203C0F8B43B00F6AC324FF00001C4F27D
:106DA00070111160A0F84E314FF00103C0F8D43BD0
:106DB00000F53E624FF07E511160C0F8DC3BC0F838
:106DC000343C4FF00003C0F8383CC0F8303CC0F809
:106DD000483C7047AFF30080AFF30080AFF3008012
:106DE000704700BFAFF30080AFF30080AFF30080C7
:106DF0004FF00603C0F8D43B4FF00001C0F8D81B99
:106E00004FF00402C0F8342CC0F8381CC0F8301C15
:106E1000704700BFAFF30080AFF30080AFF3008096
:106E2000704700BFAFF30080AFF30080AFF3008086
:106E300008B54FF28050C0F601004FF29051C0F6F5
:106E400001014FF02E02FCF753FF08BDAFF30080A5
:106E500070B503460E46154648F2EC54C2F20004E3
:106E60002046194616F054FF204631462A46FCF7C4
:106E70003FFF70BDAFF30080AFF30080AFF3008041
:106E800008B502460B4648F2B460C2F2000041F673
:106E90000C41C0F6020101F003FB08BDAFF3008016
:106EA0000FB400B583B006F07BFF40B105AA019294
:106EB00044F6B840C2F201000499FEF781F903B02C
:106EC0005DF804EB04B07047AFF30080AFF30080CF
:106ED0002DE9F04184B04FF2A850C0F60100FFF751
:106EE000DFFFFDF7BDFB04464FF2D858C0F601089E
:106EF0004FF65017C0F601074FF00006656AA36809
:106F000094F8222002F1FF30009094F8201057F8F6
:106F1000212001920295A069039040462146324605
:106F2000FFF7BEFF2046FDF7BBFB04460028E5D176
:106F300004B0BDE8F08100BFAFF30080AFF3008084
:106F400038B54FF20060C0F60100FFF7A9FFFAF76D
:106F5000BDFF024648F2B464C2F2000420464FF27C
:106F60004861C0F6010101F0E3FA4FF25C60C0F63F
:106F700001004FF27C61C0F60101FFF791FF4FF273
:106F80008460C0F60100FFF78BFF4FF2B060C0F6DF
:106F900001004FF2C061C0F60101FFF781FF2046FA
:106FA0004FF20471C0F6010148F2A062C0F2010282
:106FB00001F0BEFA20464FF21471C0F601014FF401
:106FC000E13201F0B5FA20464FF22471C0F601011A
:106FD00046F64072C0F2401201F0AAFA4FF43D4565
:106FE000C0F2015520464FF23471C0F601012A4625
:106FF00001F09EFA20464FF24871C0F601014FF4AD
:10700000F442C0F6032201F093FA20464FF25C717D
:10701000C0F601014DF68062C0F2802201F088FACC
:1070200020464FF26C71C0F601012A4601F080FA49
:1070300020464FF27C71C0F601014FF0010201F0D1
:1070400077FA20464FF29871C0F601014FF0010225
:1070500001F06EFA20464FF2AC71C0F601014FF01C
:10706000010201F065FA20464FF2CC71C0F6010131
:107070004FF0010201F05CFA20464FF2EC71C0F6CD
:1070800001014FF0010201F053FA20464FF60401CE
:10709000C0F601014FF0010201F04AFA20464FF616
:1070A0001801C0F601014FF0010201F041FA20463B
:1070B0004FF63801C0F601014FF0000201F038FA36
:1070C00020464FF65801C0F601014FF0000201F0D2
:1070D0002FFA20464FF67801C0F601014FF0010269
:1070E00001F026FA20464FF69401C0F601014FF058
:1070F000010201F01DFA4FF4FA70FDF701FA38BDF4
:1071000008B501F085FAFFF75BFA46F2A160C0F618
:10711000000000F0B5F848F2B460C2F200004FF28F
:10712000F041C0F6010101F003F8FFF709FF4FF647
:10713000A800C0F6010046F64171C0F60001FFF755
:1071400047F94FF6B000C0F6010046F63161C0F6CF
:107150000001FFF73DF94FF6B800C0F6010046F612
:10716000D161C0F60001FFF733F908BDAFF300802D
:1071700008B544F6B843C2F201031A68C1B2926876
:107180001846904708BD00BFAFF30080AFF3008002
:107190002DE9F84340F29813C1F2000398694FF6C5
:1071A0009012C0F60102826141F20016C2F200069E
:1071B0004FF47A7744F6B845C2F20105B04606F1BD
:1071C0004E0902E0464600E0464606F0E9FD18B9E1
:1071D0003846FDF795F9F8E72968CC682846A047B6
:1071E000044683B213F4004FECD118B20428EBD05C
:1071F00008280FD14645E8D0E4B22046FFF7B8FF93
:107200004FF02000FFF7B4FF2046FFF7B1FF06F173
:10721000FF36DAE71AB20D2A13D14FF00D00FFF74F
:10722000A7FF4FF00A00FFF7A3FF4FF000043470F0
:1072300048F6F036C2F200063368404698474646A4
:10724000C3E719B21F29C0DD4E45BED2E0B2FFF739
:107250008FFF06F8014BB8E7AFF30080AFF3008073
:1072600010B504460A4644F6B840C2F2010003686D
:107270001B682146984710BDAFF30080AFF3008034
:1072800000B583B048F6F033C2F20003186006F090
:107290002FFD4FF00000009048F2B870C2F20000DD
:1072A0004FF487614FF0400247F29113C0F600039C
:1072B000FDF7FEF803B000BDAFF30080AFF3008030
:1072C00008B501F025FA30B14FF0200383F311889F
:1072D000FCF7F6FD08BD4FF0200383F31188FCF79F
:1072E0003FFE08BDAFF30080AFF30080AFF3008036
:1072F00008B5FFF7E5FF08BDAFF30080AFF30080EE
:1073000008B501F005FA30B1FCF7B2FD4FF000030B
:1073100083F3118808BDFCF7FBFD4FF0000383F3F6
:10732000118808BDAFF30080AFF30080AFF3008099
:1073300008B5FFF7E5FF08BDAFF30080AFF30080AD
:1073400049F29053C2F200034FF001021A607047F5
:1073500010B5044620B14FF6A011C0F6010103E0BC
:107360004FF6A411C0F601014FF6A810C0F60100B7
:10737000FFF796FD49F29450C2F2000041F60C412D
:10738000C0F602014FF6C412C0F60102234601F016
:10739000CFF841F25413C2F200031C6010BD00BFCD
:1073A00008B541F2883400F0DBFD2046FDF7A8F86F
:1073B000F9E700BFAFF30080AFF30080AFF30080C8
:1073C000F0B52DED048B85B0064607EE901AF8EE69
:1073D000E78A9FED358AC8EE888A18EE901A0AF07F
:1073E0002FFA05460DF0ACF90AF0E2F904460DF06B
:1073F000E7F80AF0C5F907460CF092FF0AF0F0F939
:1074000009EE100A2846FAF7DFFE02460B464FF651
:10741000C810C0F60100FFF743FD2046FAF7D4FE7E
:1074200004460D463846FAF7CFFECDE9000129EEB5
:10743000080AFDEEC00ACDED020A4FF6D810C0F6DC
:10744000010022462B46FFF72BFD304618EE901A1E
:107450000AF02EFA09EE100A18EE900AFAF7B4FEB6
:1074600002460B4629EE081ABDEEC18A8DED008A50
:107470004FF60C20C0F601003146FFF711FD19EE62
:10748000100AFAF7A1FE02460B4649F28C40C2F2FE
:1074900000004FF62C21C0F6010101F001F805B003
:1074A000BDEC048BF0BD00BF0000C842AFF300800C
:1074B00070B5054610EE106A0C4649F29450C2F2BF
:1074C0000000294610EE102A234601F051F849F237
:1074D0007C30C2F2000029463246234601F048F8CB
:1074E00070BD00BFAFF30080AFF30080AFF300804A
:1074F00008B549F29450C2F2000000F0E9FD08BD61
:1075000070B549F27C36C2F20006304600F0C8FD84
:1075100040F2B413C1F20003DA6848F21F50C5F21A
:10752000EB10A0FB02144FEA541107EE901AB8EECC
:10753000E70A4FF64020C0F60100DFED510A80EE69
:10754000200A4FF00301FFF7B3FF13F069FC044674
:107550004FF64825C0F6010549F29450C2F20000EA
:107560002946224601F01CF830462946224601F001
:1075700017F80CF0EDFD00EE100A4FF64C20C0F6A7
:1075800001004FF00201FFF793FF41F27423C2F2B2
:1075900000031A68106868B14FF0050000F040FD64
:1075A00004460AF075F800EE100A20464FF002017A
:1075B000FFF77EFF0CF054FE00EE100A4FF650204D
:1075C000C0F601004FF00201FFF772FF0CF080FEE1
:1075D00000EE100A4FF65420C0F601004FF00201F1
:1075E000FFF766FF0CF09CFE00EE100A4FF65C20E1
:1075F000C0F601004FF00201FFF75AFF4FF0030001
:1076000000F00EFD04460CF093FD00EE100A20463B
:107610004FF00201FFF74CFF41F27421C2F200016A
:107620000B685A686AB14FF0010000F0F9FC04469B
:107630000CF0C6FF00EE100A20464FF00201FFF7E3
:1076400037FF4FF0020000F0EBFC04460DF078F835
:1076500000EE100A20464FF00201FFF729FF49F221
:107660007C34C2F2000420464FF67831C0F60101A6
:1076700000F08EFED4F8F40007F02AF970BD00BFC8
:1076800000007A44AFF30080AFF30080AFF30080D6
:1076900008B54FF002004FF0010105F0B9FD08BD3B
:1076A00045F21853C2F200031868003018BF0120D9
:1076B000704700BFAFF30080AFF30080AFF30080EE
:1076C00070B582B006F06CFB002800F00581FFF772
:1076D000E7FF08B34FF002004FF0010105F098FDFD
:1076E0004FF66420C0F6010045F21856C2F20006BB
:1076F000316845F20852C2F20002126845F2105396
:10770000C2F200031B68FFF7CBFB48F2A060C0F297
:107710000100FCF7F5FEFEE700F05AFF05F018FB4C
:1077200045F22843C2F20003187870B149F2945030
:10773000C2F200004FF68021C0F6010145F260322E
:10774000C2F2000200F0F4FEC6E041F25411C2F2AF
:1077500000010A68002A00F0BF8040F2B414C1F2B0
:107760000004E6684FEA561045F6C523C0F67C23B0
:10777000A3FB00124FEAD21441F25C11C2F20001E5
:107780000E68A01B03281FD941F25C15C2F2000548
:107790002C60FAF79BFB054641F27823C2F2000306
:1077A000186809F075F84FF6AC22C0F60102009097
:1077B000019249F29450C2F200004FF69421C0F6B3
:1077C00001012B4600F0E4FD13F0C2F9064641F238
:1077D0005012C2F200021168814206D141F25810E3
:1077E000C2F200000368A34276D041F25815C2F2FB
:1077F00000052C6013F014FB054641F25014C2F250
:1078000000042660FFF77CFE49F29454C2F20004A3
:1078100020464FF6B021C0F60101324600F0C0FE0E
:107820000CF096FC0646284631460AF009F8024656
:1078300020464FF6B821C0F601014FF0020300F0D8
:1078400097FE0CF07DFF09F0B3FF024620464FF68D
:10785000C421C0F601014FF0020300F089FE0CF0D4
:10786000AFFE09F08DFF024620464FF6D021C0F64C
:1078700001014FF0020300F07BFE0CF051FD09F016
:10788000AFFF024620464FF6DC21C0F601014FF063
:10789000020300F06DFE284631460AF009F8024660
:1078A00020464FF6E821C0F601014FF0020300F038
:1078B0005FFE284631460AF0DBF8024620464FF6C6
:1078C000F021C0F601014FF0020300F051FE204606
:1078D00004F0D6FBFFF70CFE02B070BDAFF30080E2
:1078E0000FB410B582B040F2B413C1F20003DA68ED
:1078F00041F26010C2F200000168501A48F29F6322
:10790000C0F20103984221DD41F26014C2F200048A
:10791000226049F29454C2F20004204600F0C0FBF9
:10792000204600F045FD05AA01922046049900F08A
:10793000DFFC20464FF6AC21C0F6010100F030FC20
:10794000204600F0FDFB4FF0000001E04FF0010089
:1079500002B0BDE8104004B0704700BFAFF3008034
:10796000F8B54FF000004FF00C0106F031F813F0BD
:1079700057FA014649F28046C2F20006304600F04E
:10798000A7FE4FF000030370801BC0F106069E4265
:1079900017DD4FF05F0506F1FF3101F001072846C2
:1079A00006F046F84FF00104B44221D109E0284620
:1079B00006F03EF8284606F03BF804F10204B44213
:1079C000F5D149F28040C2F2000006F049F849F2D0
:1079D0005C34C2F20004204606F0F2FC4FF00100D5
:1079E0004FF0000105F0F4FF204606F039F8F8BD2D
:1079F000002FDCD0284606F01BF804F10104B44245
:107A0000D5D1DEE7AFF30080AFF30080AFF30080A5
:107A100008B541F28834FFF7A3FF2046FCF770FD5C
:107A2000F9E700BFAFF30080AFF30080AFF3008051
:107A300008B549F29450C2F200004FF6F821C0F6A2
:107A4000010149F26812C2F200024FF4FA7300F029
:107A50004FFB4FF00100FFF77BFC4FF6C410C0F660
:107A6000010047F25131C0F60001FEF7B9FC49F2BE
:107A70008C40C2F200004FF60431C0F6010100F064
:107A800057FB4FF61830C0F6010047F2C131C0F67F
:107A90000001FEF7ADFC41F26C20C0F6020047F297
:107AA0004131C0F60001FEF793FC49F27C30C2F28E
:107AB00000004FF61C31C0F6010100F039FB08BD93
:107AC00010B582B04FF00004009448F6F830C2F2CE
:107AD00000004FF42E714FF0400247F61123C0F61C
:107AE0000003FCF7E5FC009448F6B060C2F2000029
:107AF0004FF42E714FF0400247F2A133C0F600035D
:107B0000FCF7D6FC02B010BDAFF30080AFF30080ED
:107B100041F25413C2F2000318687047AFF30080BB
:107B200008B54AF27833C2F200031A6802F1010282
:107B30001A604FF63030C0F6010000F039F94FF608
:107B40004830C0F601004FF00D0100F021F908BDEA
:107B500008B54AF27833C2F200035A6802F1010212
:107B60005A604AF24830C2F200004FF0300100F093
:107B70000FF908BDAFF30080AFF30080AFF30080D2
:107B800008B54AF27833C2F200039A6802F10102A2
:107B90009A604FF65830C0F6010000F009F949F23A
:107BA0009860C2F200004FF44B6100F0F1F808BD9C
:107BB00008B54FF66C30C0F6010000F0F9F84FF64A
:107BC0007C30C0F601004FF0070100F0E1F808BD7D
:107BD00008B5482804D1FFF7A3FF4FF0010008BD06
:107BE0004F2804D1FFF7B4FF4FF0010008BD57281C
:107BF00004D100F0EDF84FF0010008BD422804D197
:107C000000F026F94FF0010008BD432804D1FFF72A
:107C1000B7FF4FF0010008BD742801D0542804D1EB
:107C2000FFF7C6FF4FF0010008BD462808D14FF608
:107C30008430C0F6010000F0BBF84FF0010008BD31
:107C40004AF27833C2F200031A6902F101021A61A2
:107C50004FF0000008BD00BFAFF30080AFF300801D
:107C60002DE9F04140F29813C1F2000398694FF6F4
:107C70009032C0F6010282614AF24C27C2F201073B
:107C80004FF6A438C0F601084AF25066C2F2000668
:107C90003968CC683846A04785B228B2FFF798FF0C
:107CA00028B925B12AB240461146FFF7F9F83368E2
:107CB00003F101033360EBE7AFF30080AFF3008023
:107CC00038B54FF40065C4F20205284605F068F99E
:107CD00002464AF25464C2F2000420464FF6D03104
:107CE000C0F601014FF00B0300F0DAFB284605F067
:107CF00057F9024620464FF6E031C0F601014FF039
:107D00000A0300F0CDFB4AF27835C2F200052046A6
:107D10004FF6F031C0F601014AF25063C2F200039F
:107D20001A682B6900F0BCFB20464FF61841C0F6DC
:107D300001012A6800F0B4FB20464FF63441C0F63A
:107D400001016A684FF0300300F0AAFB20464FF6AD
:107D50005841C0F60101AA684FF44B6300F0A0FB44
:107D600020464FF67C41C0F60101EA684FF44B63B0
:107D700000F096FB20464FF6A041C0F601014AF202
:107D80009032C2F20002126800F08AFB38BD00BFD8
:107D900010B504460A464AF24C20C2F201000368BC
:107DA0001B682146984710BDAFF30080AFF30080F9
:107DB00008B5014640F6C070C0F60200FFF770F843
:107DC000FFF77EFF08BD00BFAFF30080AFF3008078
:107DD00010B54AF29033C2F200031A6802F10102B0
:107DE0001A604FF6BC40C0F60100FFF7E1FF4FF606
:107DF000CC40C0F601004FF00301FFF751F84AF202
:107E00004C20C2F2010001684AF28C34C2F2000434
:107E10004B6821464FF00302984701464FF6DC407D
:107E2000C0F60100FFF73CF84FF6E840C0F601004D
:107E3000B4F90010A278FFF733F8A078B4F9001075
:107E400041F26412C2F200021368585410BD00BF20
:107E500008B54AF27833C2F20003DA6802F101028F
:107E6000DA604FF60050C0F60100FFF7A1FF41F2C3
:107E70007820C2F20000006849F29861C2F2000165
:107E80004FF44B6215F00CF809F02AF908BD00BF59
:107E900008B549F29860C2F2000041F27823C2F2BC
:107EA000000319684FF44B6214F0FAFF08BD00BFDD
:107EB00010B582B04AF25460C2F200004FF6105181
:107EC000C0F6010100F034F94FF62050C0F6010071
:107ED000FEF7E6FF4FF40064C4F202044FF6385098
:107EE000C0F6010021464FF00B0240F2823305F04C
:107EF00017F94FF64850C0F6010021464FF00A022C
:107F000040F2823305F00CF94AF24C20C2F2010033
:107F100041F26811C2F2000102F012F8FFF7B8FF57
:107F20004FF65850C0F6010047F6C141C0F60001B7
:107F3000FEF74EFA4FF0000300934AF29830C2F277
:107F400000004FF42E714FF0400247F66143C0F637
:107F50000003FCF7ADFA02B010BD00BFAFF3008024
:107F600010B512F05DFF4AF24834C2F200042060FE
:107F70000CF026FB60600CF0E3FBA0600CF0D8F87E
:107F8000E0600CF0E5F820610CF06AF960610CF03B
:107F9000C7F9E0610CF0BCF8208409F001FB6062D5
:107FA00009F076FBA0620AF053FFE06210BD00BF4B
:107FB00070B5064615F00CFF05464EF6C054C2F2E9
:107FC00000044FF66053C0F6010393E803002060FD
:107FD000A180204615F0FCFE2018294600F078FB11
:107FE00004464FF03A0004F8010B2046314615F0E4
:107FF0008FFE66194FF00D0161554FF00A02727045
:1080000005F0CEFE48B14EF6C053C2F2000306F1B1
:1080100002061846F11AFFF723F970BDAFF300808E
:1080200008B5072828D8DFE800F0040E0936131D2C
:1080300018224FF66850C0F6010008BD4FF6705088
:10804000C0F6010008BD4FF67450C0F6010008BD2F
:108050004FF67850C0F6010008BD4FF68050C0F6CC
:10806000010008BD4FF68450C0F6010008BD4FF670
:108070008850C0F6010008BD4FF69050C0F60100D0
:108080004FF6A851C0F601014FF0A302FEF7E0FE43
:108090004FF0000008BD4FF66C50C0F6010008BD5F
:1080A00038B50446D0F8F4505DB94FF6C850C0F664
:1080B00001004FF6A851C0F601014FF49972FBF789
:1080C00017FEC4F8F85038BDAFF30080AFF300805E
:1080D00010B50446D0F8F400FFF76AFF2046FFF71A
:1080E000DFFF10BDAFF30080AFF30080AFF300807F
:1080F000F8B504460F4616461D464FF6D850C0F652
:108100000100FEF7CDFE2760C4F8F460C4F8FC500F
:108110002046FFF7C5FF43F60913C0F2B223C4F8A7
:108120000031F8BDAFF30080AFF30080AFF3008003
:1081300008B500F12C024FF0C803FFF7D9FF08BDC6
:1081400038B50446D0F8F40015F042FE0546FFF7B6
:10815000CFF84CF68420C2F2000015F039FE401929
:1081600042F22733984205DDFFF7E2F82046FFF799
:1081700097FF38BD4CF68420C2F20000D4F8F4100A
:1081800015F01EFDFFF7D4F82046FFF789FF38BD34
:10819000D0F8F820D0F8F400101A7047AFF3008040
:1081A000F8B504460F4659B94FF6E850C0F601003D
:1081B0004FF6A851C0F601014FF05E02FBF798FDA3
:1081C000384615F005FE0546D4F8F4305BBB04F1E3
:1081D00004064FF6F855C0F601050FCD6060A160AA
:1081E000E260236103CD6061A1612888A0833046ED
:1081F000216815F0E5FC304615F0EAFD21184FF630
:108200001462C0F6010213888B803046394615F09F
:10821000D7FC30464FF6A851C0F601014FF04B0293
:10822000FEF716FEF8BD2046FFF7B2FF2818D4F877
:10823000FC1001F1FF3290422BDD04F104064FF6F1
:108240001865C0F601050FCD6060A160E260236192
:1082500003CD6061A1612888A0833046216815F0B4
:10826000AFFC304615F0B4FD21184FF61462C0F68D
:10827000010213888B803046394615F0A1FC304648
:108280004FF6A851C0F601014FF05502FEF7E0FD90
:10829000F8BDD4F8F800394615F03AFDD4F8F830B6
:1082A0005D19C4F8F850F8BDAFF30080AFF300805B
:1082B00008B54FF6AC21C0F60101FFF771FF08BD0C
:1082C00070B506464EF6AC54C2F200044FF00005FD
:1082D000E5602046FCF774FF6268E368D5543046D9
:1082E00041F2E801C2F20101FFF75AFF70BD00BF81
:1082F00070B506460D4614464CF68023C2F20003C4
:10830000187860B94FF63460C0F601004FF6A851F6
:10831000C0F601014FF07002FEF79AFD70BD45F204
:108320000C51C2F200010A6845F21453C2F2000374
:10833000186828B1304629462246FFF7C1FF70BDB4
:10834000002A11DC4FF0200383F31188FBF708FEAD
:10835000304629462246FFF7B3FFFBF7D9FD4FF021
:10836000000383F3118870BD4FF0200383F311885D
:10837000FBF7A6FD304629462246FFF7A1FFFBF793
:1083800077FD4FF0000383F3118870BDAFF30080D9
:108390000EB400B582B003AA52F8041B0192FFF795
:1083A000A7FF02B05DF804EB03B07047AFF30080A5
:1083B00008B54FF66061C0F601014FF6AC22C0F679
:1083C0000102FFF7E5FF08BDAFF30080AFF30080C7
:1083D00010B5044602F1FF32052A52D8DFE802F058
:1083E00003101D2A37440846F9F7EEFE02460B46F5
:1083F00020464FF66861C0F60101FFF7C9FF10BDC6
:108400000846F9F7E1FE02460B4620464FF670613A
:10841000C0F60101FFF7BCFF10BD0846F9F7D4FE16
:1084200002460B4620464FF67861C0F60101FFF781
:10843000AFFF10BD0846F9F7C7FE02460B462046BF
:108440004FF68461C0F60101FFF7A2FF10BD084698
:10845000F9F7BAFE02460B4620464FF69061C0F689
:108460000101FFF795FF10BD0846F9F7ADFE024682
:108470000B4620464FF69C61C0F60101FFF788FFCE
:1084800010BD0846F9F7A0FE02460B46204641F60D
:108490006861C0F60201FFF77BFF10BDAFF30080FB
:1084A0000EB470B583B0044607AD55F8046BFFF702
:1084B000F7FD2046FFF77CFF0195204631462A460E
:1084C000FFF716FF2046FFF7F3FE2046FFF738FEC2
:1084D00003B0BDE8704003B0704700BFAFF3008049
:1084E00070B504460D461646FFF7DAFD20462946CC
:1084F000FFF756FE4FF6AC25C0F60105204629468B
:10850000FFF74EFE204642F27001C0F602013246ED
:10851000FFF73EFF20462946FFF742FE2046FFF7C1
:108520000FFE70BDAFF30080AFF30080AFF30080AB
:108530000EB470B583B0054607AC54F8046BFFF772
:1085400037FF0194284631462246FFF7D1FE2846E0
:108550004FF6AC21C0F60101FFF722FE2846FFF7D7
:10856000B7FD03B0BDE8704003B07047AFF30080C3
:10857000F8B5044617461E46FFF712FE4FF6AC2527
:10858000C0F6010520462946FFF70AFE2046394677
:108590003246FFF71DFF20462946FFF701FEF8BDD2
:1085A00070B505461646FFF7FBFD4FF6AC24C0F646
:1085B000010428462146FFF7F3FD284641F61451F1
:1085C000C0F6020132462346FFF7E2FE70BD00BF4F
:1085D00038B5FEF78DFE4AF25874C2F200044CF62C
:1085E0008425C2F200052046294615F091FB4FF084
:1085F00000032B70FEF79CFE207810B12046FFF799
:10860000D7FC38BDAFF30080AFF30080AFF300803C
:1086100008B54EF6AC50C2F2000041F2E801C2F2D9
:1086200001014FF4FA624FF00003FDF759F84CF6E0
:108630008023C2F200034FF001021A7008BD00BF90
:10864000F0B4074600F10B0007F10A040D46B1FB38
:10865000F2F602FB161101F13003392BC8BF01F10C
:108660003703264604F80139B5FBF2F10029EDD1B4
:10867000821BB8186FEA0704011901F0010406F122
:10868000FF3212F8011F3B4603F8011B834210D151
:108690000DE002F101045278194601F8012B04F1B2
:1086A000010264785C7001F101038342F1D1F0BCF6
:1086B0007047002CEDD012F8011F03F8011B834214
:1086C000E7D1F4E7AFF30080AFF30080AFF30080B1
:1086D00008B500290DDA4FF02D0200F8012BC1F189
:1086E00000014FF00A02FFF7ABFF4FF000010170ED
:1086F00008BD4FF00A02FFF7A3FF4FF0000303701D
:1087000008BD00BFAFF30080AFF30080AFF300807F
:1087100045F20C53C2F2000318680028D4BF0020B1
:1087200001207047AFF30080AFF30080AFF300800B
:10873000F8B504460F4616461D46FFF7E9FFB8B1E7
:108740004FF0200383F31188FBF7BAFBE06810B108
:108750002046FBF795FC2046394632462B46FBF770
:1087600057FCFBF785FB4FF0000383F31188F8BD3E
:108770004FF0200383F31188FBF7F2FBE36813B19A
:108780002046FBF77DFC2046394632462B46FBF758
:108790003FFCFBF7BDFB4FF0000383F31188F8BDEE
:1087A0002DE9F04387B004460D46084601A9FDF7C0
:1087B00047FC07462046FFF773FC2046FFF7F8FD0D
:1087C00020464FF6B061C0F601012A46FFF7E0FDF2
:1087D000002F26DD4FF6C068C0F6010807F1FF3311
:1087E00003F001096D462046414655F8042FFFF776
:1087F000CFFD4FF00106BE4223D112E005F104097E
:10880000204641466A68FFF7C3FD05F1080520468A
:108810004146D9F80420FFF7BBFD06F10206BE422F
:10882000ECD120464FF6C461C0F60101FFF7B0FD60
:108830002046FFF73DFD2046FFF782FC07B0BDE86C
:10884000F083B9F1000FD9D02046414655F8042FE6
:10885000FFF79EFD06F10106BE42CFD1E1E700BF62
:1088600008B50CF0EDFA42F62060C0F602000DF0FB
:10887000D7F800F04DF800F0D3F800F001F900F05F
:108880009FF901F02DFA01F02BFB01F009FE02F037
:108890000FF800F0F5FE01F06BFC01F071FA0FF03B
:1088A000AFFB08BDAFF30080AFF30080AFF30080F3
:1088B0004FF48053CEF200035A68814209D98242B4
:1088C00004D38A422CBF0020012070474FF00000E3
:1088D0007047824204D28A422CBF00200120704798
:1088E0004FF00100704700BFAFF30080AFF300808E
:1088F00038B54FF48053CEF200035C68051920466A
:108900002946FFF7D5FF0028F9D138BDAFF3008025
:1089100008B50CF08DFB08BDAFF30080AFF300800D
:1089200008B54FF0010303704FF000014160816012
:10893000C1600161416100F11800FBF739FF08BD1A
:1089400038B50D46044658B94FF6D060C0F6010060
:108950004FF6E061C0F601014FF07102FBF7C8F974
:108960004FF0200383F31188FBF7FAFA237803F121
:10897000FF30C1B201290BD94FF6FC60C0F60100EF
:108980004FF6E061C0F601014FF07502FBF7B0F958
:10899000656020460CF084FB4FF002022270FBF76A
:1089A000B7FA4FF0000383F3118838BDAFF30080AE
:1089B000F8B504460E4617461D46FBF7D9F934B103
:1089C0002EB127B1012D0ED015F0010F0BD04FF6AF
:1089D0002870C0F601004FF6E061C0F601014FF0CB
:1089E000C302FBF785F9207802280FD004280DD0A8
:1089F00005280BD04FF64070C0F601004FF6E0613D
:108A0000C0F601014FF0C702FBF772F9A760E560FD
:108A100026614FF00303237020460CF0C9FBF8BD1C
:108A200008B50CF0C5FF08BDAFF30080AFF30080C0
:108A300038B504464FF0010303704FF00005456060
:108A400000F108002946FBF763FE04F114002946F3
:108A5000FBF75EFE04F12000206204F12401616254
:108A600004F12802A26204F12C03E36204F1300055
:108A7000206338BDAFF30080AFF30080AFF3008018
:108A800008B50DF065FA08BDAFF30080AFF30080C4
:108A900008B54FF0010303704FF00001416000F191
:108AA0000C00FBF785FE08BDAFF30080AFF300803C
:108AB0002DE9F04685B00F46924699460D9D0E9ED3
:108AC000044630B129B123B11AB10DB10C9B03B1E9
:108AD0005EB940F26C00C0F6020040F21001C0F630
:108AE00002014FF0C602FBF703F9207802280BD0F1
:108AF00040F28C00C0F6020040F21001C0F6020104
:108B00004FF0C902FBF7F4F84FF0200383F311880C
:108B1000FBF726FA4FF00001A1604FF0030222702C
:108B20000C9B0093019502962046394652464B46CF
:108B30000DF026FA0546B0F1FF3F0CBF05200220DC
:108B40002070FBF7E5F94FF0000383F31188284606
:108B500005B0BDE8F08600BFAFF30080AFF3008042
:108B600010B5044658B940F2E000C0F6020040F2E9
:108B70001001C0F602014FF48B72FBF7B9F804F153
:108B80000C00FBF7D5FE10BDAFF30080AFF3008003
:108B900008B558B940F2F400C0F6020040F21001E6
:108BA000C0F602014FF49572FBF7A2F8FBF7D8FE6E
:108BB00008BD00BFAFF30080AFF30080AFF30080CB
:108BC00008B50EF0D5FC08BDAFF30080AFF3008010
:108BD0004FF0010303704FF000014160704700BF88
:108BE00038B50D46044600B159B940F21010C0F630
:108BF000020040F22011C0F602014FF06002FBF7C4
:108C000077F84FF0200383F31188FBF7A9F9237855
:108C100003F1FF30C1B201290BD940F23C10C0F67C
:108C2000020040F22011C0F602014FF06402FBF78F
:108C30005FF8656020460EF0CBFC4FF00202227018
:108C4000FBF766F94FF0000383F3118838BD00BFCE
:108C500010B5044658B940F24C10C0F6020040F27C
:108C60002011C0F602014FF07402FBF741F84FF0FB
:108C7000200383F31188FBF773F9237803F1FF30A6
:108C8000C1B201290BD940F25810C0F6020040F2DF
:108C90002011C0F602014FF07802FBF729F82046B8
:108CA0000EF0B6FD4FF001022270FBF731F94FF0E4
:108CB000000383F3118810BDAFF30080AFF3008091
:108CC00010B5044658B940F26810C0F6020040F2F0
:108CD0002011C0F602014FF08702FBF709F84FF0B0
:108CE000200383F31188FBF73BF92378022B0BD089
:108CF00040F27810C0F6020040F22011C0F60201E6
:108D00004FF08A02FAF7F4FF20460EF0E1FD4FF033
:108D100003002070FBF7FCF84FF0000383F3118889
:108D200010BD00BFAFF30080AFF30080AFF3008051
:108D300010B5044658B940F28810C0F6020040F25F
:108D40002011C0F602014FF09902FAF7D1FF4FF05F
:108D5000200383F31188FBF703F92378A3F10203BF
:108D6000D8B203280BD940F29810C0F6020040F2A6
:108D70002011C0F602014FF09E02FAF7B9FF20461B
:108D80000EF0DEFD4FF002012170FBF7C1F84FF04D
:108D9000000383F3118810BDAFF30080AFF30080B0
:108DA00038B50C46054600B159B940F2E020C0F68E
:108DB000020040F2F021C0F6020140F23B32FAF725
:108DC00097FF2B79052B07D1A86A60604FF40071DB
:108DD00021604FF0000038BD4FF0010038BD00BFEA
:108DE00010B582B00446C36A18684FF0010101AAA9
:108DF00001F0FEFC9DF80400FF2855D1E06A0068F0
:108E00004FF0010101AA01F0F3FC9DF80400FF28D6
:108E10004AD1E16A08684FF0010101AA01F0E8FCBB
:108E20009DF80400FF283FD1E26A10684FF001016D
:108E300001AA01F0DDFC9DF80400FF2834D1E36AAB
:108E400018684FF0010101AA01F0D2FC9DF804005E
:108E5000FF2829D1E06A00684FF0010101AA01F062
:108E6000C7FC9DF80400FF281ED1E16A08684FF096
:108E7000010101AA01F0BCFC9DF80400FF2813D1F8
:108E8000E26A10684FF0010101AA01F0B1FC9DF8FF
:108E90000400FF2808D1E36A18684FF0010101AA15
:108EA00001F0A6FC9DF8040002B010BDAFF30080F5
:108EB00030B583B00446C36A18684FF0010101AAB7
:108EC00001F096FC9DF80400FF2800F0B980E16AEB
:108ED00008684FF0010101AA01F08AFC9DF8042006
:108EE000FF2A00F0AD80E36A18684FF0010101AA83
:108EF00001F07EFC9DF80400FF2800F0A180E16AEB
:108F000008684FF0010101AA01F072FC9DF80420ED
:108F1000FF2A00F09580E36A18684FF0010101AA6A
:108F200001F066FC9DF80400FF2800F08980E16AEA
:108F300008684FF0010101AA01F05AFC9DF80420D5
:108F4000FF2A7DD0E36A18684FF0010101AA01F001
:108F50004FFC9DF80400FF2872D0E16A08684FF0CA
:108F6000010101AA01F044FC9DF80420FF2A67D00A
:108F7000E36A18684FF0010101AA01F039FC9DF87D
:108F80000400FF285CD0E16A08684FF0010101AAE3
:108F900001F02EFC9DF80420FF2A51D0E36A1868E6
:108FA0004FF0010101AA01F023FC9DF80400FF2805
:108FB00046D0E16A08684FF0010101AA01F018FCEF
:108FC0009DF80420FF2A3BD0E36A18684FF00101A6
:108FD00001AA01F00DFC9DF80400FF2830D0E16AE1
:108FE00008684FF0010101AA01F002FC9DF804207D
:108FF000FF2A25D0E36A18684FF0010101AA01F0A9
:10900000F7FB9DF80400FF281AD0E16A08684FF0CA
:10901000010101AA01F0ECFB9DF80420FF2A0FD00A
:109020004FF00105E36A1868294601AA01F0E0FB48
:109030009DF80400FF2803D02846FBF761FAF1E70A
:1090400003B030BDAFF30080AFF30080AFF300801A
:10905000F0B583B007460D461446FFF729FF45F0EB
:1090600040018DF800104FEA14668DF801604FEA58
:1090700014408DF802004FEA14228DF803208DF879
:10908000044040F2B013C0F602035D5C86EA450678
:10909000995DC0B280EA4105595DD2B282EA4100D1
:1090A000195CE4B284EA41041B5D4FEA430242F0DA
:1090B00001008DF80500F96A08684FF006016A465C
:1090C00001F036FB03B0F0BDAFF30080AFF30080DA
:1090D00070B504460E461546C36A186801F068FA72
:1090E000204631462A46FFF7B3FF2046FFF778FEB9
:1090F0000546E06A006801F08BFA284670BD00BFA3
:10910000F8B504460F4615461E46C36A186801F0B6
:109110004FFA204639462A46FFF79AFF2046FFF7C6
:109120005FFE0546E06A00684FF00401324601F038
:109130005FFBE16A086801F06BFA2846F8BD00BFE2
:1091400030B583B00546C36A186801F031FA4FF0B4
:109150000104E86A0068214601AA01F049FB9DF874
:109160000410FF2903D02046FBF7CAF9F1E7EA6AA9
:10917000106801F04DFA03B030BD00BFAFF30080BE
:1091800010B5044658B940F21030C0F6020040F263
:10919000F021C0F6020140F21D32FAF7A9FD237951
:1091A000052B10D14FF008002071E16A086889682A
:1091B00001F08EF92046FFF7C3FF4FF00502227140
:1091C0004FF0000010BD4FF0010010BDAFF3008064
:1091D000F0B585B004460D461746C36A186801F01D
:1091E000E7F9204629464FF00002FFF731FF2046FD
:1091F000FFF7F6FD30B1E26A106801F009FA4FF0AE
:10920000010077E042F210754FF00106E06A006855
:1092100031466A4601F0ECFA9DF80010FE295AD159
:10922000E06A00684FF010016A4601F0E1FA17F1B8
:109230000C0F43D29DF800109DF801204FEA024325
:1092400043EA01609DF8031040EA01039DF8022003
:1092500043EA0220F8609DF804109DF805304FEABB
:10926000034242EA01609DF8071040EA01039DF8BD
:10927000062043EA0220B8609DF808109DF80930E6
:109280004FEA034242EA01609DF80B1040EA0103F5
:109290009DF80A2043EA022078609DF80C109DF8A2
:1092A0000D304FEA034242EA01609DF80F1040EA98
:1092B00001039DF80E2043EA02203860E16A086845
:1092C0004FF0020101F0D4F9E36A186801F0A0F947
:1092D0004FF000000EE005F1FF35E26A10683146FC
:1092E0006A4601F085FA9DF80030FE2B04D197E71D
:1092F0004FF0010005B0F0BD013D87D1F8E700BF98
:1093000010B5044658B940F21C30C0F6020040F2D5
:10931000F021C0F602014FF40B72FAF7E9FC4FF0AE
:10932000200383F31188FAF71BFE2379022B10D058
:10933000052B15D040F23030C0F6020040F2F0218B
:10934000C0F602014FF40C72FAF7D2FC2079022821
:1093500006D1FAF7DDFD4FF0000383F3118817E023
:109360004FF004012171FAF7D3FD4FF0000383F3AE
:109370001188E26A1068916801F0AAF82046FFF7A8
:10938000DFFEE36A186801F0DBF84FF0020020719D
:109390004FF0000010BD00BFAFF30080AFF30080BE
:1093A0002DE9F04782B0044658B940F24430C0F687
:1093B000020040F2F021C0F6020140F2C312FAF7B7
:1093C00097FC2379022B0DD0052B0BD040F25430A3
:1093D000C0F6020040F2F021C0F602014FF4E37241
:1093E000FAF786FC4FF003002071E16A08684968CB
:1093F00001F06EF8E26A10684FF0100101F038F9E0
:1094000020464FF000010A46FFF762FE01286CD0AB
:109410004FF47A70FBF774F820464FF000010A46CB
:10942000FFF756FE012860D04FF47A70FBF768F81A
:1094300020464FF000010A46FFF74AFE012854D0AB
:109440004FF47A70FBF75CF820464FF000010A46B3
:10945000FFF73EFE012848D04FF47A70FBF750F832
:1094600020464FF000010A46FFF732FE01283CD0AB
:109470004FF47A70FBF744F820464FF000010A469B
:10948000FFF726FE012830D04FF47A70FBF738F84A
:1094900020464FF000010A46FFF71AFE012824D0AB
:1094A0004FF47A70FBF72CF820464FF000010A4683
:1094B000FFF70EFE012818D04FF47A70FBF720F862
:1094C00020464FF000010A46FFF702FE01280CD0AB
:1094D0004FF47A70FBF714F820464FF000010A466B
:1094E000FFF7F6FD012840F0888020464FF0080184
:1094F0004FF4D57201ABFFF703FE05283AD04FF0C9
:1095000064074FF037064FF000054FF4D579C4F2E9
:1095100000094FF0290A4FF47A78204631462A464E
:10952000FFF7D6FD012806D1204651464A4601AB39
:10953000FFF7E6FD60B1013F5FD04046FAF7E0FF7C
:10954000204631462A46FFF7C3FD01287DD174E04D
:1095500020464FF03A014FF0000201ABFFF7D0FD7B
:109560009DF8045005F04006F7B21FB14FF001031B
:1095700084F830304FF064074FF001064FF00005DB
:109580004FF47A78204631462A46FFF7A1FD68B1AC
:10959000012832D1013F30D04046FAF7B1FF2046D2
:1095A00031462A46FFF794FD002832D1E16A086867
:1095B000896800F08DFF20464FF010014FF40072D3
:1095C000FFF786FDC8B904F1180520464FF00901E0
:1095D0002A46FFF7FDFD80B9284600F041FBA06256
:1095E00058B120464FF00A0104F10802FFF7F0FDE0
:1095F00018B94FF00502227108E0E06A006800F037
:109600009FFF4FF0020323714FF0010002B0BDE84D
:10961000F0870128F1D14046FAF772FF2046314623
:109620002A46FFF755FD0028C0D00128E5D1A7F153
:1096300002074046FAF764FFA4E7204651464A462F
:1096400001ABFFF75DFD002882D04046FAF758FFD6
:10965000204631462A46FFF73BFD012808D1204627
:1096600051464A4601ABFFF74BFD00283FF470AF6F
:10967000A7F102074046FAF743FF4EE7AFF3008039
:10968000704700BFAFF30080AFF30080AFF30080FE
:1096900040F2C023C0F6020303604FF001010171E4
:1096A0004FF00002C26280F830207047AFF30080B4
:1096B00038B50D46044600B159B940F26830C0F6DD
:1096C000020040F2F021C0F6020140F29512FAF7D2
:1096D0000FFB237903F1FF30C1B201290BD940F20E
:1096E0007830C0F6020040F2F021C0F6020140F2EC
:1096F0009712FAF7FDFAE5624FF00202227138BDC7
:1097000010B5044658B940F28830C0F6020040F265
:10971000F021C0F602014FF4D372FAF7E9FA237987
:1097200003F1FF30C1B201290BD940F29430C0F6E9
:10973000020040F2F021C0F602014FF4D472FAF7B1
:10974000D7FAE26A106800F0FBFE4FF001032371C4
:1097500010BD00BFAFF30080AFF30080AFF3008017
:1097600038B50D46044658B940F2A430C0F60200A0
:1097700040F2F021C0F6020140F24F22FAF7B8FAA7
:109780002379052B0BD040F2C030C0F6020040F226
:10979000F021C0F6020140F25122FAF7A9FA4FF087
:1097A00006002071E16A0868896800F091FEE26AAB
:1097B000106800F0FDFE94F8303033B120464FF0D1
:1097C00012012A46FFF744FC06E020464FF0120142
:1097D0004FEA4522FFF73CFC2046FFF701FB48B16A
:1097E000E06A006800F0ACFE4FF0050121714FF017
:1097F000010038BD4FF0000038BD00BFAFF300805E
:10980000F8B50C46064600B159B940F2E030C0F652
:10981000020040F2F021C0F6020140F27722FAF78E
:1098200067FA3379062B36D142F210754FF00107F3
:10983000F06A00683946224600F0DAFF2178FE29F6
:109840000FD1F36A18684FF40071224600F0D0FF80
:10985000F06A00684FF0020100F00AFF4FF00000CC
:10986000F8BD05F1FF35F26A10683946224600F06E
:10987000BFFF2378FE2B11D1E3E7F06A006800F008
:10988000C7FEF16A086800F05BFE4FF00502327116
:109890004FF00100F8BD4FF00100F8BD013DC7D108
:1098A000EBE700BFAFF30080AFF30080AFF30080C1
:1098B00010B5044658B940F2F830C0F6020040F244
:1098C000F021C0F6020140F29B22FAF711FA237947
:1098D000062B16D1E06A00684FF0070140F2A04263
:1098E000C0F6020200F024FF2046FFF779FAE16A91
:1098F000086800F08DFE4FF0050222714FF0000065
:1099000010BD4FF0010010BDAFF30080AFF3008039
:10991000F8B5054614461E46FFF722FFE8B9C6B162
:1099200006F1FF3303F0010728462146FFF768FFE1
:10993000C8B115E028462146FFF762FF80B904F55B
:10994000007406F1FF3628462146FFF759FFD8B1CB
:1099500006E02846FFF7ACFFF8BD4FF00100F8BD68
:109960004FF00100F8BD04F50074013EF1D0002F66
:10997000E0D028462146FFF743FF0028F0D104F548
:109980000074013ED6D1E4E704F50074013ED1D164
:10999000DFE700BFAFF30080AFF30080AFF30080DC
:1099A00038B50D46044658B940F21440C0F60200DE
:1099B00040F2F021C0F6020140F2B922FAF798F91C
:1099C0002379052B0BD040F23040C0F6020040F264
:1099D000F021C0F6020140F2BB22FAF789F94FF0FC
:1099E00007002071E16A0868896800F071FDE26A89
:1099F000106800F0DDFD94F8303033B120464FF0B0
:109A000019012A46FFF724FB06E020464FF0190112
:109A10004FEA4522FFF71CFB2046FFF7E1F948B16A
:109A2000E06A006800F08CFD4FF0050121714FF0F5
:109A3000010038BD4FF0000038BD00BFAFF300801B
:109A400030B583B00D46044600B159B940F25040DC
:109A5000C0F6020040F2F021C0F602014FF4387265
:109A6000FAF746F92379072B37D1E06A00684FF0FF
:109A7000020140F2B022C0F6020200F059FEE16A93
:109A800008684FF400712A4600F052FEE26A10683E
:109A90004FF0020100F0ECFDE36A18684FF001019D
:109AA00001AA00F0A5FE9DF8040000F01F010529A1
:109AB00005D12046FFF7FCF94FF000000FE0E26A05
:109AC000106800F0A5FDE36A186800F039FD4FF05A
:109AD000050020714FF0010001E04FF0010003B0DC
:109AE00030BD00BFAFF30080AFF30080AFF3008064
:109AF00010B5044658B940F26840C0F6020040F282
:109B0000F021C0F6020140F20332FAF7F1F82379AE
:109B1000072B13D1E06A00684FF0020140F2B04217
:109B2000C0F6020200F004FEE16A086800F070FD71
:109B30004FF0050222714FF0000010BD4FF0010000
:109B400010BD00BFAFF30080AFF30080AFF3008023
:109B5000F8B5054614461E46FFF722FFE8B9C6B120
:109B600006F1FF3303F0010728462146FFF768FF9F
:109B7000C8B115E028462146FFF762FF80B904F519
:109B8000007406F1FF3628462146FFF759FFD8B189
:109B900006E02846FFF7ACFFF8BD4FF00100F8BD26
:109BA0004FF00100F8BD04F50074013EF1D0002F24
:109BB000E0D028462146FFF743FF0028F0D104F506
:109BC0000074013ED6D1E4E704F50074013ED1D122
:109BD000DFE700BFAFF30080AFF30080AFF300809A
:109BE00070B506460C461546914202D38B1A1F2BC0
:109BF0000BD940F2C040C0F6020040F2D441C0F69A
:109C000002014FF04902FAF773F84FEA551105F0D7
:109C10001F054FEA541204F01F0404F101044FF031
:109C2000010000FA04F000F1FF3091420CD256F826
:109C300022201040C5F1200300FA03F056F821104D
:109C400021FA05F5284370BD56F82130184020FA56
:109C500005F070BDAFF30080AFF30080AFF300807C
:109C600070B50446C368980F02D001282ED121E0B8
:109C700020464FF049014FF03E02FFF7B1FF064684
:109C800020464FF031014FF02F02FFF7A9FF0546A4
:109C900020464FF053014FF05002FFF7A1FF06F1AD
:109CA000010605F1020506FA05F5A0F1090005FA1D
:109CB00000F070BD20464FF045014FF03002FFF735
:109CC0008FFF00F101004FEA802070BD4FF00000CF
:109CD00070BD00BFAFF30080AFF30080AFF3008032
:109CE00008B50DF095FE08BDAFF30080AFF300801E
:109CF0004FF0010303704FF000014160704700BF57
:109D000038B50D46044600B159B940F2F040C0F6EE
:109D1000020040F20051C0F602014FF06502F9F76F
:109D2000E7FF4FF0200383F31188FAF719F923783E
:109D300003F1FF30C1B201290BD940F21C50C0F62B
:109D4000020040F20051C0F602014FF06902F9F73B
:109D5000CFFF6560AA88228120460DF079FE4FF082
:109D600002032370FAF7D4F84FF0000383F311884D
:109D700038BD00BFAFF30080AFF30080AFF30080C9
:109D800008B50DF0A5F808BDAFF30080AFF3008073
:109D900038B50C46054600B159B940F2C050C0F67E
:109DA000020040F2D051C0F602014FF05702F9F71D
:109DB0009FFF4FF0200383F31188FAF7D1F828466C
:109DC00021460DF0BDF8FAF7A3F84FF0000383F336
:109DD000118838BDAFF30080AFF30080AFF300808F
:109DE00038B50C46054600B159B940F2EC50C0F602
:109DF000020040F2D051C0F602014FF06802F9F7BC
:109E000077FF4FF0200383F31188FAF7A9F828466B
:109E100021460DF0BDF8FAF77BF84FF0000383F30D
:109E2000118838BDAFF30080AFF30080AFF300803E
:109E300010B5044658B940F2C050C0F6020040F2D6
:109E4000D051C0F602014FF0BB02F9F751FF204696
:109E50000DF0C6F810BD00BFAFF30080AFF3008077
:109E600008B500F10C00FAF7D3FE08BDAFF300808F
:109E700008B500F10C004FF0FF33FAF7C9FE08BD3A
:109E800008B500F13000FAF7ABFF08BDAFF3008072
:109E900008B500F130004FF0FF33FAF7A1FF08BD1D
:109EA00008B500F10C00FAF77BFE08BDAFF30080A7
:109EB00008B500F10C004FF0FF31FAF771FE08BD54
:109EC00008B500F13000FAF72BFF08BDAFF30080B2
:109ED00008B500F130004FF0FF32FAF721FF08BD5E
:109EE00008B50DF0BDFF08BDAFF30080AFF30080F3
:109EF00030B583B004460B46154640F2A062C0F66A
:109F0000020240F8042B60604FF0010121720094BE
:109F100004F10C0004F154014FF01002FAF7E0FDD7
:109F2000009404F1300004F164014FF010022B465C
:109F3000FAF7C6FE03B030BDAFF30080AFF3008088
:109F400038B50D46044658B940F22060C0F602000C
:109F500040F22C61C0F602014FF0A102F9F7C8FEF1
:109F60004FF0200383F31188F9F7FAFF237A03F106
:109F7000FF30C1B201290BD940F24860C0F602009F
:109F800040F22C61C0F602014FF0A602F9F7B0FED4
:109F9000204629460DF09CFF4FF002022272F9F78D
:109FA000B7FF4FF0000383F3118838BDAFF3008093
:109FB00038B504460D46F9F7DBFE5CB940F2746033
:109FC000C0F6020040F22C61C0F602014FF0D80248
:109FD000F9F78EFE63692BB904F104004FF0040118
:109FE000FAF746FD04F10C002946FAF7A9FD00280E
:109FF00005DA04F104004FF08001FAF739FD38BDAD
:10A0000038B5046AD4F854321A68117804292AD170
:10A01000207A022827D112891B7942FA03F111F024
:10A02000010F20D1256CE06B2A1AA36BD51A1AD028
:10A03000F9F76EFF4FF0000383F31188D4F8541240
:10A040000868097904F130022B4600F009FD4FF051
:10A05000200383F31188F9F783FFD4F854221068A2
:10A06000117900F03DFD38BDAFF30080AFF3008003
:10A0700070B5046AD4F854321A681178042932D1C0
:10A08000207A02282FD1597902EB8105EB685D8A8D
:10A09000528942FA01F010F0010F24D1E669A1695A
:10A0A000721A6369D61AB5421DD8F9F731FF4FF01D
:10A0B000000383F31188B6FBF5F3D4F85412086853
:10A0C000497904F10C0205FB03F300F0B9FC4FF0F1
:10A0D000200383F31188F9F743FFD4F85422106862
:10A0E000517900F0CDFC70BDAFF30080AFF300807C
:10A0F00008B500F10C00FAF78BFD08BDAFF3008046
:10A1000008B500F10C004FF0FF33FAF781FD08BDF0
:10A1100008B500F13000FAF763FE08BDAFF3008028
:10A1200008B500F130004FF0FF33FAF759FE08BDD3
:10A1300008B500F10C00FAF733FD08BDAFF300805D
:10A1400008B500F10C004FF0FF31FAF729FD08BD0A
:10A1500008B500F13000FAF7E3FD08BDAFF3008069
:10A1600008B500F130004FF0FF32FAF7D9FD08BD15
:10A17000704700BFAFF30080AFF30080AFF3008003
:10A1800010B582B00446034640F21072C0F60202D7
:10A1900043F8042B43604FF001002072009404F157
:10A1A0000C0004F154014FF480724AF27103C0F6BE
:10A1B0000003FAF795FC009404F1300004F5AA714D
:10A1C0004FF480724AF20103C0F60003FAF778FDFB
:10A1D00002B010BDAFF30080AFF30080AFF300809A
:10A1E00070B50D460E68044658B940F2C060C0F61E
:10A1F000020040F2D061C0F602014FF0DA02F9F736
:10A2000077FD4FF0200383F31188F9F7A9FE237A35
:10A2100003F1FF30C1B201290BD940F2F060C0F662
:10A22000020040F2D061C0F602014FF0DF02F9F700
:10A230005FFD2A7906EB82039C61687900F10900D1
:10A2400046F82040A97906EB8106B461C4F854525F
:10A250004FF002022272F9F75BFE4FF0000383F326
:10A26000118870BDAFF30080AFF30080AFF30080C2
:10A2700070B50446D0F854321D6800F10C06304623
:10A28000FAF73EFC04F13000FAF72AFD04F104006D
:10A290004FF00101FAF7ECFBD4F85402417905EBD9
:10A2A0008102D368284632465B8A00F0C9FBD4F8A5
:10A2B00054122846497900F0E3FB70BDAFF30080EB
:10A2C00090F8443003F0600120292CD190F845200B
:10A2D000212A04D0222A1ED0202A27D10DE041F2C3
:10A2E0007411C2F2000181634FF00702C2634FF0A4
:10A2F000000303644FF00100704741F27413C2F28F
:10A30000000383634FF00701C1634FF00002026452
:10A310004FF0010070474FF000038363C363036491
:10A320004FF0010070474FF0000070474FF0000001
:10A33000704700BFAFF30080AFF30080AFF3008041
:10A34000F8B506460D4600EB81039C69002C50D001
:10A350004FF0200383F31188F9F7B2FD04F10400F4
:10A360004FF00801FAF784FB226CE06B111AA76B1F
:10A37000CF1B17D0F9F77CFD4FF0000383F3118852
:10A380003046294604F130023B4600F069FB4FF0AD
:10A39000200383F31188F9F793FD3046294600F036
:10A3A0009FFB20E006EB8503DA6850694168D1B174
:10A3B000138A03F1FF320A4215D1F9F759FD4FF024
:10A3C000000383F311883046294604F1300200F07F
:10A3D00047FB4FF0200383F31188F9F771FD3046F6
:10A3E000294600F07DFBF9F743FD4FF0000383F3AE
:10A3F0001188F8BDAFF30080AFF30080AFF30080A9
:10A400002DE9F04106460D4601F1090350F82340BD
:10A41000002C37D04FF0200383F31188F9F750FD5B
:10A4200004F104004FF00401FAF722FB06EB85006B
:10A43000C1684F8AE269A369D01A6169C1EB00085B
:10A44000474519D8F9F714FD4FF0000383F311883D
:10A45000B8FBF7F33046294604F10C0207FB03F37F
:10A4600000F0EEFA4FF0200383F31188F9F728FD8E
:10A470003046294600F004FBF9F7FAFC4FF00003E0
:10A4800083F31188BDE8F081AFF30080AFF3008063
:10A49000704700BFAFF30080AFF30080AFF30080E0
:10A4A00008B50CF055FE08BDAFF30080AFF3008097
:10A4B00008B54FF0010303704FF000014160816067
:10A4C00000F10C00FAF774F908BD00BFAFF300808B
:10A4D00038B50D46044600B159B940F23070C0F6A7
:10A4E000020040F24071C0F602014FF06D02F9F730
:10A4F000FFFB4FF0200383F31188F9F731FD237838
:10A5000003F1FF30C1B201290BD940F25C70C0F6F3
:10A51000020040F24071C0F602014FF07102F9F7FB
:10A52000E7FB656020460CF03BFE4FF00202227014
:10A53000F9F7EEFC4FF0000383F3118838BD00BF3C
:10A5400010B5044658B940F26C70C0F6020040F2F3
:10A550004071C0F602014FF08302F9F7C9FB4FF0DA
:10A56000200383F31188F9F7FBFC237803F1FF3014
:10A57000C1B201290BD940F27870C0F6020040F256
:10A580004071C0F602014FF08702F9F7B1FB204697
:10A590000CF0BEFE20460CF08BFE4FF00102227044
:10A5A000F9F7B6FC4FF0000383F3118810BD00BF2C
:10A5B00010B5044658B940F28870C0F6020040F267
:10A5C0004071C0F602014FF09702F9F791FB4FF08E
:10A5D000200383F31188F9F7C3FC2378022B0BD0F7
:10A5E00040F29870C0F6020040F24071C0F60201DD
:10A5F0004FF09A02F9F77CFB20460CF079FEF9F750
:10A6000087FC4FF0000383F3118810BDAFF3008087
:10A6100010B5044658B940F2A870C0F6020040F2E6
:10A620004071C0F602014FF0A902F9F761FB4FF04B
:10A63000200383F31188F9F793FC2378022B0BD0C6
:10A6400040F2B870C0F6020040F24071C0F602015C
:10A650004FF0AC02F9F74CFB20460CF059FEF9F72D
:10A6600057FC4FF0000383F3118810BDAFF3008057
:10A6700038B50D46044600B159B940F67C00C0F625
:10A68000020040F24071C0F602014FF49572F9F7F2
:10A690002FFB4FF0200383F31188F9F761FC237837
:10A6A000022B0BD040F69000C0F6020040F2407141
:10A6B000C0F6020140F22D12F9F71AFB606801683A
:10A6C00059B140F6A000C0F6020040F24071C0F659
:10A6D00002014FF49772F9F70BFB4FF0030222705F
:10A6E000204629460CF024FEA3685BB140F6B0007A
:10A6F000C0F6020040F24071C0F602014FF49872B9
:10A70000F9F7F6FA40F29810C1F200008169A160F1
:10A710004FF00200F9F764FDF9F7FAFB4FF0000380
:10A7200083F3118838BD00BFAFF30080AFF3008022
:10A7300070B50D461646044608B101B15AB940F647
:10A74000F800C0F6020040F24071C0F6020140F28B
:10A750006712F9F7CDFA4FF0200383F31188F9F768
:10A76000FFFB2378022B0BD040F60410C0F602004A
:10A7700040F24071C0F602014FF4B572F9F7B8FA31
:10A780006068016859B140F61410C0F6020040F24A
:10A790004071C0F6020140F26B12F9F7A9FA4FF0CE
:10A7A000030222702046294632460CF0F1FDA368D0
:10A7B0005BB140F6B000C0F6020040F24071C0F656
:10A7C000020140F26D12F9F793FA40F29810C1F2CB
:10A7D00000008169A1604FF00200F9F701FDF9F76F
:10A7E00097FB4FF0000383F3118870BDAFF3008037
:10A7F00070B50D461646044608B101B15AB940F687
:10A800002410C0F6020040F24071C0F602014FF47D
:10A81000C272F9F76DFA4FF0200383F31188F9F74C
:10A820009FFB2378022B0BD040F63410C0F60200B9
:10A8300040F24071C0F6020140F28712F9F758FA6F
:10A840006068016859B140F64810C0F6020040F255
:10A850004071C0F6020140F28912F9F749FA4FF04F
:10A86000030222702046294632460CF0C1FDA3683F
:10A870005BB140F6B000C0F6020040F24071C0F695
:10A88000020140F28B12F9F733FA40F29810C1F24C
:10A8900000008169A1604FF00200F9F7A1FCF9F70F
:10A8A00037FB4FF0000383F3118870BDAFF30080D6
:10A8B00008B50CF065F808BDAFF30080AFF3008079
:10A8C0004FF0010303704FF000014160C1618162EC
:10A8D0000162C1624162016301814181704700BF31
:10A8E00038B50D46044600B159B940F6B010C0F66F
:10A8F000020040F6C011C0F6020140F20F12F9F753
:10A90000F7F94FF0200383F31188F9F729FB237837
:10A9100003F1FF30C1B201290BD940F6DC10C0F6BB
:10A92000020040F6C011C0F6020140F21312F9F71E
:10A93000DFF965604FF00005E56025616561A5619F
:10A9400020460CF035F84FF002022270F9F7E0FAD9
:10A950002B4683F3118838BDAFF30080AFF300803E
:10A9600070B504460E461546F9F702FA04B15DB912
:10A9700040F60820C0F6020040F6C011C0F6020101
:10A9800040F24112F9F7B4F92378042B0BD040F6CA
:10A990002020C0F6020040F6C011C0F6020140F2CD
:10A9A0004312F9F7A5F904EB8600C16859B140F6E6
:10A9B0003C20C0F6020040F6C011C0F6020140F291
:10A9C0004512F9F795F9686928B14FF000014FF089
:10A9D000100212F00DFBA86928B14FF000014FF0F2
:10A9E000100212F005FB04EB8602D56020463146CA
:10A9F0000CF0D6F870BD00BFAFF30080AFF300805D
:10AA000038B500EB8104E568AC694FF000052570AE
:10AA1000E2606360A5600CF0BBF938BDAFF3008065
:10AA200038B500EB8104E5686C694FF000052570CE
:10AA3000E2606360A5600CF0C3F938BDAFF300803D
:10AA400038B500EB8104E568AC694FF0010525706D
:10AA5000E26063604FF00003A3600CF099F938BD29
:10AA600038B500EB8104E5686C694FF0010525708D
:10AA7000E26063604FF00003A3600CF0A1F938BD01
:10AA800038B504460D46F9F773F95CB940F69020E5
:10AA9000C0F6020040F6C011C0F602014FF4F47295
:10AAA000F9F726F9638943FA05F212F0010F0DD187
:10AAB0004FF0010000FA05F040EA030161812046F1
:10AAC00029460CF09DF94FF0000038BD4FF0010011
:10AAD00038BD00BFAFF30080AFF30080AFF300805C
:10AAE00038B504460D46F9F743F95CB940F6A8209D
:10AAF000C0F6020040F6C011C0F6020140F2032287
:10AB0000F9F7F6F8238943FA05F212F0010F0DD197
:10AB10004FF0010000FA05F040EA030121812046D0
:10AB200029460CF07DF94FF0000038BD4FF00100D0
:10AB300038BD00BFAFF30080AFF30080AFF30080FB
:10AB400008B503464FF0020202704FF00002A0F871
:10AB50004C2083F84E2080F84F2002814281C26051
:10AB600002614261826183F834200BF099FF08BDD5
:10AB700070B504464FF0000380F8343000F1440211
:10AB80000CF0F6F86068816821B1204688470028FB
:10AB900040F05B8194F8443013F0600F40F03F8147
:10ABA00094F8452003F07F0040EA0221B1F5407F90
:10ABB00047D010DC022900F0B98004DC31B3012950
:10ABC00040F02D81A6E0B1F5807F29D0B1F5817FDD
:10ABD00040F02581F3E0B1F5C06F5FD009DC40F2B1
:10ABE0000230814200F00381B1F5A06F40F017817F
:10ABF00038E0B1F5106F74D040F60242914200F097
:10AC00008980B1F5006F40F00A8160E004F14C03E7
:10AC1000A3634FF00202E2634FF00000206414E1EE
:10AC200094F84600012840F0FA80B4F84C1021F066
:10AC30000203A4F84C304FF00002A263E2632264E6
:10AC400003E194F84610012940F0E980B4F84C2063
:10AC500042F00200A4F84C004FF00003A363E3634A
:10AC60002364F2E0B4F84430B3F5A06F10D194F847
:10AC7000462084F84E2020460BF082FF61680B6866
:10AC80001BB120464FF0010198474FF003002070A0
:10AC90004FF00002A263E2632264D6E0656894F894
:10ACA000496094F848306D68204694F8471094F84D
:10ACB000462043EA0623A847002800F0B0804268F7
:10ACC000A2630068E0634FF000032364BDE004F179
:10ACD0004F01A1634FF00103E3634FF000002064D4
:10ACE000B3E094F8460084F84F0018B94FF0030120
:10ACF000217002E04FF00402227063681A681AB1F2
:10AD000020464FF0020190474FF00000A063E0633F
:10AD100020649AE040F69012C0F60202A2634FF05F
:10AD20000201E1634FF0000323648EE094F84810C1
:10AD300011F0800F21D0204601F00F010CF000F837
:10AD4000012802D002286AD10BE040F6F023C0F6B9
:10AD50000203A3634FF00202E2634FF0000121649B
:10AD600073E040F6A012C0F60202A2634FF00201A7
:10AD7000E1634FF00000206467E0204601F00F011E
:10AD80000BF0C6FF012802D0022848D10BE040F6A4
:10AD9000F021C0F60201A1634FF00200E0634FF022
:10ADA0000003236451E040F6A010C0F60200A06347
:10ADB0004FF00203E3634FF00002226445E094F891
:10ADC000461061BB94F8483013F00F0109D013F01E
:10ADD000800F03D020460CF06BF802E020460CF008
:10ADE00057F84FF00002A263E26322642DE094F86A
:10ADF0004610A1B994F8483013F00F0109D013F0B0
:10AE0000800F03D020460CF033F802E020460CF00F
:10AE10001FF84FF00000A063E063206415E02046B7
:10AE20004FF000010CF024F820464FF000010CF028
:10AE30000FF8626813681BB120464FF00501984770
:10AE40004FF0060084F8340070BD94F84B1094F86D
:10AE50004A2042EA0120E36B984238BFE06394F94C
:10AE6000441000293ADAE36BDBB14FF0010184F8BA
:10AE7000341020464FF00001A26BFFF7D1FD4FF0D8
:10AE8000200383F31188F9F71BF820464FF00001E7
:10AE9000FFF726FEF8F7ECFF4FF0000383F311886D
:10AEA00070BD4FF0030384F8343020464FF00001AA
:10AEB0000A460B46FFF7A4FD4FF0200383F31188E9
:10AEC000F8F7FEFF20464FF00001FFF7D9FDF8F735
:10AED000CFFF4FF0000383F3118870BDE36BDBB14C
:10AEE0004FF0040084F8340020464FF00001A26BBC
:10AEF000FFF786FD4FF0200383F31188F8F7E0FF9A
:10AF000020464FF00001FFF7BBFDF8F7B1FF4FF00F
:10AF1000000383F3118870BD4FF0050284F83420DC
:10AF200020464FF000010A460B46FFF779FD4FF02F
:10AF3000200383F31188F8F7C3FF20464FF0000188
:10AF4000FFF7CEFDF8F794FF4FF0000383F311886D
:10AF500070BD00BFAFF30080AFF30080AFF300809F
:10AF600010B5044690F83430022B30D0052B4BD06E
:10AF7000012B51D1C36B90F84B0094F84A2042EA60
:10AF80000021994223D9E068028AB3FBF2F102FB67
:10AF90001133E3B920464FF000010A460B46FFF794
:10AFA0003FFD4FF0200383F31188F8F789FF204617
:10AFB0004FF00001FFF794FDF8F75AFF4FF0000340
:10AFC00083F311884FF0020084F8340010BD4FF075
:10AFD000030384F8343020464FF000010A460B4644
:10AFE000FFF70EFD4FF0200383F31188F8F768FF99
:10AFF00020464FF00001FFF743FDF8F739FF4FF00F
:10B00000000383F3118810BD026C02B190474FF02A
:10B01000000184F8341010BD4FF000010BF028FF40
:10B0200020464FF000010BF013FF606802681AB170
:10B0300020464FF0050190474FF0060184F8341088
:10B0400010BD00BFAFF30080AFF30080AFF300800E
:10B0500010B5044690F83430032B1ED0042B28D1B1
:10B060004FF0050084F8340020464FF000010A46F6
:10B070000B46FFF7D5FC4FF0200383F31188F8F758
:10B080001FFF20464FF00001FFF72AFDF8F7F0FE02
:10B090004FF0000383F3118810BDC1688A6993687B
:10B0A0003BB9016C01B188474FF0000084F83400CF
:10B0B00010BD20464FF000010BF0DAFE20464FF0A5
:10B0C00000010BF0C5FE626813681BB120464FF00B
:10B0D000050198474FF0060184F8341010BD00BFF9
:10B0E0002DE9F84F2DED028B40F2B413C1F20003AD
:10B0F000DA6848F21F51C5F2EB11A1FB02144FEAC6
:10B100005418061E40F3058348F2D427C4F20D07F5
:10B1100040F6B47506F1FF3202F0010928463946BF
:10B1200006F08EFBB7EE008A07EE900A38EE270A8B
:10B13000BDEEC08A4FF00104B44240F029851BE007
:10B140002846394606F07CFBB8EEC82A02EE900A83
:10B1500032EE223ABDEEC38A2846394606F070FB2D
:10B16000F8EEC83A04EE100A73EE844ABDEEE48AA3
:10B1700004F10204B442E3D140F2B411C1F200017F
:10B18000CB6818EE100A70B148F21F57C5F2EB17E2
:10B19000A7FB0315C8EB551240F60030C0F60200BD
:10B1A0003146FBF77DFE40F2B414C1F20004E268C0
:10B1B000E36806EBD6724FEA620000280DDD00F16D
:10B1C000FF3101F001074FF00103834240F0D684C4
:10B1D00003E003F102038342FBD140F2B415C1F254
:10B1E0000005EA68E868002E40F3A1822A4606F1CD
:10B1F000FF3101F00107EC684FF00103B34240F06A
:10B20000B18407E0D1686718D5687C1903F102039F
:10B21000B342F7D140F2B412C1F20002D368002C5D
:10B2200000F06B8348F21F51C5F2EB11A1FB03271D
:10B23000A1FB00504FEA501540F63030C0F6020036
:10B240003146C5EB5712FBF72BFE56E34B4683F313
:10B250001188F8F785FED8F80C002418F8F758FE86
:10B260003B4683F3118805F101054B4683F31188B2
:10B27000F8F776FED8F80C20A418F8F749FE3B46FC
:10B2800083F3118805F10105B542DFD140F2B4170F
:10B29000C1F20007FB6894B148F21F55C5F2EB15E7
:10B2A000A5FB03E7A5FB0B0B4FEA5B1240F66430EE
:10B2B000C0F602003146C2EB5712FBF7F1FD46F231
:10B2C0006761C6F2666181FB06204FEAE673C3EB55
:10B2D000A00140F2B415C1F20005EF68002921DD9C
:10B2E000284648F21F52C5F2EB1201F1FF3303F07A
:10B2F0000105C368A2FB03E304EB53144FF0010301
:10B300008B4240F008840DE0C568A2FB05E504EB24
:10B310005514C568A2FB05E504EB551403F10203BF
:10B320008B42F1D140F2B410C1F20000C2688CB17E
:10B3300048F21F53C5F2EB13A3FB0205A3FB074022
:10B340004FEA501440F6A830C0F60200C4EB551284
:10B35000FBF7A6FD40F2B411C1F20001CA6848F241
:10B360001F53C5F2EB13A3FB02504FEA5012002EFD
:10B3700040F3128206F1FF3303F001014FF00104A4
:10B38000B44240F0BF83DCE104F10204B442FBD1DB
:10B39000D7E14FEA820203F10203B342F9D140F24E
:10B3A000B414C1F20004E068002A40F0C98248F2F7
:10B3B0001F51C5F2EB11A1FB00E3A1FB05454FEACC
:10B3C000551240F6E030C0F602003146C2EB53128F
:10B3D000FBF766FDB4E200F10200B042FBD120E2CF
:10B3E0004FEA820201F10201B142F9D140F2B413F5
:10B3F000C1F20003DC68002A40F0B98248F21F5114
:10B40000C5F2EB11A1FB0453A1FB00E04FEA50127F
:10B4100040F61440C0F602003146C2EB5312FBF76F
:10B420003FFDA4E203F10203B342FBD11AE275EE41
:10B43000055A35EEA55A01F10201B142F7D140F2A9
:10B44000B413C1F20003DA68B5EE405AF1EE10FA17
:10B4500000F0A48248F21F55C5F2EB15A5FB0220AF
:10B46000A5FB04414FEA5113C3EB501240F648408C
:10B47000C0F602003146FBF713FD40F2B412C1F2F0
:10B480000002D46848F21F55C5F2EB15A5FB045025
:10B490004FEA5012002E40F306824FF00004B7EE40
:10B4A000006ADFEDBB6A9FEDBB7A6FEA0400831987
:10B4B00003F0010176EE267A87EE870A76EE001A0F
:10B4C00004F10104B44240F0DB820FE031EEA62A21
:10B4D000C2EE072A31EEA23A73EE263A83EE874A8D
:10B4E00073EE041A04F10204B442EFD140F2B41432
:10B4F000C1F20004E068F5EE401AF1EE10FA00F037
:10B500005F8248F21F51C5F2EB11A1FB00E0C2EBD4
:10B51000501240F67C40C0F602003146FBF7C0FCFA
:10B5200040F2B412C1F20002D46848F21F53C5F2CF
:10B53000EB13A3FB04014FEA5118002E40F3C18125
:10B540004FF000074FF000044FF00005C3F6F07510
:10B550004FF0000A4FF0000BC3F6E07B6FEA0709DB
:10B5600009EB060101F001092046294652465B46D7
:10B57000F6F77EFE02460B4620462946F6F7C6FC45
:10B5800004460D4607F10107B74240F063821DE013
:10B590002046294652465B46F6F76AFE02460B46AF
:10B5A00020462946F6F7B2FC04460D4652465B4655
:10B5B000F6F75EFE02460B4620462946F6F7A6FC45
:10B5C00004460D4607F10207B742E1D140F2B41735
:10B5D000C1F20007FF68204629464FF000024FF0F5
:10B5E0000003F7F7B3F8002840F0008248F21F503C
:10B5F000C5F2EB10A0FB0712C8EB521240F6B040A8
:10B60000C0F602003146FBF74BFC40F2B413C1F226
:10B610000003D96848F21F54C5F2EB14A4FB0140A3
:10B620004FEA5018002E40F35A814FF000074FF0B8
:10B6300000044FF00005C3F6F0759FED538B4FF0FB
:10B64000000A4FF4804BC4F2600B6FEA070C0CEB5E
:10B65000060E0EF001092046294653EC182BF6F78A
:10B6600055FC52465B46F6F72DFF02460B46204638
:10B670002946F6F74BFC04460D4607F10107B74291
:10B6800040F0CE8125E02046294653EC182BF6F7F2
:10B690003DFC52465B46F6F715FF02460B46204638
:10B6A0002946F6F733FC04460D4653EC182BF6F703
:10B6B0002DFC52465B46F6F705FF02460B46204638
:10B6C0002946F6F723FC04460D4607F10207B74268
:10B6D000D9D140F2B417C1F20007FF6820462946CD
:10B6E0004FF000024FF00003F7F730F8002840F069
:10B6F000938148F21F52C5F2EB12A2FB0751C8EB2F
:10B70000511240F6E840C0F602003146FBF7C8FB94
:10B7100082E140F2B410C1F20000C56848F21F5740
:10B72000C5F2EB17A7FB05E3C8EB531234E540F273
:10B73000B414C1F20004E268D4F80CB04FF0000475
:10B74000A4E540F2B415C1F20005E86848F21F53C1
:10B75000C5F2EB13A3FB000440F61C50C0F6020038
:10B760003146C2EB5412FBF79BFBED6806F1FF314B
:10B7700001F001004FF002024FF00103B34240F02C
:10B78000B6810CE6AFF300800000000000005940D5
:10B790000000C8420000024340F2B414C1F20004A9
:10B7A000E16848F21F55C5F2EB15A5FB011340F601
:10B7B0001C50C0F602003146C2EB5312FBF770FB7F
:10B7C000E368E368E068E268A5FB02E2A5FB00012C
:10B7D0004FEA511340F64C50C0F602003146C3EB1D
:10B7E0005212FBF75DFBE368E368E068E268A5FBE3
:10B7F0000212A5FB00E14FEA511340F68050C0F65B
:10B8000002003146C3EB5212FBF74AFBE168E468E1
:10B81000A5FB0402A5FB01154FEA5510C0EB52121F
:10B8200024E640F2B414C1F20004E36848F21F5168
:10B83000C5F2EB11A1FB035340F64C50C0F60200D9
:10B840003146C2EB5312FBF72BFBE06806F1FF32E7
:10B8500002F001044FF002024FF00101B14240F04A
:10B860003281C3E540F2B414C1F20004E06848F24A
:10B870001F51C5F2EB11A1FB00E340F68050C0F66A
:10B8800002003146C2EB5312FBF70AFBE46806F1F3
:10B89000FF3202F00100B0EE005A4FF00101B14258
:10B8A00040F0FD80CBE540F2B411C1F20001CC685C
:10B8B00048F21F53C5F2EB13A3FB0401C2EB511274
:10B8C00027E640F2B410C1F20000C26848F21F54EB
:10B8D000C5F2EB14A4FB0213C8EB53128EE640F240
:10B8E000B412C1F20002D16848F21F53C5F2EB1343
:10B8F000A3FB0140C8EB501203E740F2B412C1F2BF
:10B900000002D2F80CB04FF0200990464FF000072B
:10B9100006F1FF3A0AF0010A4B4683F31188F8F763
:10B920001FFBD8F80C30E418F8F7F2FA3B4683F323
:10B9300011883D4605F10105B54240F0FB80A5E4C4
:10B9400040F2B414C1F20004E06848F21F51C5F29D
:10B95000EB11A1FB00534FEA531206F1FF3505F03E
:10B9600001044FF00100B04240F0B88059E740F2C6
:10B97000B414C1F20004E16848F21F53C5F2EB139E
:10B98000A3FB01E04FEA501206F1FF3404F001017D
:10B990004FF00103B34240F08D8063E740F2B414EE
:10B9A000C1F20004E06848F21F51C5F2EB11A1FB9F
:10B9B00000034FEA53124FF00004B7EE006A70E53F
:10B9C00040F2B417C1F20007FA6848F21F55C5F2F9
:10B9D000EB15A5FB02134FEA53184FF000074FF089
:10B9E00000044FF00005C3F6F075B1E540F2B41065
:10B9F000C1F20000C26848F21F53C5F2EB13A3FB6B
:10BA000002414FEA51184FF000074FF000044FF089
:10BA10000005C3F6F07510E6BDEC028BBDE8F88FAB
:10BA2000B9F1000F3FF42FAE53EC182BF6F76EFA76
:10BA300052465B46F6F746FD02460B46204629462F
:10BA4000F6F764FA04460D4607F10107B7427FF4A2
:10BA50001AAE3EE6B9F1000F3FF49AAD52465B468E
:10BA6000F6F706FC02460B4620462946F6F74EFA44
:10BA700004460D4607F10107B7427FF489ADA5E5FD
:10BA800000293FF423AD71EEA60A80EE871A71EE0D
:10BA9000811A04F10104B4427FF418AD26E50028B0
:10BAA0003FF4C5AC35EE055A01F10101B1427FF416
:10BAB000BEACC4E400293FF4B5AC03F10103B342CA
:10BAC0007FF4B0ACCEE6002C3FF48AAC4FEA4202E1
:10BAD00001F10101B1427FF483AC87E4002C3FF413
:10BAE0007AAC00F10100B0427FF475AC99E6002811
:10BAF0003FF44FAC4FEA420203F10103B3427FF43B
:10BB000048AC4CE400293FF43FAC04F10104B442DA
:10BB10007FF43AAC15E6002D3FF4F6ABC568A2FB06
:10BB200005E504EB551403F101038B427FF4ECAB04
:10BB3000FFF7F8BBBAF1000F3FF488AB4B4683F335
:10BB40001188F8F70DFAD8F80C106418F8F7E0F936
:10BB50003B4683F3118805F10105B5427FF476ABCE
:10BB6000FFF794BB002F3FF44DABED68641903F170
:10BB70000103B3427FF446ABFFF74CBB002F3FF409
:10BB800028AB03F1010383427FF423ABFFF725BB0E
:10BB9000B9F1000F3FF4D4AA2846394605F050FE0B
:10BBA000F8EEC80A01EE100A70EE811ABDEEE18AC5
:10BBB00004F10104B4427FF4C3AAFFF7DDBA00BF69
:10BBC00008B540F6B450C0F602004BF2E101C0F6F1
:10BBD0000001FAF705FC08BDAFF30080AFF3008069
:10BBE00070B582B004460E4642F64443C2F20103E9
:10BBF0001868002878D00FF053F946F26762C6F251
:10BC0000666282FB00324FEAE071C1EBE20303EBB4
:10BC10008302B0EB820F21D042F64040C2F2010015
:10BC20000168002960D042F64840C2F201004FF698
:10BC3000AC21C0F60101FCF7ABFBFBF769FF28B1B3
:10BC400042F64840C2F20100FCF77AFA42F640435D
:10BC5000C2F201034FF000021A6045E042F6404094
:10BC6000C2F201000168F9B942F64045C2F201058D
:10BC70004FF001032B6042F64845C2F20105284609
:10BC8000FCF70EFA28464FF66061C0F601014FF648
:10BC9000AC22C0F60102FCF77BFB284640F6C051FF
:10BCA000C0F60201FCF774FB42F64840C2F2010004
:10BCB000FCF76EFA41F22332904215D82046F6F78F
:10BCC00083FA04460D463046F6F77EFACDE90001C8
:10BCD00042F64840C2F2010040F6D051C0F60201DF
:10BCE00022462B46FCF754FB02B070BDAFF3008038
:10BCF00008B542F64840C2F2010040F6D851C0F6FD
:10BD0000020141F6B802C2F2010241F28833FCF7A7
:10BD1000EFF942F64443C2F201034FF001021A6008
:10BD200008BD00BFAFF30080AFF30080AFF3008029
:10BD300081B940F2B413C1F20003DA6843F2080398
:10BD4000C2F201031868101A43F2FC51C2F2010159
:10BD500008601A60704700BFAFF30080AFF3008047
:10BD60002DE9F04180460D4617461E4643F2006419
:10BD7000C2F20104236803F10103236004290BDDEF
:10BD800040F6F050C0F6020040F60461C0F6020131
:10BD90004FF07402F7F7ACFF43F20C00C2F201005F
:10BDA0004FF4987101FB0504C4F80C8104F11400F0
:10BDB0004BF69161C0F600012246F9F7E9FD04F166
:10BDC00090004BF62161C0F600012246F9F7E0FD34
:10BDD000204639463246069B02F0F2FF606801F0C9
:10BDE000DFF8024640F62060C0F602002946A3684C
:10BDF000FBF756F82046079903F03AF8BDE8F081C2
:10BE000008B543F20C03C2F201034FF4987202FB2F
:10BE1000003003F02DF808BDAFF30080AFF30080D1
:10BE200038B5044640F2B413C1F20003DD68D0F81F
:10BE3000100100F10100C4F81001C4F81451D4F845
:10BE40000C0140F63861C0F602014FF24462C0F6C0
:10BE500001020FF02DF8D4F81C116A1AC4F82C2135
:10BE6000C4F8185143F2FC53C2F20103186843F2BC
:10BE70000801C2F201010A68AD1A00EBD073B5EBFC
:10BE8000630FC8BFC0EB0505C4F8245138BD00BF1F
:10BE900038B5044640F2B413C1F20003DD68D0F8AF
:10BEA000100100F10100C4F81001C4F81451D4F8D5
:10BEB0000C0140F64061C0F602014FF24462C0F648
:10BEC00001020EF0F5FFD4F818116A1AC4F82821FF
:10BED000D4F81C31E81AC4F82001C4F81C5138BD4C
:10BEE00038B540F29813C1F20003986940F64462F5
:10BEF000C0F60202826148F2A064C0F2010449F671
:10BF00003805C2F201052046F8F7FAFA284607F08C
:10BF100087F9F8E7AFF30080AFF30080AFF300805C
:10BF200008B503695BB940F65460C0F6020040F6FC
:10BF30000461C0F602014FF02A02FAF789FF08BD3A
:10BF400010B543F20C04C2F201044FF4987303FBE2
:10BF500000442046FFF7E4FF40F2B410C1F20000B5
:10BF6000C168D4F8143143F2FC52C2F201021068E5
:10BF7000C91AB1EB800F94BFD4F82C01002010BD7A
:10BF800010B543F20C04C2F201044FF4987303FBA2
:10BF900000442046FFF7C4FFD4F8200110BD00BFC5
:10BFA000F8B52DED048B04460E460846FFF7C8FF92
:10BFB00009EE100A3046FFF7E3FF08EE900A4FF64D
:10BFC000AC25C0F60105204640F68461C0F60201AA
:10BFD00032462B46FCF7DCF9B8EEC99AF8EEE88A4F
:10BFE0009FED238A69EE087A204687EEA80A10EEB4
:10BFF000101A4FF00202FCF7EBF94FF69027C0F64B
:10C000000107204639462A46FCF7C2F9204640F689
:10C010009061C0F6020132462B46FCF7B9F9204682
:10C0200089EE089A19EE101A4FF00202FCF7D0F9C7
:10C03000204639462A46FCF7ABF9204640F69C617B
:10C04000C0F6020132462B46FCF7A2F9204688EEE4
:10C05000888A18EE101A4FF00202FCF7B9F9204650
:10C0600039462A46FCF794F9BDEC048BF8BD00BFB5
:10C070000000C842AFF30080AFF30080AFF3008050
:10C0800010B504464FF00001FFF78AFF20464FF03D
:10C090000101FFF785FF10BDAFF30080AFF3008013
:10C0A00010B582B043F20460C2F2010040F6A8610C
:10C0B000C0F60201FCF73CF84FF0080300934FF084
:10C0C0000104019440F6B060C0F602004FF0000198
:10C0D0004AF21C12C2F201020B46C4F20203FFF73D
:10C0E0003FFE4FF007000090019440F6BC60C0F6A0
:10C0F000020021464AF20412C2F201024FF48053B8
:10C10000C4F20203FFF72CFE4BF63150C0F60000DC
:10C1100040F6C861C0F602010EF022FD40F6D8607C
:10C12000C0F602004BF60161C0F60001FAF760F9B3
:10C130004FF00001009142F65050C2F201004FF45E
:10C140002E714FF040024BF6E163C0F60003F8F7A2
:10C15000AFF902B010BD00BFAFF30080AFF30080B5
:10C1600070B584B005460E4649F6A424C2F2010417
:10C170002046FCF7F5FC43F20872C2F20102167089
:10C180004FF00003009301934FF0FF3002902046E0
:10C19000A9B24FF00103FCF78BFC2046FCF7F8FC3A
:10C1A00004B070BDAFF30080AFF30080AFF3008048
:10C1B00010B54FF48064C4F2020440F6E060C0F6AB
:10C1C000020021464FF0030240F2023300F0A8FFC4
:10C1D00040F6EC60C0F6020021464FF0050240F246
:10C1E000023300F09DFF40F6FC60C0F602002146DD
:10C1F0004FF0040240F2023300F092FF10BD00BF86
:10C2000008B5F9F77DFD01F06BF904F0C9FF02F004
:10C210007FF901F075F900F003FD0EF0A1FD00F0CB
:10C22000C7FDFFF7C5FF02F09BFB02F0E1FC01F048
:10C2300027FC40F63C70C0F602004CF26111C0F6DB
:10C240000001FAF7D5F802F05BFD08BDAFF30080FE
:10C2500070B4002A1FDD4FEA430301EB40014FF0A9
:10C2600000052C466FEA0500861806F001004E5BBB
:10C2700004F10104ED18944214D10EE0485B361825
:10C28000ED18485B10FA86F6B6B204F10204ED1818
:10C290009442F3D101E04FF0000696FBF2F290B227
:10C2A00070BC70470028E9D0485B3618B6B204F17C
:10C2B0000104ED189442E1D1EFE700BFAFF3008035
:10C2C00038B50378042B78D143F67010C2F2010020
:10C2D000026802F10102026040F2B411C1F20001F1
:10C2E000CD6843F67414C2F20104A56143F6041547
:10C2F000C2F201054FF0000029464FF001024FF055
:10C300000A03FFF7A5FF20804FF0010029460246EF
:10C310004FF00A03FFF79CFF60804FF002002946B0
:10C320004FF001024FF00A03FFF792FFA0804FF099
:10C33000030029464FF001024FF00A03FFF788FF80
:10C34000E0804FF0040029464FF001024FF00A034D
:10C35000FFF77EFF20814FF0050029464FF00102D4
:10C360004FF00A03FFF774FF60814FF00600294683
:10C370004FF001024FF00A03FFF76AFFA0814FF070
:10C38000070029464FF001024FF00A03FFF760FF54
:10C39000E0814FF0080029464FF001024FF00A03F8
:10C3A000FFF756FF20824FF0090029464FF00102A7
:10C3B0004FF00A03FFF74CFF608238BDAFF30080F7
:10C3C00008B54FF0200383F31188F7F779FD49F69C
:10C3D0000020C2F2010040F64071C0F6020143F2B3
:10C3E0000C72C2F201024FF00103FCF7E1FAF7F719
:10C3F0003FFD4FF0000383F3118808BDAFF30080C9
:10C4000008B54FF0200383F31188F7F759FD49F67B
:10C41000CC10C2F2010041F2E411C2F2000143F675
:10C420000412C2F201024FF00103FCF7C1FAF7F760
:10C430001FFD4FF0000383F3118808BDAFF30080A8
:10C4400008B50378042B11D14FF0000043F20C71B2
:10C45000C2F201014FF001021346FFF7F9FE43F665
:10C460001C11C2F20101086005F0A2F808BD00BF6E
:10C4700008B543F6E410C2F2010040F67071C0F650
:10C48000020143F6E013C2F201031A68FCF728F830
:10C4900008BD00BFAFF30080AFF30080AFF30080B2
:10C4A00008B543F6E013C2F201031860FFF7E0FF9E
:10C4B00008BD00BFAFF30080AFF30080AFF3008092
:10C4C00043F67413C2F2010333F8100080B27047D0
:10C4D00008B543F69013C2F2010353F82000FFF7AA
:10C4E000EFFF08BDAFF30080AFF30080AFF3008033
:10C4F00008B5FFF7EDFF07EE900AB8EEE77AB0EE69
:10C50000080A67EE000A9FED101AC0EE811A41F288
:10C510007823C2F20003186800F53B6191ED002A10
:10C5200061EE822A12EE900AF5F74EFE02460B46A5
:10C5300043F6E410C2F2010040F67C71C0F602013D
:10C54000FBF7AEFF08BD00BF00F07F45AFF30080F2
:10C5500008B50F282CD8DFE800F0080808080808FC
:10C5600008083A3A0D12171C21264FF00000C4F2B9
:10C57000020008BD4FF40060C4F2020008BD4FF491
:10C580000060C4F2020008BD4FF40060C4F2020073
:10C5900008BD4FF40060C4F2020008BD4FF4006013
:10C5A000C4F2020008BD4FF40060C4F2020008BDEE
:10C5B00040F69070C0F6020040F6A471C0F6020189
:10C5C0004FF0F802FAF744FC4FF0000008BD4FF4BA
:10C5D0008060C4F2020008BDAFF30080AFF30080BA
:10C5E00008B50F282AD8DFE800F008380B0E111420
:10C5F000171A083808381D2023264FF0000008BD00
:10C600004FF0020008BD4FF0030008BD4FF00400DA
:10C6100008BD4FF0050008BD4FF0060008BD4FF003
:10C62000070008BD4FF0020008BD4FF0030008BD31
:10C630004FF0040008BD4FF0050008BD40F69070B3
:10C64000C0F6020040F6A471C0F602014FF49172E8
:10C65000FAF7FEFB4FF0FF3008BD4FF0010008BDB8
:10C6600038B50C4643F69013C2F2010343F821009B
:10C6700043F62011C2F2010141F8204005280BDCED
:10C6800041F2E415C2F2000500EB800004FA00F369
:10C690006A6A991869620CE041F2E415C2F2000579
:10C6A00000EB8000A0F11E0004FA00F32A6A99183A
:10C6B00029622046FFF74CFF05462046FFF790FF12
:10C6C000044640F6BC70C0F6020040F6C871C0F6E1
:10C6D0000201FAF7E5FB40F6CC70C0F602002946ED
:10C6E00022464FF0030300F01BFD38BDAFF300807E
:10C6F00043F62013C2F2010353F82000704700BF35
:10C700002DE9F04F2DED028B83B043F6E414C2F215
:10C7100001042046FBF74CFE4FF00000FFF7E8FF56
:10C720000546FFF715FF07462846FFF759FF06465F
:10C730004FF00000FFF7C4FE8046384600F030FCA2
:10C74000034640F6D877C0F60207009620463946E1
:10C750004FF00002FBF71CFE40F6E476C0F602063E
:10C76000204631462A464346FBF712FE40F6F47552
:10C77000C0F6020507EE108AF8EEC77AF0EE088AD6
:10C7800027EEA80A9FEDC08AC0EE080A10EE900AB4
:10C79000F5F71AFD02460B4620462946FBF7F8FD41
:10C7A0002046FBF785FD2046FBF7CAFC2046FBF739
:10C7B000FFFD4FF00100FFF79BFF8046FFF7C8FE2B
:10C7C00083464046FFF70CFF82464FF00100FFF71B
:10C7D00077FE8146584600F0E3FB0346CDF800A003
:10C7E000204639464FF00102FBF7D2FD2046314684
:10C7F00042464B46FBF7CCFD01EE109AF8EEC11A0B
:10C8000021EEA82AC2EE082A12EE900AF5F7DCFC07
:10C8100002460B4620462946FBF7BAFD2046FBF7A9
:10C8200047FD2046FBF78CFC2046FBF7C1FD4FF08F
:10C830000200FFF75DFF8046FFF78AFE8346404611
:10C84000FFF7CEFE82464FF00200FFF739FE814629
:10C85000584600F0A5FB0346CDF800A02046394617
:10C860004FF00202FBF794FD2046314642464B460C
:10C87000FBF78EFD03EE109AF8EEC33A23EEA84ABA
:10C88000C4EE084A14EE900AF5F79EFC02460B46E9
:10C8900020462946FBF77CFD2046FBF709FD204694
:10C8A000FBF74EFC2046FBF783FD4FF00300FFF73C
:10C8B0001FFF8046FFF74CFE83464046FFF790FE81
:10C8C00082464FF00300FFF7FBFD8146584600F01B
:10C8D00067FB0346CDF800A0204639464FF003021F
:10C8E000FBF756FD2046314642464B46FBF750FDCE
:10C8F00005EE109AF8EEC55A25EEA86AC6EE086A4B
:10C9000016EE900AF5F760FC02460B4620462946D3
:10C91000FBF73EFD2046FBF7CBFC2046FBF710FC67
:10C920002046FBF745FD4FF00400FFF7E1FE80468F
:10C93000FFF70EFE83464046FFF752FE82464FF059
:10C940000400FFF7BDFD8146584600F029FB034671
:10C95000CDF800A0204639464FF00402FBF718FD41
:10C960002046314642464B46FBF712FD07EE109A31
:10C97000F8EEC77A27EEA80AC0EE080A10EE900A71
:10C98000F5F722FC02460B4620462946FBF700FD40
:10C990002046FBF78DFC2046FBF7D2FB2046FBF739
:10C9A00007FD4FF00500FFF7A3FE8046FFF7D0FD1F
:10C9B00083464046FFF714FE82464FF00500FFF71E
:10C9C0007FFD8146584600F0EBFA0346CDF800A003
:10C9D000204639464FF00502FBF7DAFC2046314687
:10C9E00042464B46FBF7D4FC01EE109AF8EEC11A12
:10C9F00021EEA82AC2EE082A12EE900AF5F7E4FB0F
:10CA000002460B4620462946FBF7C2FC2046FBF7B0
:10CA10004FFC2046FBF794FB2046FBF7C9FC4FF088
:10CA20000600FFF765FE8046FFF792FD834640460D
:10CA3000FFF7D6FD82464FF00600FFF741FD814625
:10CA4000584600F0ADFA0346CDF800A0204639461E
:10CA50004FF00602FBF79CFC2046314642464B460F
:10CA6000FBF796FC03EE109AF8EEC33A23EEA84AC1
:10CA7000C4EE084A14EE900AF5F7A6FB02460B46F0
:10CA80002046294602E000BF00F07F45FBF780FC0E
:10CA90002046FBF70DFC2046FBF752FB2046FBF738
:10CAA00087FC4FF00700FFF723FE8046FFF750FD9D
:10CAB00083464046FFF794FD82464FF00700FFF79C
:10CAC000FFFC8146584600F06BFA0346CDF800A003
:10CAD000204639464FF00702FBF75AFC2046314604
:10CAE00042464B46FBF754FC05EE109AF8EEC55A49
:10CAF00025EEA86AC6EE086A16EE900AF5F764FB02
:10CB000002460B4620462946FBF742FC2046FBF72F
:10CB1000CFFB2046FBF714FB2046FBF749FC4FF008
:10CB20000800FFF7E5FD8046FFF712FD834640460B
:10CB3000FFF756FD82464FF00800FFF7C1FC814623
:10CB4000584600F02DFA0346CDF800A0204639469D
:10CB50004FF00802FBF71CFC2046314642464B468C
:10CB6000FBF716FC07EE109AF8EEC77A27EEA80A34
:10CB7000C0EE080A10EE900AF5F726FB02460B46B7
:10CB800020462946FBF704FC2046FBF791FB204694
:10CB9000FBF7D6FA2046FBF70BFC4FF00900FFF736
:10CBA000A7FD8046FFF7D4FC83464046FFF718FDFB
:10CBB00082464FF00900FFF783FC8146584600F09B
:10CBC000EFF90346CDF800A0204639464FF00902A0
:10CBD000FBF7DEFB2046314642464B46FBF7D8FBCF
:10CBE00001EE109AF8EEC11A61EEA88AC8EE888AA2
:10CBF00018EE900AF5F7E8FA02460B462046294659
:10CC0000FBF7C6FB2046FBF753FB2046FBF798FAE1
:10CC100003B0BDEC028BBDE8F08F00BFAFF3008026
:10CC200008B543F6E410C2F2010040F6FC71C0F60C
:10CC3000020143F21072C2F201024FF4FA73FBF7E1
:10CC400057FAFFF715FC40F67070C0F602004CF280
:10CC5000A141C0F60001F9F7C3FB49F6CC10C2F2BE
:10CC600001004FF00001FBF76BFE49F60020C2F215
:10CC700001004FF00001FBF763FE41F2E413C2F242
:10CC800000034FF00001196259620846FFF7E8FC03
:10CC90004FF001000146FFF7E3FC4FF002000146B0
:10CCA000FFF7DEFC4FF003000146FFF7D9FC4FF021
:10CCB00004000146FFF7D4FC4FF005004FF00601D9
:10CCC000FFF7CEFC4FF006004FF00701FFF7C8FC5E
:10CCD0004FF007004FF00B01FFF7C2FC4FF00800C8
:10CCE0004FF00C01FFF7BCFC4FF009004FF00D01B5
:10CCF000FFF7B6FC4AF24810C2F2010041F27C1183
:10CD0000C2F20001FCF7FCFF4AF23410C2F201004B
:10CD100041F2B011C2F20001FCF7F2FF41F2000053
:10CD2000C0F602004CF2F141C0F60001F9F758FBE1
:10CD300041F20400C0F602004CF20171C0F600019D
:10CD4000F9F746FB08BD00BFAFF30080AFF30080EA
:10CD500008B543F6E013C2F20103186808B1FFF703
:10CD6000CFFC08BDAFF30080AFF30080AFF30080CD
:10CD700008B5044B834214BF032001200DF008FFC7
:10CD800008BD00BFECA00120AFF30080AFF300802E
:10CD900008B5044B834214BF022000200DF0F8FEBA
:10CDA00008BD00BFECA00120AFF30080AFF300800E
:10CDB00070B54AF2EC04C2F201044FF40065C4F20B
:10CDC000020543F6F430C2F2010021462A464FF034
:10CDD000060301F0F5FF41F20C26C2F200064FF007
:10CDE00000033375284600F0DBF8014641F21000DD
:10CDF000C0F602004FF00602FAF752F8204631461C
:10CE0000FBF7EEFE2046FBF75BFF41F27820C2F213
:10CE100000000168D1F8482C5AB34AF2D404C2F297
:10CE200001044FF00005C4F2020543F6E820C2F207
:10CE3000010021462A464FF0050301F0C1FF41F2EF
:10CE40000C26C2F200064FF000033375284600F0AE
:10CE5000A7F8014641F23800C0F602004FF0050283
:10CE6000FAF71EF820463146FBF7BAFE2046FBF7DC
:10CE700027FF70BDAFF30080AFF30080AFF30080F9
:10CE800008B54FF00003C4F20203984232D04FF4C9
:10CE90008061C4F2020188422FD04FF40062C4F2D4
:10CEA000020290422CD04FF44063C4F20203984235
:10CEB00029D04FF48051C4F20201884226D04FF4A9
:10CEC000A052C4F20202904223D04FF4E053C4F2C5
:10CED0000203984220D041F26000C0F6020041F205
:10CEE0006C01C0F602014FF03C02F9F7B1FF4FF0C0
:10CEF000FF3008BD4FF0000008BD4FF0010008BD35
:10CF00004FF0020008BD4FF0030008BD4FF00400D1
:10CF100008BD4FF0050008BD4FF0060008BD00BF7A
:10CF2000F8B5154D4FF0000441F28807C0F602072E
:10CF300005F104066A681AB138462146F9F7B0FFD0
:10CF400004F10104214606F10405726862B90EE09D
:10CF500041F29800C0F6020043F63063C2F20103CA
:10CF60001968F9F79DFFF8BD3846F9F799FF04F104
:10CF70000104702CDCD1EBE7303E0120AFF30080E0
:10CF80000EB400B582B003AA52F8041B0192F8F760
:10CF900017F902B05DF804EB03B07047AFF30080FF
:10CFA0004FF00003C4F20203984228D04FF480618E
:10CFB000C4F20201884227D04FF40062C4F2020298
:10CFC000904226D04FF44063C4F20203984225D029
:10CFD0004FF48051C4F20201884224D04FF4A05291
:10CFE000C4F20202904223D04FF4E053C4F2020391
:10CFF000984222D141F2C800C0F60200704741F2C7
:10D00000B000C0F60200704741F2B400C0F6020062
:10D01000704741F2B800C0F60200704741F2BC0010
:10D02000C0F60200704741F2C000C0F6020070472F
:10D0300041F2C400C0F60200704741F2CC00C0F6D5
:10D0400002007047AFF30080AFF30080AFF30080C1
:10D05000F8B5044600F0FCF90746204600F008FA4F
:10D06000064643F60054C2F201044FF00005E560A5
:10D070003846FFF795FF0246204641F60C41C0F6C0
:10D0800002013346FFF77CFF6268E368D55443F63C
:10D090001860C2F20100F8BDAFF30080AFF300806A
:10D0A00008B543F61450C2F2010041F2D401C0F6B3
:10D0B0000201FBF73DF843F60050C2F2010043F6CF
:10D0C0001861C2F201014FF014024FF00003F8F7AB
:10D0D00007FB43F63460C2F20100A0F1040300F53F
:10D0E000DE704FF0000103F10402596003F1080300
:10D0F00051608342F7D143F62C63C2F201034FF033
:10D100000100186041F2E000C0F602004CF6217107
:10D11000C0F60001F9F75CF908BD00BFAFF300806D
:10D120002DE9F04383B0064688461446994643F6F7
:10D130002C63C2F20103186858B941F2E800C0F646
:10D14000020041F26C01C0F602014FF06E02F9F7E5
:10D150007FFE4046FFF724FF074641F20010C0F66D
:10D16000020031463A462346F9F79AFE43F6145533
:10D17000C2F20105284641F21011C0F60201324602
:10D18000FBF706F94FF6AC21C0F6010100912846E5
:10D1900041F21811C0F602013A462346FBF7F8F8AF
:10D1A0002846FAF795FF4046FFF76AFE04EB0012A7
:10D1B00043F63463C2F2010353F8220050B10090E9
:10D1C00041F22410C0F60200394622463346F4F7F5
:10D1D00043FE15E043F63461C2F2010141F82260DA
:10D1E00043F63063C2F201031A6802F101021A60C9
:10D1F00040464FF0010101FA04F14A4608F070FC84
:10D2000003B0BDE8F08300BFAFF30080AFF3008050
:10D2100038B504460D4644F61823C2F2010353F80C
:10D22000200058B941F2E010C0F6020041F200219E
:10D23000C0F602014FF03802F6F75AFD44F6182105
:10D24000C2F2010151F824202846116804F0B0FB15
:10D25000014604EB440444F2B023C2F2010303EBA1
:10D2600084002A4601F02CFD38BD00BFAFF30080DA
:10D27000F8B540F29813C1F20003986941F2182200
:10D28000C0F6020282614FF002054FF0010640F63F
:10D29000E4444FF00007F3F72BFC10B9F3F746FA1C
:10D2A00018B128463146FFF7B3FF2046F7F728F9B3
:10D2B000FAF7F6F918B928463946FFF7A9FF2046CC
:10D2C000F7F71EF9E7E700BFAFF30080AFF3008088
:10D2D0002DE9F04740F29813C1F20003986941F23A
:10D2E0002822C0F6020282614FF003084FF00007C7
:10D2F0004FF004064FF0010548F2A06AC0F2010A9F
:10D3000044F6D359C1F2620900F04AFD00280CBF6F
:10D310002124642440463946FFF77AFF30462946E7
:10D32000FFF776FF0AFB04F101F1FF33A9FB03309D
:10D330004FEA901404F101042046F7F7E1F8404663
:10D340002946FFF765FF30463946FFF761FF204663
:10D35000F7F7D6F8D8E700BFAFF30080AFF300804F
:10D3600008B54FF00001FFF753FF08BDAFF3008091
:10D3700008B54FF00101FFF74BFF08BDAFF3008088
:10D3800008B500EB400044F2B023C2F2010303EB06
:10D39000800001F08DFC08BDAFF30080AFF300808A
:10D3A00038B504460D460B68032B0BD941F23820E3
:10D3B000C0F6020041F20021C0F602014FF0310236
:10D3C000F6F796FC44F61820C2F2010040F824500B
:10D3D00020464FF00001FFF71BFF38BDAFF3008080
:10D3E0002DE9F04182B080460D4617461E46089C46
:10D3F0002368032B0BD941F23820C0F6020041F21A
:10D400000021C0F602014FF03102F6F771FC2068EE
:10D4100001288CBF0521012105EB45020091404602
:10D4200044F2B023C2F2010303EB82013A463346D1
:10D4300001F02EFC28462146FFF7B2FF02B0BDE8FE
:10D44000F08100BFAFF30080AFF30080AFF3008046
:10D450004FEA101041F2C013C0F6020353F8200047
:10D46000704700BFAFF30080AFF30080AFF30080E0
:10D4700000F00F00704700BFAFF30080AFF30080F3
:10D480002DE9F04182B007460E46144698461046F4
:10D49000FFF7DEFF05462046FFF7EAFF0346CDF81B
:10D4A0000080384631462A46FFF79AFF02B0BDE8B1
:10D4B000F08100BFAFF30080AFF30080AFF30080D6
:10D4C00010B582B043F6F474C2F201040094FFF781
:10D4D00087FF02B010BD00BFAFF30080AFF3008044
:10D4E00008B541F25820C0F602004FF002014FF497
:10D4F0004062C4F202024FF00E03FFF7E1FF08BDE5
:10D5000030B583B04FF44064C4F2020441F26020AD
:10D51000C0F602004FF0000122464FF00D03FFF766
:10D52000CFFF41F27420C0F602004FF00101224605
:10D530004FF00C03FFF7C4FF41F28820C0F6020051
:10D540004FF0030122464FF00F03FFF7B9FF4FF4EE
:10D550000065C4F2020541F2A020C0F602004FF0BF
:10D5600004012A464FF00E03FFF7AAFF41F2AC2058
:10D57000C0F602004FF0070122464FF00603FFF706
:10D580009FFF41F2B420C0F602004FF030012A465E
:10D590004FF00903FFF794FF41F2CC20C0F60200E0
:10D5A0004FF0330122464FF00703FFF789FF41F2A6
:10D5B000D420C0F602004FF034014FF4E052C4F220
:10D5C00002024FF00003FFF77BFF41F2DC20C0F6C0
:10D5D00002004FF0350122464FF00503FFF770FFC0
:10D5E00041F2E420C0F602004FF0360122464FF02F
:10D5F0000303FFF765FF41F2EC20C0F602004FF095
:10D60000370122464FF00403FFF75AFF41F2F4209E
:10D61000C0F602004FF031012A464FF00D03FFF72C
:10D620004FFF41F20430C0F602004FF032012A46AB
:10D630004FF00F03FFF744FF4FF000004FF00101E0
:10D64000FFF7E6FD4FF001000146FFF7E1FD4FF067
:10D6500002004FF00101FFF7DBFD4FF003004FF038
:10D660000101FFF7D5FD4FF007004FF00101FFF773
:10D67000CFFD4FF004004FF00101FFF7C9FD4FF05F
:10D6800030004FF00101FFF7C3FD42F21070F6F7D2
:10D6900037FF4FF000000146FFF7BAFD4FF00100E1
:10D6A0004FF00001FFF7B4FD4FF002004FF0000112
:10D6B000FFF7AEFD4FF003004FF00001FFF7A8FDAC
:10D6C0004FF007004FF00001FFF7A2FD4FF00400FC
:10D6D0004FF00001FFF79CFD4FF030004FF00001CC
:10D6E000FFF796FD4FF00004009444F26070C2F220
:10D6F00001004FF42E714FF040024DF2D123C0F6DD
:10D700000003F6F7D5FE009443F6F870C2F201006C
:10D710004FF42E714FF040024DF27123C0F600031A
:10D72000F6F7C6FE03B030BDAFF30080AFF3008064
:10D7300008B544F6A833C2F20103196811B34FF0DB
:10D74000A80202FB00F000280FDD4FF000024FF0AE
:10D75000010383422BD107E0D21803F10103D21851
:10D7600003F101038342F7D102BB41F21030C0F64E
:10D77000020041F21C31C0F602014FF04002F6F700
:10D78000B7FA08BD48F2A062C0F2010202FB00F045
:10D7900000F1FF304DF68363C4F21B33A3FB00217D
:10D7A0004FEA914000F10100F6F7AAFE08BD4FF0E4
:10D7B00001010029D0D0D2185B188342CCD1D3E725
:10D7C000F0B585B041F27823C2F200031968D1F8B0
:10D7D000E42B012A47D144B2002CACBF4FF00055D6
:10D7E0000025002CB4BF4FF4005300231D434FF419
:10D7F0008061C4F202018D6100F04002D4B2002CBD
:10D8000014BF4FF400654FF000654FF48063C4F21D
:10D8100002039D6100F02001CAB2002A14BF4FF438
:10D8200000444FF000444FF48055C4F20205AC614F
:10D8300000F01000C3B2002B14BF4FF400514FF0A2
:10D8400000514FF48054C4F20204A1614FF400650A
:10D8500025834FF00A00FFF76BFF65834FF0280028
:10D86000FFF766FF2FE049F6A425C2F2010528461E
:10D87000FBF776F944F6AC36C2F201064FF004002D
:10D8800030704FF00004009401944FF0FF3702977E
:10D8900028464FF0200132464FF00103FBF708F90C
:10D8A0004FF00A00FFF744FF347000940194029790
:10D8B00028464FF0200132464FF00103FBF7F8F8FD
:10D8C0002846FBF765F905B0F0BD00BFAFF3008057
:10D8D000F0B583B04FF48054C4F202042046FFF741
:10D8E0005FFB07462046FFF75BFB44F6B035C2F20C
:10D8F000010500904FF00B060196284641F23831A1
:10D90000C0F602013A464FF00903FAF7C9FD204676
:10D91000FFF746FB07462046FFF742FB00904FF01B
:10D920000F030193284641F25031C0F602013A46F6
:10D930004FF00D03FAF7B4FD4FF48064C4F2020413
:10D940002046FFF72DFB07462046FFF729FB0090F6
:10D950004FF00D000190284641F26831C0F60201F7
:10D960003A463346FAF79CFD03B0F0BDAFF30080B2
:10D9700010B504464FF48053C4F202034FF4007212
:10D980005A83FFF71DFF4FEA041000F0F000FFF785
:10D9900017FF10BDAFF30080AFF30080AFF300803E
:10D9A00070B506464FF48054C4F202044FF400757B
:10D9B0002583FFF705FF4FEA061000F0F000FFF7A0
:10D9C000FFFE658370BD00BFAFF30080AFF3008042
:10D9D00038B504460D4641F27823C2F200031868B8
:10D9E000D0F8F41B8C420BDD41F28030C0F602000F
:10D9F00041F21C31C0F602014FF08202F6F778F9CD
:10DA000044F6B442C2F201021460A5F1800541F26D
:10DA10000043C0F6020353F824002918C8B2FFF7E8
:10DA2000A7FF38BDAFF30080AFF30080AFF30080F5
:10DA300008B50A280DD144F6B443C2F201031868B0
:10DA400000F101001860C0B24FF00001FFF7C0FF05
:10DA500008BDFFF7A5FF08BDAFF30080AFF300805E
:10DA600010B50446007828B1FFF7E2FF14F8010F63
:10DA70000028F9D110BD00BFAFF30080AFF30080E4
:10DA800038B544F6B030C2F2010041F29031C0F630
:10DA90000201FAF74DFB41F2A030C0F602004DF64C
:10DAA000D101C0F60001F8F793FC41F27823C2F2ED
:10DAB00000031868D0F8E43B012B55D14FF4805493
:10DAC000C4F2020441F2A830C0F6020021464FF031
:10DAD0000902FFF725FB41F2B030C0F602002146F3
:10DAE0004FF00B024FF00103FFF71AFB41F2B83081
:10DAF000C0F6020021464FF00D024FF00103FFF780
:10DB00000FFB41F2C030C0F6020021464FF00F0279
:10DB10004FF00103FFF704FB4FF48065C4F20205E8
:10DB200041F2C830C0F6020029464FF00B024FF018
:10DB30000103FFF7F5FA41F2D030C0F602002946A2
:10DB40004FF00D024FF00103FFF7EAFA4FF00071BA
:10DB5000A1614FF00062A2614FF00053A3614FF04A
:10DB60000040A061AA61AB6141F28830F6F7C8FCC1
:10DB70004FF03000FFF724FE4FF06400F6F7C0FCD2
:10DB80004FF03000FFF71CFE4FF02000FFF718FEAB
:10DB90004FF00400F6F7B4FC4FF02000FFF710FE42
:10DBA0004FF08000FFF70CFE4FF00400F6F7A8FCE2
:10DBB0004FF00000FFF704FE4FF0C000FFF700FE3B
:10DBC0004FF00400F6F79CFC4FF00000FFF7F8FD63
:10DBD0004FF00100FFF7F4FD4FF0C800F6F790FC9E
:10DBE0004FF00000FFF7ECFD4FF06000FFF7E8FD9D
:10DBF0004FF000000146FFF7EBFE41F2D830C0F6CF
:10DC00000200FFF72DFF41F2E830C0F60200FFF7F7
:10DC100027FF38BDAFF30080AFF30080AFF3008083
:10DC200010B5044644F6A833C2F201034FF00102D6
:10DC30001A604FF000000146FFF7CAFE41F2F430CF
:10DC4000C0F60200FFF70CFF2046FFF709FF10BDEA
:10DC5000022914D0032906D001290DD141F2C05068
:10DC6000C0F602007047032A0ED841F29050C0F669
:10DC7000020000EBC20070474FF00000704741F215
:10DC80009040C0F6020070474FF00000704700BFA0
:10DC900010B50446022923D14FF0200383F31188E5
:10DCA000F6F70EF920464FF0010141F21042C0F69E
:10DCB0000202FCF755FE20464FF0020141F2A0425D
:10DCC000C0F60202FCF74CFE44F6B840C2F2010076
:10DCD000FCF7CEFAF6F7CCF84FF0000383F3118887
:10DCE00010BD00BFAFF30080AFF30080AFF3008042
:10DCF00038B544F6B845C2F201052846FCF740FAAB
:10DD000041F2B054C0F6020428462146FCF768FAF6
:10DD10002468236D9A6B22F40020986348F2A06077
:10DD2000C0F20100F6F7ECFB204641F2D041C0F60C
:10DD30000201FCF7D5FD216D8C6B44F400238B634D
:10DD40004AF2D410C2F201004FF00001FCF7F8F8DB
:10DD50004FF00004C4F2020420464FF0040140F2E8
:10DD6000823207F0BDFE20464FF0080140F28232B9
:10DD700007F0B6FE38BD00BFAFF30080AFF3008000
:10DD800044F6B843C2F20103D3F85402016808789C
:10DD9000042814BF00200120704700BFAFF30080AB
:10DDA00008B5FFF7EDFF08BDAFF30080AFF30080CB
:10DDB0004FF47053C4F202031869002811DA4FF4CB
:10DDC0007051C4F2020140F22312C4F267524A6059
:10DDD00048F6AB13CCF6EF534B6008694FEAD070AE
:10DDE00070474FF000007047AFF30080AFF3008042
:10DDF0004FF47053C4F202031A6942F001021A612F
:10DE000001604FF47050C4F20200C16811F4803F09
:10DE1000FBD14FF47053C4F202031A6922F00100DF
:10DE200018617047AFF30080AFF30080AFF300805C
:10DE300003280BD904280CD0A0F1050000F0FF0046
:10DE4000062894BF4FF40030002070474FF4804004
:10DE500070474FF480307047AFF30080AFF300801D
:10DE600070B50446E0B100F1FF3303F00106DCB207
:10DE70002046FFF7DDFF00F10065ACB912E004F1C8
:10DE8000FF31CCB22046FFF7D3FF2D1804F1FF324B
:10DE9000D4B22046FFF7CCFF2D18002CEFD101E0C3
:10DEA0004FF00065284670BD76B2002EE7D004F131
:10DEB000FF30C4B22046FFF7BBFF2D18002CDED187
:10DEC000F0E700BFAFF30080AFF30080AFF3008056
:10DED00008B500F10100C0B2FFF7C2FF08BD00BFE6
:10DEE00038B505464FF0000402E004F10104E4B245
:10DEF0002046FFF7EDFFA842F7D9204638BD00BF06
:10DF0000032914D90368B3F1FF3F05D025E0186851
:10DF1000B0F1FF3F42D023E011F0040F36D000F102
:10DF200004031846A1F104021146032AEFD8D1B127
:10DF30000378FF2B1AD1091801F1FF32131A13F0DD
:10DF4000010F05D018E010F8013FFF2B19D010E0A9
:10DF50009042F8D14FF0010070474FF00000704739
:10DF60004FF0000070474FF0010070474FF0000085
:10DF700070474FF00000704710F8011FFF29E7D0ED
:10DF8000F7E710F8011FFF29E2D0F2E7A1F1040141
:10DF900050F8042FB2F1FF3FC1D0E1E703F10400D4
:10DFA000A2F104015A68B2F1FF3FB8D0D8E700BF30
:10DFB00038B50446FFF7FCFE002877D14FF47052C5
:10DFC000C4F20202D36813F4803FFBD14FF47050C7
:10DFD000C4F20200016921F480750561026942F40E
:10DFE00000730361016921F07805056114F0010FE8
:10DFF00007D04FF47050C4F20200026942F00803E7
:10E00000036104F00201CDB23DB14FF47050C4F28F
:10E010000200026942F01003036104F00401CDB272
:10E020003DB14FF47050C4F20200026942F0200387
:10E03000036104F00801CDB23DB14FF47050C4F259
:10E040000200026942F0400303614FF47051C4F2D0
:10E0500002010D6945F0020008610A6942F480334B
:10E060000B614FF47051C4F20201CD6815F4803F8A
:10E07000FBD14FF47050C4F20200026922F0020397
:10E080000361016941F0004505612046FFF7E8FEA4
:10E0900005462046FFF7CCFE01462846FFF730FF35
:10E0A000002814BF00206FF00A0038BD4FF0FF3089
:10E0B00038BD00BFAFF30080AFF30080AFF3008046
:10E0C000F8B506460C4699B13046FFF709FF0546FC
:10E0D000FFF76EFF074668B92846FFF7F9FE0646C8
:10E0E0002846FFF7A5FEA04204D2241AECD101E095
:10E0F0004FF000073846F8BDAFF30080AFF3008063
:10E1000008B50346084619460EF0CAFE4FF0000057
:10E1100008BD00BFAFF30080AFF30080AFF3008015
:10E120002DE9F04782B0074689469046FFF740FE4A
:10E1300000287BD14FF47052C4F20202D36813F46A
:10E14000803FFBD14FF47050C4F20200016921F40A
:10E1500080720261036943F40071016117F00300EA
:10E1600016D03D1A2C6802AA42F8044DC0F10404EE
:10E17000444528BF44461018494622460EF090FEFA
:10E1800028460199FFF734FE3F19A144C4EB080863
:10E19000B8F1030F30D945463C46C7EB0906A8F154
:10E1A000040ACAF3800A3846F159FFF721FE04F148
:10E1B0000404A5F10405032D3DD80FE02046315994
:10E1C000FFF716FE04F1040420463159FFF710FE54
:10E1D00004F10404A5F10805032DEFD8A8F1040308
:10E1E0004FEA930107F1040707EB810701F10101F1
:10E1F00009EB810908F00308B8F1000F0BD03A6869
:10E2000002A840F8042D494642460EF049FE384621
:10E210000199FFF7EDFD4FF47050C4F2020003695D
:10E2200043F0004101614FF0000001E04FF0FF308A
:10E2300002B0BDE8F087BAF1000FBFD020463159D7
:10E24000FFF7D6FD04F10404A5F10405032DB5D8AC
:10E25000C4E700BFAFF30080AFF30080AFF30080EE
:10E2600008B541F2D050C0F60200F8F719FE41F2AD
:10E27000E450C0F60200F8F713FE41F2F850C0F681
:10E280000200F8F70DFE41F20C60C0F60200F8F74C
:10E2900007FE41F23C60C0F60200F8F701FE08BD3F
:10E2A00010B504460378B3B1F7F7BAFC07EE900A4D
:10E2B000BDEEE70A10EE101A44F64470C2F20100F7
:10E2C00080ED000A002906DD4AF29800C2F2010042
:10E2D000F7F73EFB10BD41F23470C0F60200214654
:10E2E000F8F7DEFD10BD00BFAFF30080AFF3008094
:10E2F00000B58FB04AF29800C2F20100F7F710FBA8
:10E30000014644F64873C2F201031860B0F1FF3FC2
:10E3100006D141F25C70C0F60200F8F7C1FD29E0B9
:10E3200041F27C70C0F6020041F28472C0F6020233
:10E33000F8F7B6FD4AF29800C2F2010005A9F7F716
:10E34000BFFA41F29470C0F60200F8F7A9FD0798F1
:10E35000009006990191059A029241F2B470C0F6BC
:10E3600002000A9B03F26C71099A02F10102089BF8
:10E37000F8F796FD0FB000BDAFF30080AFF300805B
:10E3800008B501464AF29800C2F20100F7F7B0FA68
:10E3900008BD00BFAFF30080AFF30080AFF3008093
:10E3A00008B501464AF29800C2F20100F7F788FA70
:10E3B00008BD00BFAFF30080AFF30080AFF3008073
:10E3C00010B58AB004464EF6B003C0F6010307CB81
:10E3D00020606160A2601A889878A281A0734AF2D6
:10E3E0009800C2F2010001A9F7F76AFA44F64070FA
:10E3F000C2F20100059901F10101FAF769F90599E5
:10E40000082909DC4FF03001217044F64073C2F254
:10E4100001031A78627007E044F64073C2F2010308
:10E420001A7822705878607044F64070C2F2010089
:10E430000499FAF74DF90498092809DC4FF03000E7
:10E44000E07044F64071C2F201010B78237107E0DD
:10E4500044F64071C2F201010B78E3704A782271F0
:10E4600044F64070C2F201000399FAF731F9039AB9
:10E47000092A09DC4FF03002A27144F64070C2F262
:10E4800001000178E17107E044F64070C2F201003A
:10E490000178A1714378E37144F64070C2F2010043
:10E4A0000299FAF715F9029B092B09DC4FF03003AA
:10E4B000637244F64070C2F201000278A27207E073
:10E4C00044F64070C2F20100027862724178A17293
:10E4D00044F64070C2F201000199FAF7F9F8019987
:10E4E000092909DC4FF03001217344F64073C2F270
:10E4F00001031878607307E044F64073C2F2010329
:10E50000187820735A7862730AB010BDAFF3008098
:10E5100008B54AF29800C2F2010049F6A171C5F2AD
:10E52000F621F7F715FA41F2D470C0F602004EF268
:10E53000F121C0F60001F7F74BFF41F2E070C0F6A1
:10E5400002004EF2A121C0F60001F7F759FF41F297
:10E55000EC70C0F602004EF26121C0F60001F7F740
:10E5600037FF08BDAFF30080AFF30080AFF300804A
:10E5700008B503460A4641F60000C0F602001946F7
:10E58000F8F78EFC08BD00BFAFF30080AFF300804A
:10E590002DE9F0439DB0064645F2AC13C2F20103EB
:10E5A000187830B941F60020C0F60200F8F778FC80
:10E5B00077E013A831460BF01BFF38B141F6180085
:10E5C000C0F602003146F8F76BFC6AE030460FF007
:10E5D000FFFB054641F63809C0F602090DF1350882
:10E5E0004FF02D0713A80BA90BF052FF002858D1AC
:10E5F0009DF83510002954D011990A782E2AF1D0AF
:10E600009DF8344004F01003D8B258B14FF02F02F7
:10E61000725505F1010570190FF07AFB4FF00003F8
:10E620007355DFE704F0010204F00201CBB204F0FD
:10E63000040E5FFA8EF000280CBF4FF02D0C4FF047
:10E64000530C04F02004E1B200290CBF2D24412416
:10E65000BDF83010BDF83200CDF800C001944FEA8B
:10E66000512404F2BC740294C1F34314039401F0E6
:10E670001F0104914FEAD0210591C0F34510069087
:10E680000B990791CDF8208048463946002A0CBFE7
:10E690002D225222002B0CBF2D234823F8F700FC1B
:10E6A000A0E71DB0BDE8F083AFF30080AFF30080BA
:10E6B00038B545F2AC13C2F20103187830B941F60F
:10E6C0006800C0F60200F8F7EBFB38BD44F64C7466
:10E6D000C2F2010420460BF09BFD20460BF0C8FC63
:10E6E00045F27815C2F201052846FAF709FE2846D8
:10E6F000FBF706F84FF0000001460BF009F9204641
:10E700004FF000014FF409720EF072FC45F2AC11AB
:10E71000C2F201014FF000020A7041F6A000C0F6FB
:10E720000200F8F7BDFB38BDAFF30080AFF3008007
:10E7300010B545F2AC13C2F20103187830B141F6BE
:10E74000B800C0F60200F8F7ABFB10BD45F2781434
:10E75000C2F201042046FAF79BFF204641F228212D
:10E76000C2F20001FAF7A4FF2046FAF719FE30B111
:10E7700041F6E400C0F60200F8F792FB10BD45F246
:10E780006844C2F2010420464FF000014FF40C72BD
:10E790000EF02EFC4FF0000021460BF0B9F80028D7
:10E7A00042D144F64C74C2F2010420464FF00001FD
:10E7B0004FF409720EF01CFC204641F60411C0F61D
:10E7C00002014FF012020BF0C3F8014640B10828D5
:10E7D00006D041F61010C0F60200FFF7C9FE1DE09A
:10E7E00044F64C71C2F201010846C9680BF020FDE5
:10E7F000014630B141F65810C0F60200FFF7B8FEEE
:10E800000CE044F64C70C2F201000BF031FC45F212
:10E81000AC13C2F201034FF001021A7041F664100A
:10E82000C0F60200F8F73CFB10BD00BFAFF300805C
:10E8300010B54FF44060C4F20200FEF7B1FB02468F
:10E8400045F29864C2F20104204641F6B811C0F6C0
:10E8500002014FF00403F9F723FE204641F6C811E8
:10E86000C0F6020145F2AC13C2F201031A7845F278
:10E870007013C2F201031B68F9F712FE10BD00BF4E
:10E8800008B540F29813C1F20003986941F6E81206
:10E89000C0F60202826145F27814C2F2010445F228
:10E8A000AC16C2F201064CF2503521680B682046C6
:10E8B000984718B1307808B9FFF73AFF2846F5F7BE
:10E8C0001FFEF2E7AFF30080AFF30080AFF30080EC
:10E8D00030B583B0044645F2AC13C2F20103187898
:10E8E00098B945F27411C2F201010A682AB941F6D9
:10E8F000F410C0F60200F8F7D3FA45F27413C2F22E
:10E9000001034FF00100186023E020460FF060FA89
:10E91000054645F27011C2F201010A6813180B6036
:10E9200044F64C70C2F2010021462A4601AB0BF0BE
:10E9300097FA01460198854205D941F62420C0F690
:10E940000200FFF715FE44F64C70C2F201000BF016
:10E950008FFB03B030BD00BFAFF30080AFF300808A
:10E9600010B582B045F29860C2F2010041F6402134
:10E97000C0F60201F9F7DCFB45F27814C2F201049B
:10E980002046FAF785FE204641F22821C2F2000116
:10E99000FAF78EFE4FF00003009345F2B010C2F27A
:10E9A00001004FF42E714FF002024EF68103C0F6C3
:10E9B0000003F5F77DFD41F64820C0F602004EF653
:10E9C0003101C0F60001F7F703FD41F65020C0F613
:10E9D00002004EF23171C0F60001F7F7F9FC41F682
:10E9E0005820C0F602004EF6D101C0F60001F7F73C
:10E9F00007FD41F66420C0F602004EF2B161C0F698
:10EA00000001F7F7E5FC41F67020C0F602004EF277
:10EA10009151C0F60001F7F7F3FC02B010BD00BF42
:10EA20002DE9F04140F29813C1F20003986941F6D4
:10EA30008022C0F6020282614FF000044AF25C15A7
:10EA4000C2F2010545F6CC36C2F2010645F29C77CA
:10EA5000C2F2010707F114082968CB6828469847D5
:10EA60000A2803D0B4F5807F34D101E0002C04DD06
:10EA700034194FF0000004F8010C3846314605F017
:10EA8000B7F845F6A830C2F20100FFF789FCFA6B2F
:10EA9000042A0DD1B96A00290ADD7B6945F6A8343C
:10EAA000C2F201042068834202D04046FFF768FCAE
:10EAB00045F6A431C2F201010A6802F101020A60BE
:10EAC00030464FF000014FF480720EF091FA4FF093
:10EAD0000004C1E7305504F10104BDE7AFF3008045
:10EAE00045F29C73C2F2010398687047AFF300804F
:10EAF00070B582B04FF48065C4F202052846FEF777
:10EB00004FFA024645F6A024C2F20104204641F61F
:10EB10008C21C0F602014FF00703F9F7C1FC28462B
:10EB2000FEF73EFA0246204641F69821C0F6020161
:10EB30004FF00603F9F7B4FC45F6A435C2F201051F
:10EB40002E68FFF7CDFFF3F73FFBCDE9000120462C
:10EB500041F6A421C0F6020132464FF00003F9F756
:10EB60009FFC40F2B413C1F20003D3ED037A95ED9C
:10EB7000007AB8EEC70AF8EE670ADFED196A80EE90
:10EB8000A61ADFED181A81EE212AC0EE022A12EE33
:10EB9000900AF3F719FB02460B46204641F6C421C2
:10EBA000C0F60201F9F77CFC45F29C74C2F2010444
:10EBB0002068F3F709FB02460B4641F6DC20C0F65D
:10EBC0000200F8F76DF96068F3F7FEFA02460B46AB
:10EBD00041F6F020C0F60200F8F762F902B070BD0D
:10EBE0000000C84200007A44AFF30080AFF3008019
:10EBF00010B582B045F6A020C2F2010041F60831FE
:10EC0000C0F60201F9F794FA4AF25C10C2F2010070
:10EC100041F24C21C2F20001FBF792F94FF48064FB
:10EC2000C4F2020441F61430C0F6020021464FF04F
:10EC3000060240F28233FEF773FA41F61C30C0F64A
:10EC4000020021464FF0070240F28233FEF768FAD5
:10EC50004FF00003009345F2E870C2F201004FF458
:10EC60002E714FF002024EF62123C0F60003F5F795
:10EC70001FFC41F62430C0F602004EF6F121C0F62A
:10EC80000001F7F7A5FB02B010BD00BFAFF3008095
:10EC900010B54FF0FF348C600A604B6011461A4685
:10ECA000029BFEF73DFA10BDAFF30080AFF300808A
:10ECB00080687047AFF30080AFF30080AFF300804F
:10ECC00070B504460E461546FFF7F2FFA84210D075
:10ECD0002268636816F0010614BF0020012003F1CA
:10ECE000100100FA01F006FA03F340EA0301916112
:10ECF000A56070BDAFF30080AFF30080AFF300807C
:10ED0000704700BFAFF30080AFF30080AFF3008027
:10ED100038B545F6CC43C2F201031D68002D1BDD5A
:10ED200045F6D041C2F201010B681A68824221D037
:10ED300045F6D042C2F201024FF0000115F0010F7A
:10ED400006D119E052F8043F1C6884421CD111E03E
:10ED500001F10101A942F5D141F63030C0F60200BF
:10ED600041F64431C0F602014FF01F02F8F770F887
:10ED70004FF00003184638BD01F1010152F8043F7D
:10ED80001C688442E4D1F5E701F1010152F8043F27
:10ED90001C688442DCD1EDE7AFF30080AFF3008064
:10EDA00008B5FFF7B5FF00F19000F6F711FE08BDBA
:10EDB00008B5FFF7ADFF00F11400F6F709FE08BD36
:10EDC00070B5044616461D4601606260A3604AF2B3
:10EDD0001C13C2F20103994222D04AF2D400C2F2BB
:10EDE000010081421FD04AF2EC02C2F201029142BC
:10EDF0001CD04AF20413C2F20103994208BF032354
:10EE000017D041F66430C0F6020041F64431C0F636
:10EE100002014FF04C02F8F71BF84FF0FF3308E007
:10EE20004FF0010305E04FF0010302E04FF0020351
:10EE3000FFE74FEAC31341F67430C0F602003146D3
:10EE40002A4643F00203FEF76BF945F6CC40C2F2C6
:10EE50000100026845F6D041C2F2010141F82240AA
:10EE600002F10102026070BDAFF30080AFF30080D9
:10EE700038B50446C16039B141F25820C2F20000F1
:10EE80004FF00001017006E041F25823C2F2000386
:10EE90004FF001021A70256823692BB12846F9F753
:10EEA00047FF2846F9F7D4FE284641F25821C2F21E
:10EEB0000001F9F795FE2846F9F702FF4FF001022D
:10EEC000226138BDAFF30080AFF30080AFF3008064
:10EED0002DE9F84F05460F468368022B0BDD41F6FE
:10EEE0008030C0F6020041F69431C0F602014FF0C6
:10EEF0001B02F4F7FDFEA868002823DD05EB87065A
:10EF000006F10C064FF0000441F6B03AC0F6020AD2
:10EF100041F69439C0F602094FF01E0815F804B006
:10EF2000952F04DD504649464246F4F7E1FE584627
:10EF30003168FEF76DF904F1010406F51676A9684B
:10EF4000A142EBDCBDE8F88FAFF30080AFF30080A7
:10EF500008B545F6F040C2F2010041F6C431C0F6F2
:10EF60000201F9F7E5F808BDAFF30080AFF30080C8
:10EF700038B50BF065FF04460BF052FF002804DDA6
:10EF8000D4F1010138BF002101E04FF000014FF042
:10EF90000100FEF73DF94FF000002146FEF738F979
:10EFA00005F0CEFB05F0E4FA4FF06E0103F008FF28
:10EFB00005F006FB05F0B4FA4FF0730103F000FF13
:10EFC0004FF03200FEF7DCF90546A0B105F0F8FA83
:10EFD00041F27824C2F20004236803F53C6191ED0C
:10EFE000000A00EE900AF4EEC00AF1EE10FAD4BF67
:10EFF0000024012413E005F0E3FA41F27823C2F281
:10F000000003196801F6BC32D2ED007A07EE100A4F
:10F01000B4EEE77AF1EE10FAD4BF00240124A54241
:10F0200018D024B141F6D032C0F6020203E041F616
:10F03000D432C0F6020246F61030C2F2010041F6A8
:10F04000D831C0F60201F9F72BFA4FF03200214611
:10F05000FEF7DEF845F60860C2F201004FF47A715F
:10F060004EF67172C0F600024FF00003F9F760FB34
:10F0700038BD00BFAFF30080AFF30080AFF3008076
:10F0800008B559BB4FF03100FEF77AF990B94FF44B
:10F090000060C4F20200FDF783FF024646F610301E
:10F0A000C2F2010041F6E831C0F602014FF00D0353
:10F0B000F9F7F6F94FF03100FEF75AF945F6F4503A
:10F0C000C2F201004FF4D451C0F206014FF2E10246
:10F0D000C0F600024FF00003F9F72AFB08BD00BF9D
:10F0E00008B54FF03100FEF74BF990B14FF40060D6
:10F0F000C4F20200FDF754FF024646F61030C2F299
:10F10000010041F6FC31C0F602014FF00D03F9F7A2
:10F11000C7F94FF03100FEF723F908BDAFF30080C7
:10F1200038B505460C46FDF713FAFDF739FF0146E1
:10F1300020460EF0EDFD2846FDF752FA014604F197
:10F140000200F9F7C5FA204638BD00BFAFF30080D2
:10F1500070B584B005460C4610EE106A084646F6B7
:10F160000031C2F20101FFF7DBFF00903046F3F7F8
:10F170002BF8CDE9020146F61030C2F2010041F64B
:10F180001441C0F602012A462346F9F789F904B072
:10F1900070BD00BFAFF30080AFF30080AFF300801D
:10F1A00038B505460C460846FDF792F907EE900A79
:10F1B000B8EEE70AF0EE080A20EE201ADFED091A91
:10F1C00081EE212A41F27823C2F20003186800F58B
:10F1D0003B61D1ED002A2846214622EE220AFFF7A4
:10F1E000B7FF38BD00F07F45AFF30080AFF300807C
:10F1F00010B541F27824C2F20004236841F62C4095
:10F20000C0F60200D3F8F81BFFF7CAFF21684FF6DB
:10F210007450C0F60100D1F88C1CFFF7C1FF2268C2
:10F2200041F63040C0F60200D2F8901CFFF7B8FF5C
:10F2300023684FF68050C0F60100D3F8941CFFF706
:10F24000AFFF216841F63440C0F60200D1F8981CA7
:10F25000FFF7A6FF2068D0F8844C05F061F800EEB7
:10F26000100A41F63840C0F602002146FFF770FF51
:10F2700010BD00BFAFF30080AFF30080AFF300809C
:10F2800008B546F61030C2F2010041F64041C0F622
:10F290000201F8F74DFF04F053FFFFF759FEFCF7AA
:10F2A00027FD04F0C5FCFCF7FBFE0BF0E9FEF8F7C8
:10F2B000FFFD45F60860C2F201004FF47A714EF688
:10F2C0007172C0F600024FF00003F9F731FA00F056
:10F2D000AFF900F045FA03F003FD02F079F802F00F
:10F2E000E7F9F1F7D3F94FF28100C0F6000041F6DB
:10F2F0005441C0F602010BF033FC4FF00000014610
:10F30000FFF7BEFE41F66040C0F602004FF2F11179
:10F31000C0F60001F7F75CF808BD00BFAFF300804E
:10F320002DE9F0432DED048B85B00D461446F6F71C
:10F3300077FC09EE900A2846F6F772FC09EE100AEF
:10F340002046F6F705FC804619EE900AF2F73CFFDE
:10F3500004460D4619EE100AF2F736FFCDE900011A
:10F36000CDF8088041F67040C0F6020022462B46D8
:10F37000F7F796FD41F27823C2F200031868D0F83F
:10F380004C0CFDF765FE024646F64440C2F2010011
:10F3900041F6AC41C0F60201F9F782F8B8F1000F6E
:10F3A00069DD4FF012044FF00107DFED4A8A9FED4F
:10F3B0004A8A4FF0000608F1FF3101EA07092046AA
:10F3C0003946FDF725FF69EEA87A87EE880AFDEE3B
:10F3D000C00A10EE900AF5F793F820463146FDF783
:10F3E00017FF29EE281AC1EE081ABDEEE12A12EE27
:10F3F000100AF5F785F83D46474547D13BE02046E2
:10F400003946FDF705FF69EEA85A85EE886AFDEEDC
:10F41000C66A16EE900AF5F773F820463146FDF7F6
:10F42000F7FE29EE287AC7EE087ABDEEE70A10EE5D
:10F43000100AF5F765F820463946FDF7E9FE69EE52
:10F44000A80A80EE881AFDEEC11A11EE900AF5F7AF
:10F4500057F820463146FDF7DBFE29EE282AC2EE9A
:10F46000082ABDEEE23A13EE100AF5F749F805F165
:10F4700002054545C3D141F6C840C0F60200F7F782
:10F480000FFD05B0BDEC048BBDE8F083B9F1000FB2
:10F49000B5D020463946FDF7BBFE69EEA82A82EEBC
:10F4A000883AFDEEC33A13EE900AF5F729F82046A4
:10F4B0003146FDF7ADFE29EE284AC4EE084ABDEEFE
:10F4C000E45A15EE100AF5F71BF805F1010545455C
:10F4D00095D1D0E70050C34700007A44AFF30080D5
:10F4E0004FF00100704700BFAFF30080AFF3008022
:10F4F00008B5021E08DD41F27823C2F20003186845
:10F50000D0F8D43B9A4205DD41F6E440C0F6020053
:10F51000F7F7C6FC08BD00BFAFF30080AFF3008073
:10F5200010B5044641F6F841C0F60201FFF7E0FFCE
:10F5300004F1FF3446F61443C2F2010353F82400E9
:10F5400010BD00BFAFF30080AFF30080AFF30080C9
:10F550002DE9F84341F27823C2F200031868D0F88D
:10F56000D41B002934DD4FF0010546F64444C2F2B5
:10F57000010441F60C59C0F602094FF6AC26C0F65C
:10F58000010642F27008C0F6020841F27827C2F282
:10F5900000072046F8F784FD204649462A463346B0
:10F5A000F8F7F6FE2846FFF7BBFF02462046414625
:10F5B000F8F7EEFE20463146F8F7EAFE2046F8F767
:10F5C000BFFD05F101053A68D2F8D43BAB42E0DA61
:10F5D000BDE8F883AFF30080AFF30080AFF30080A5
:10F5E00038B50D46041E08DB41F27823C2F2000351
:10F5F0001868D0F8D41B8C420BDB41F61C50C0F6C7
:10F60000020041F62C51C0F602014FF04F02F4F710
:10F610006FFB46F61442C2F2010242F82450FFF793
:10F6200097FF38BDAFF30080AFF30080AFF30080E9
:10F6300010B546F64440C2F2010041F65051C0F602
:10F640000201F8F775FD41F27823C2F20003186851
:10F65000D0F8D44B002C15DD4FF0010004F1FF3140
:10F6600001403B4B43F8040F0246A04266DB09E031
:10F6700003F10401586003F10803486002F102023B
:10F68000A242F5DBFFF764FF41F27824C2F20004E6
:10F69000236841F66050C0F602004FF01201D3F823
:10F6A0004C2C03F69833FDF7EBFE236841F66C50C3
:10F6B000C0F602004FF01301D3F8502C03F6983334
:10F6C000FDF7DEFE236841F67850C0F602004FF0E9
:10F6D0001401D3F8542C03F69833FDF7D1FE2368B8
:10F6E00041F68450C0F602004FF01501D3F8582CB3
:10F6F00003F69833FDF7C4FE236841F69050C0F638
:10F7000002004FF01601D3F85C2C03F69833FDF796
:10F71000B7FE41F69C50C0F602004FF2E151C0F630
:10F720000001F6F765FE41F6A850C0F602004FF260
:10F730002131C0F60001F6F76BFE10BD002997D00D
:10F7400043F8040F02F10102A24291DB9AE700BFE5
:10F75000106C0120AFF30080AFF30080AFF30080A6
:10F7600010B546F64850C2F2010041F6C051C0F64D
:10F770000201F8F7DDFC41F27824C2F200042368AC
:10F7800041F6D050C0F602004FF00C01D3F8FC2B2C
:10F7900003F69C33FDF774FE236841F6DC50C0F697
:10F7A00002004FF00D01D3F8002C03F69C33FDF757
:10F7B00067FE236841F6E850C0F602004FF00E01E4
:10F7C000D3F8042C03F69C33FDF75AFE236841F668
:10F7D000F450C0F602004FF00F01D3F8082C03F6E6
:10F7E0009C33FDF74DFE10BDAFF30080AFF30080FA
:10F7F00070B52DED028B82B00D461446F6F710FA67
:10F8000006462846F6F70CFA05462046F6F7A0F914
:10F8100007EE900AB8EEE78A41F27824C2F20004BB
:10F82000206800F2C4604FF01001324603F0D8F8AF
:10F8300020EAE076216801F284604FF010012A4648
:10F8400003F0CEF820EAE075236806EB051203EB1F
:10F85000820080EDA18A18EE100AF2F7B5FCCDE91E
:10F86000000147F24420C2F2010041F60061C0F6F7
:10F87000020132462B46F8F713FE02B0BDEC028BB4
:10F8800070BD00BFAFF30080AFF30080AFF3008026
:10F8900010B50446F2F798FC02460B4647F24420A6
:10F8A000C2F2010041F62861C0F60201F8F7F8FD46
:10F8B00041F27823C2F200031868C0F88442C0F80D
:10F8C0008842C0F88C42C0F89042C0F89442C0F818
:10F8D0009842C0F89C42C0F8A042C0F8A442C0F8C8
:10F8E000A842C0F8AC42C0F8B042C0F8B442C0F878
:10F8F000B842C0F8BC42C0F8C042C0F8C442C0F828
:10F90000C842C0F8CC42C0F8D042C0F8D442C0F8D7
:10F91000D842C0F8DC42C0F8E042C0F8E442C0F887
:10F92000E842C0F8EC42C0F8F042C0F8F442C0F837
:10F93000F842C0F8FC42C0F80043C0F80443C0F8E5
:10F940000843C0F80C43C0F81043C0F81443C0F893
:10F950001843C0F81C43C0F82043C0F82443C0F843
:10F960002843C0F82C43C0F83043C0F83443C0F8F3
:10F970003843C0F83C43C0F84043C0F84443C0F8A3
:10F980004843C0F84C43C0F85043C0F85443C0F853
:10F990005843C0F85C43C0F86043C0F86443C0F803
:10F9A0006843C0F86C43C0F87043C0F87443C0F8B3
:10F9B0007843C0F87C43C0F88043C0F88443C0F863
:10F9C0008843C0F88C43C0F89043C0F89443C0F813
:10F9D0009843C0F89C43C0F8A043C0F8A443C0F8C3
:10F9E000A843C0F8AC43C0F8B043C0F8B443C0F873
:10F9F000B843C0F8BC43C0F8C043C0F8C443C0F823
:10FA0000C843C0F8CC43C0F8D043C0F8D443C0F8D2
:10FA1000D843C0F8DC43C0F8E043C0F8E443C0F882
:10FA2000E843C0F8EC43C0F8F043C0F8F443C0F832
:10FA3000F843C0F8FC4300F58062146000F2044112
:10FA40000C6000F581631C6000F20C42146000F54C
:10FA500082610C6000F214431C6000F58362146044
:10FA600000F21C410C6000F584631C6000F224422B
:10FA7000146000F585610C6000F22C431C6000F5F9
:10FA80008662146000F234410C6000F587631C60EC
:10FA900000F23C42146000F588610C6000F24443BF
:10FAA0001C6000F58962146000F24C410C6000F5A6
:10FAB0008A631C6000F25442146000F58B610C6094
:10FAC00000F25C431C6000F58C62146000F264413B
:10FAD0000C6000F58D631C6000F26C42146000F550
:10FAE0008E610C6000F274431C6000F58F6214603C
:10FAF00000F27C410C6000F590631C6000F28442CF
:10FB0000146000F591610C6000F28C431C6000F5FC
:10FB10009262146000F294410C6000F593631C60E3
:10FB200000F29C42146000F594610C6000F2A44362
:10FB30001C6000F59562146000F2AC410C6000F5A9
:10FB400096631C6000F2B442146000F597610C608B
:10FB500000F2BC431C6000F59862146000F2C441DE
:10FB60000C6000F599631C6000F2CC42146000F553
:10FB70009A610C6000F2D4431C6000F59B62146033
:10FB800000F2DC410C6000F59C631C6000F2E44272
:10FB9000146000F59D610C6000F2EC431C6000F500
:10FBA0009E62146000F2F4410C6000F59F631C60DB
:10FBB00000F2FC42146000F5A0610C6000F20453F6
:10FBC0001C6000F5A162146000F20C510C6000F59D
:10FBD000A2631C6000F21452146000F5A3610C6073
:10FBE00000F21C531C6000F5A462146000F2245162
:10FBF0000C6000F5A5631C6000F22C52146000F547
:10FC0000A6610C6000F234531C6000F5A76214601A
:10FC100000F23C510C6000F5A8631C6000F24452F5
:10FC2000146000F5A9610C6000F24C531C6000F5F3
:10FC3000AA62146000F254510C6000F5AB631C60C2
:10FC400000F25C52146000F5AC610C6000F2645389
:10FC50001C6000F5AD62146000F26C510C6000F5A0
:10FC6000AE631C6000F27452146000F5AF610C606A
:10FC700000F27C531C6000F5B062146000F2845105
:10FC80000C6000F5B1631C6000F28C52146000F54A
:10FC9000B2610C6000F294531C6000F5B362146012
:10FCA00000F29C510C6000F5B4631C6000F2A45299
:10FCB000146000F5B5610C6000F2AC531C6000F5F7
:10FCC000B662146000F2B4510C6000F5B7631C60BA
:10FCD00000F2BC52146000F5B8610C6000F2C4532D
:10FCE0001C6000F5B962146000F2CC510C6000F5A4
:10FCF000BA631C6000F2D452146000F5BB610C6062
:10FD000000F2DC531C6000F5BC62146000F2E451A8
:10FD10000C6000F5BD631C6000F2EC52146000F54D
:10FD2000BE610C6000F2F4531C6000F5BF62146009
:10FD300000F2FC510C6000F5C0631C6000F204622C
:10FD4000146000F5C1610C6000F20C631C6000F5EA
:10FD5000C262146000F214610C6000F5C3631C60A1
:10FD600000F21C62146000F5C4610C6000F22463B0
:10FD70001C6000F5C562146000F22C610C6000F597
:10FD8000C6631C6000F23462146000F5C7610C6049
:10FD900000F23C631C6000F5C862146000F244612C
:10FDA0000C6000F5C9631C6000F24C62146000F541
:10FDB000CA610C6000F254631C6000F5CB621460F1
:10FDC00000F25C610C6000F5CC631C6000F26462C0
:10FDD000146000F5CD610C6000F26C631C6000F5EE
:10FDE000CE62146000F274610C6000F5CF631C6099
:10FDF00000F27C62146000F5D060046010BD00BFAA
:10FE000070B52DED028B82B00D461446F5F708FF54
:10FE100006462846F5F704FF05462046F5F798FE06
:10FE200007EE900AB8EEE78A41F27824C2F20004A5
:10FE3000206800F658304FF01001324602F0D0FD35
:10FE400020EAE076216801F618304FF010012A46CA
:10FE500002F0C6FD20EAE075226806EB051303F503
:10FE6000E37002EB800181ED008A18EE100AF2F7D0
:10FE7000ABF9CDE9000147F24420C2F2010041F69E
:10FE80004861C0F6020132462B46F8F709FB02B082
:10FE9000BDEC028B70BD00BFAFF30080AFF30080FC
:10FEA00010B50446F2F790F902460B4647F244209B
:10FEB000C2F2010041F66C61C0F60201F8F7F0FAF7
:10FEC00041F27823C2F20003186800F5E36214607F
:10FED00000F21C710C6000F5E4631C6000F22472F7
:10FEE000146000F5E5610C6000F22C731C6000F5F5
:10FEF000E662146000F234710C6000F5E7631C6088
:10FF000000F23C72146000F5E8610C6000F244738A
:10FF10001C6000F5E962146000F24C710C6000F5A1
:10FF2000EA631C6000F25472146000F5EB610C602F
:10FF300000F25C731C6000F5EC62146000F2647106
:10FF40000C6000F5ED631C6000F26C72146000F54B
:10FF5000EE610C6000F274731C6000F5EF621460D7
:10FF600000F27C710C6000F5F0631C6000F284729A
:10FF7000146000F5F1610C6000F28C731C6000F5F8
:10FF8000F262146000F294710C6000F5F3631C607F
:10FF900000F29C72146000F5F4610C6000F2A4732E
:10FFA0001C6000F5F562146000F2AC710C6000F5A5
:10FFB000F6631C6000F2B472146000F5F7610C6027
:10FFC00000F2BC731C6000F5F862146000F2C471AA
:10FFD0000C6000F5F9631C6000F2CC72146000F54F
:10FFE000FA610C6000F2D4731C6000F5FB621460CF
:10FFF00000F2DC710C6000F5FC631C6000F2E4723E
:020000040801F1
:10000000146000F5FD610C6000F2EC731C6000F5FB
:10001000FE62146000F2F4710C6000F5FF631C6076
:1000200000F2FC72146000F500610C6000F604033D
:100030001C6000F60802146000F60C010C6000F56C
:1000400001631C6000F61402146000F618010C60D5
:1000500000F61C031C6000F50262146000F6240127
:100060000C6000F628031C6000F62C02146000F5FA
:1000700003610C6000F634031C6000F63802146063
:1000800000F63C010C6000F504631C6000F64402BD
:10009000146000F648010C6000F64C031C6000F58B
:1000A0000562146000F654010C6000F658031C60F1
:1000B00000F65C02146000F506610C6000F6640353
:1000C0001C6000F66802146000F66C010C6000F51C
:1000D00007631C6000F67402146000F678010C607F
:1000E00000F67C031C6000F50862146000F68401D1
:1000F0000C6000F688031C6000F68C02146000F5AA
:1001000009610C6000F694031C6000F6980214600C
:1001100000F69C010C6000F50A631C6000F6A40266
:10012000146000F6A8010C6000F6AC031C6000F53A
:100130000B62146000F6B4010C6000F6B8031C609A
:1001400000F6BC02146000F50C610C6000F6C403FC
:100150001C6000F6C802146000F6CC010C6000F5CB
:100160000D631C6000F6D402146000F6D8010C6028
:1001700000F6DC031C6000F50E62146000F6E4017A
:100180000C6000F6E8031C6000F6EC02146000F559
:100190000F610C6000F6F4031C6000F6F8021460B6
:1001A00000F6FC010C6000F510631C6000F6041200
:1001B000146000F608110C6000F60C131C6000F5CA
:1001C0001162146000F614110C6000F618131C6024
:1001D00000F61C12146000F512610C6000F6241386
:1001E0001C6000F62812146000F62C110C6000F55B
:1001F00013631C6000F63412146000F638110C60B2
:1002000000F63C131C6000F51462146000F6441103
:100210000C6000F648131C6000F64C12146000F5E8
:1002200015610C6000F654131C6000F6581214603F
:1002300000F65C110C6000F516631C6000F6641299
:10024000146000F668110C6000F66C131C6000F579
:100250001762146000F674110C6000F678131C60CD
:1002600000F67C12146000F518610C6000F684132F
:100270001C6000F68812146000F68C110C6000F50A
:1002800019631C6000F69412146000F698110C605B
:1002900000F69C131C6000F51A62146000F6A411AD
:1002A0000C6000F6A8131C6000F6AC12146000F598
:1002B0001B610C6000F6B4131C6000F6B8121460E9
:1002C00000F6BC110C6000F51C631C6000F6C41243
:1002D000146000F6C8110C6000F6CC131C6000F529
:1002E0001D62146000F6D4110C6000F6D8131C6077
:1002F00000F6DC12146000F51E610C6000F6E413D9
:100300001C6000F6E812146000F6EC110C6000F5B9
:100310001F631C6000F6F412146000F6F8110C6004
:1003200000F6FC131C6000F52062146000F6042146
:100330000C6000F608231C6000F60C22146000F527
:1003400021610C6000F614231C6000F61822146072
:1003500000F61C210C6000F522631C6000F62422CC
:10036000146000F628210C6000F62C231C6000F5B8
:100370002362146000F634210C6000F638231C6000
:1003800000F63C22146000F524610C6000F6442362
:100390001C6000F64822146000F64C210C6000F549
:1003A00025631C6000F65422146000F658210C608E
:1003B00000F65C231C6000F52662146000F66421E0
:1003C0000C6000F668231C6000F66C22146000F5D7
:1003D00027610C6000F674231C6000F6782214601C
:1003E00000F67C210C6000F528631C6000F6842276
:1003F000146000F688210C6000F68C231C6000F568
:100400002962146000F694210C6000F698231C60A9
:1004100000F69C22146000F52A610C6000F6A4230B
:100420001C6000F6A822146000F6AC210C6000F5F8
:100430002B631C6000F6B422146000F6B8210C6037
:1004400000F6BC231C6000F52C62146000F6C42189
:100450000C6000F6C8231C6000F6CC22146000F586
:100460002D610C6000F6D4231C6000F6D8221460C5
:1004700000F6DC210C6000F52E631C6000F6E4221F
:10048000146000F6E8210C6000F6EC231C6000F517
:100490002F62146000F6F4210C6000F6F8231C6053
:1004A00000F6FC22146000F530610C6000F60433A5
:1004B0001C6000F60832146000F60C310C6000F588
:1004C00031631C6000F61430046010BDAFF300808F
:1004D00008B52DED028B08EE100ADFED147AB4EEAC
:1004E000E78AF1EE10FA1DD49FED110AB4EEC08A2E
:1004F000F1EE10FA16DCF1F767FE02460B4647F202
:100500004420C2F2010041F68C61C0F60201F7F707
:10051000C7FF41F27823C2F20003186800F6884151
:1005200081ED008ABDEC028B08BD00BF0AD7233CD9
:1005300000004842AFF30080AFF30080AFF30080CB
:100540002DE9F0432DED028B89B005460C46D1F81C
:1005500004804046FBF7BCFF07EE900AB8EEE78A3E
:10056000B0EE080A68EE000A9FED331AC0EE811A59
:1005700041F27823C2F20003186800F53B6191ED67
:10058000002A21EE828A204603F06AFF06462046B2
:1005900003F0A6FF814647F24427C2F2010718EE96
:1005A000100AF1F711FECDE900014846F1F70CFE03
:1005B000CDE902013046F1F707FECDE90401CDF89F
:1005C0001880384641F6A461C0F602012A46F7F7C2
:1005D00067FF2668B069F1F7F7FD04460D46F0693C
:1005E000F1F7F2FDCDE90001306AF1F7EDFDCDE95B
:1005F0000201706AF1F7E8FDCDE90401384641F6E1
:10060000C461C0F6020122462B46F7F749FF404677
:1006100047F23421C2F20101FEF782FD024638465C
:1006200041F6DC61C0F60201F7F73AFF09B0BDEC14
:10063000028BBDE8F08300BF00F07F45AFF3008080
:100640002DE9F04782B041F27424C2F2000421681F
:100650004FF67450C0F6010001F11001FFF770FF72
:10066000216841F63040C0F6020001F10801FFF7B1
:1006700067FF206800F1100003F0F2FE8246206858
:1006800000F1080003F0ECFE814623685F6947F241
:100690003425C2F2010538462946FEF741FD804661
:1006A00047F24426C2F201065046F1F78DFD02469C
:1006B0000B460097CDF80480304641F6E061C0F665
:1006C0000201F7F7EDFE2068C46820462946FEF7D0
:1006D00027FD07464846F1F777FD02460B46009492
:1006E0000197304641F6FC61C0F60201F7F7D8FEEB
:1006F00041F27828C2F20008D8F8009041F6187745
:10070000C0F60207D9F85801F1F75EFD04460D4620
:10071000D9F85001F1F758FDCDE9000130463946CE
:1007200022462B46F7F7BCFED8F80080D8F85C01CB
:10073000F1F74AFD04460D46D8F85401F1F744FD9F
:10074000CDE900013046394622462B46F7F7A8FE90
:1007500002B0BDE8F08700BFAFF30080AFF30080C8
:1007600008B541F27823C2F200031A6807EE101AA6
:10077000F8EEC77AC2ED557A00EE100AF8EEC00A1C
:10078000C2ED570AFFF75CFF08BD00BFAFF3008062
:1007900008B541F27823C2F200031A6807EE101A76
:1007A000F8EEC77AC2ED547A00EE100AF8EEC00AED
:1007B000C2ED560AFFF744FF08BD00BFAFF300804B
:1007C0002DE9F84305460F46164647F24424C2F287
:1007D00001042046F7F7ECFD20462946F7F7D8FD3F
:1007E000002E34DD254641F63474C0F6020406F1CD
:1007F000FF3909F00109A7F1040757F8040FF1F7D1
:10080000E3FC02460B4628462146F7F7C1FD4FF0B0
:100810000108B04527D11AE007F104097868F1F71B
:10082000D3FC02460B4628462146F7F7B1FD07F1F7
:100830000807D9F80400F1F7C7FC02460B46284622
:100840002146F7F7A5FD08F10208B045E4D147F2CB
:100850004424C2F201042046F7F72AFD2046F7F7A8
:100860006FFCBDE8F883B9F1000FD5D057F8040F3D
:10087000F1F7AAFC02460B4628462146F7F788FD09
:1008800008F10108B045C7D1E1E700BFAFF3008030
:10089000D0F81437A3F10203092B2ED8DFE803F0B8
:1008A00005300A0F14191E232D2841F63870C0F6A2
:1008B0000200704741F65070C0F60200704741F6E2
:1008C0005C70C0F60200704741F66C70C0F6020022
:1008D000704741F67C70C0F60200704741F6907098
:1008E000C0F60200704741F69C70C0F602007047E7
:1008F00041F6AC70C0F6020070474FF00000704740
:1009000041F64470C0F60200704700BFAFF30080AC
:100910002DE9F04182B00446FFF7BAFF014647F2E5
:100920004425C2F201052846F7F7BAFD01F018F98F
:100930000246284641F6B871C0F60201F7F7B0FD4D
:1009400041F6D070C0F6020004F658314FF01002A4
:10095000FFF736FF41F6DC70C0F6020004F61831EE
:100960004FF01002FFF72CFF41F6E470C0F60200D2
:1009700004F188014FF01002FFF722FF41F6EC70FE
:10098000C0F6020004F148014FF01002FFF718FF13
:1009900041F6F870C0F6020004F584714FF01002C1
:1009A000FFF70EFF42F20000C0F6020004F1C8019A
:1009B0004FF01002FFF704FF42F20C00C0F60200F5
:1009C00004F128014FF00802FFF7FAFE42F214008A
:1009D000C0F6020004F108014FF00802FFF7F0FE34
:1009E000284642F22401C0F60201B4F94821F7F783
:1009F00057FD04F53E631868F1F7E6FB02460B4627
:100A0000284642F23801C0F60201F7F749FD2846B0
:100A100042F24C01C0F60201B4F94A21F7F740FD59
:100A2000284642F25801C0F60201B4F94C21F7F70A
:100A300037FD284642F26401C0F60201D4F80C27C3
:100A4000F7F72EFD04F5E260D0ED007A284642F279
:100A50007401C0F60201BDEEE70A10EE102AF7F7A6
:100A60001FFD04F5E1610868F1F7AEFB02460B4695
:100A7000284642F28801C0F60201F7F711FD04F69C
:100A8000AC321068F1F7A0FB02460B46284642F252
:100A9000A001C0F60201F7F703FD284642F2BC01AF
:100AA000C0F60201B4F94E21F7F7FAFC284642F2EB
:100AB000D001C0F60201B4F96021F7F7F1FC284635
:100AC00042F2E001C0F60201D4F8982BF7F7E8FCF7
:100AD000284642F2F801C0F60201D4F89C2BF7F741
:100AE000DFFC284642F20C11C0F60201D4F8A02B1C
:100AF000F7F7D6FC284642F21C11C0F60201D4F8E2
:100B0000A42BF7F7CDFC284642F23011C0F60201C3
:100B1000D4F8A82BF7F7C4FC04F53B663068F1F76E
:100B200053FB02460B46284642F25011C0F6020122
:100B3000F7F7B6FCD4F8FC7B3846FCF789FC804616
:100B40003846FCF795FC07464046FCF729FA034671
:100B500042F27416C0F602060097284631464FF05E
:100B60000002F7F79DFCD4F8007C3846FCF770FCD7
:100B700080463846FCF77CFC07464046FCF710FAF6
:100B800003460097284631464FF00102F7F788FCEC
:100B9000D4F8047C3846FCF75BFC80463846FCF70A
:100BA00067FC07464046FCF7FBF9034600972846DA
:100BB00031464FF00202F7F773FCD4F8084C204698
:100BC000FCF746FC07462046FCF752FC0446384634
:100BD000FCF7E6F903460094284631464FF003023D
:100BE000F7F75EFC02B0BDE8F08100BFAFF3008014
:100BF00008B541F27823C2F20003186841F274216B
:100C0000C2F200010968FFF783FE08BDAFF3008060
:100C100008B541F27823C2F20003196801F53E627B
:100C200007EE100AF8EEC77AC2ED007AFFF7E0FF90
:100C300008BD00BFAFF30080AFF30080AFF30080CA
:100C400008B541F27823C2F200031968C1F8A80B75
:100C5000FFF7CEFF08BD00BFAFF30080AFF3008009
:100C600008B541F27823C2F200031968C1F8A40B59
:100C7000FFF7BEFF08BD00BFAFF30080AFF30080F9
:100C800008B541F27823C2F200031968C1F8A00B3D
:100C9000FFF7AEFF08BD00BFAFF30080AFF30080E9
:100CA00008B541F27823C2F200031968C1F89C0B21
:100CB000FFF79EFF08BD00BFAFF30080AFF30080D9
:100CC00008B541F27823C2F200031968C1F8980B05
:100CD000FFF78EFF08BD00BFAFF30080AFF30080C9
:100CE00008B541F27823C2F200031968C1F814076D
:100CF00041F27422C2F20002126801F019FD00F004
:100D0000EFF9F1F71FF800F033FFFFF771FF08BDAF
:100D100008B541F27823C2F200031968C1F80C0744
:100D2000FFF766FF08BD00BFAFF30080AFF30080A0
:100D300008B541F27823C2F20003196801F5E262B6
:100D400007EE100AF8EEC77AC2ED007AFFF750FFFF
:100D500008BD00BFAFF30080AFF30080AFF30080A9
:100D600008B541F27823C2F200031968A1F84E01D8
:100D7000FFF73EFF08BD00BFAFF30080AFF3008078
:100D800008B541F27823C2F20003196801F6AC32CB
:100D900007EE100AF8EEC77AC2ED007AFFF728FFD7
:100DA00008BD00BFAFF30080AFF30080AFF3008059
:100DB00008B541F27823C2F20003196801F2047207
:100DC00007EE100AF8EEC77AC2ED007AFFF710FFBF
:100DD00008BD00BFAFF30080AFF30080AFF3008029
:100DE00008B547F24420C2F2010042F28811C0F671
:100DF000020146F64C62C2F201024FF47A73F7F731
:100E000077F942F29C10C0F6020040F6F131C0F6CC
:100E10000101F5F7DDFA42F2A810C0F6020040F237
:100E20004161C0F60101F5F7D3FA42F2B410C0F601
:100E3000020040F6B151C0F60101F5F7D1FA42F2D5
:100E4000C810C0F6020040F68151C0F60101F5F766
:100E5000C7FA42F2E810C0F6020040F66151C0F64F
:100E60000101F5F7BDFA42F20020C0F6020040F69B
:100E70003151C0F60101F5F7B3FA42F21820C0F67D
:100E8000020040F61151C0F60101F5F7A9FA42F24D
:100E90002820C0F6020040F6E141C0F60101F5F756
:100EA0009FFA42F23820C0F6020040F6C141C0F677
:100EB0000101F5F795FA42F25020C0F6020040F623
:100EC000A141C0F60101F5F78BFA42F26820C0F6A5
:100ED000020040F68141C0F60101F5F781FA42F2C5
:100EE0007C20C0F6020040F66141C0F60101F5F732
:100EF00077FA42F29420C0F6020040F64141C0F673
:100F00000101F5F76DFA42F2B820C0F6020040F692
:100F10001141C0F60101F5F763FA42F2CC20C0F6A8
:100F2000020040F2D141C0F60101F5F779FA42F230
:100F3000E820C0F6020040F29171C0F60101F5F719
:100F400057FA42F20030C0F6020040F26171C0F67A
:100F50000101F5F74DFA42F21830C0F602004FF6E3
:100F6000A161C0F60001F5F75BFA42F22C30C0F641
:100F700002004FF60161C0F60001F5F749FA42F2AE
:100F80003C30C0F602004FF69101C0F60001F5F7C3
:100F900047FA42F25430C0F602004FF2F171C0F647
:100FA0000001F5F735FA08BDAFF30080AFF300801C
:100FB00008B54FF0030041F27823C2F2000319682C
:100FC00041F27422C2F20002126801F0B1FB08BDC6
:100FD00070B541F20074C2F200044FF00000C0F698
:100FE0000600214640F6B842FDF78AF841F2782320
:100FF000C2F200031D68F0F769FFC5F8EC0B41F27F
:101000007420C2F20000006801F01AFB226845F269
:101010001511C0F233118A420AD047F24830C2F2A9
:10102000010042F27031C0F60201F7F739FA2BE005
:1010300041F20075C2F2000505F104004FF44B6166
:10104000F4F7FEFC044695F8B42C824229D047F20E
:101050004836C2F20106304642F29031C0F6020133
:101060002246F7F71DFA41F20075C2F2000530463C
:1010700042F29C31C0F6020195F8B42CF7F710FA51
:1010800095F8B43CA3420CD047F24830C2F20100BC
:1010900042F2B031C0F60201F7F702FAFFF788FF1B
:1010A00070BD47F24830C2F2010042F2D831C0F6BA
:1010B0000201F7F7F5F941F27820C2F20000036867
:1010C000184641F27421C2F200010968D3F81427CE
:1010D00001F0BEFA70BD00BFAFF30080AFF3008037
:1010E0002DE9F04141F20075C2F2000545F21512FA
:1010F000C0F233122E4646F8042B47F24834C2F2AF
:101100000104204642F2F431C0F60201F7F7C8F9B3
:1011100030464FF44B61F4F793FC074685F8B40C66
:10112000204642F20C41C0F6020140F6B842F7F701
:10113000B7F94FF00006C0F60606304640F6B84153
:10114000FCF7BEFF204642F22041C0F602013A46BB
:10115000F7F7A6F940F2B417C1F20007D7F80C80F0
:101160003046294640F6B842FCF7DAFF0546FA68F1
:10117000204642F23841C0F60201C8EB0202F7F7FE
:101180008FF9204642F25841C0F60201EAB2F7F761
:1011900087F9BDE8F08100BFAFF30080AFF30080B6
:1011A00008B547F24830C2F2010042F26441C0F68D
:1011B0000201F6F7BDFF42F27440C0F60200F5F7F7
:1011C0006FFE42F28440C0F6020040F6D171C0F6D4
:1011D0000101F5F7FDF842F29040C0F6020041F23D
:1011E000E101C0F60101F5F7F3F842F29C40C0F6C8
:1011F000020040F6B171C0F60101F5F7E9F8FFF71A
:10120000E7FE08BDAFF30080AFF30080AFF30080CE
:101210002DE9F843B0F1000847DD48F2A063C0F2C1
:10122000010303FB01F707F1FF3044F6D351C1F28C
:101230006201A1FB00244FEA941707F101074FF068
:10124000300449F6404608F1FF3202F00109204619
:10125000FCF78EF83846F3F753F92046FCF780F890
:101260003046F3F74DF94FF0010545451FD1BDE874
:10127000F8832046FCF77CF83846F3F741F920461E
:10128000FCF76EF83046F3F73BF92046FCF770F8B0
:101290003846F3F735F92046FCF762F83046F3F7A5
:1012A0002FF905F102054545E3D1BDE8F883B9F111
:1012B000000FDED02046FCF75BF83846F3F720F944
:1012C0002046FCF74DF83046F3F71AF905F1010511
:1012D0004545CED1BDE8F883AFF30080AFF3008081
:1012E0002DE980488FB040F29813C1F2000398694D
:1012F00042F2B042C0F60202826144F2402AC0F2D9
:101300000F0A46F26766C6F266669FED2D8B4FF0B8
:10131000010701E0DDF804A05046F3F7F1F803A857
:1013200001F05EFD03990029F6DD0DF1080B4FF089
:10133000000440F2DC594FF4C878CDF804A0A2466E
:101340000BF1040BDBF80440002C30DD22464FF09B
:10135000000586FB02104FEAE273C3EBA00205F121
:101360000105002AF5DC013D21D42846F0F71AFFDB
:1013700002460B4651EC180B0AF012FAF1F718FA74
:101380000346A04206DC3846E41A00F10100A342FD
:10139000FADD00E0384615F0010F0CBF4146494622
:1013A000FFF736FF05F1FF35B5F1FF3FDDD10AF15B
:1013B000010A03995145ADDDC2E700BFAFF30080DC
:1013C0000000000000002440AFF30080AFF3008075
:1013D00000B583B04FF00003009347F25040C2F2D3
:1013E00001004FF42E714FF0020241F2E123C0F6EA
:1013F0000103F3F75DF84FF0730001F079FC4FF053
:101400006E0001F075FC03B000BD00BFAFF30080BB
:1014100008B547F22873C2F201031A6847F2447014
:10142000C2F2010042F2C041C0F60201F7F738F8FB
:1014300008BD00BFAFF30080AFF30080AFF30080C2
:1014400038B52DED028B00295ED147F22473C2F22C
:101450000103196847F22872C2F2010211604FF0CD
:1014600000051D6047F20870C2F20100046847F6EB
:101470004803C2F201031C604FF00001016041F219
:101480007822C2F20002146809F0CAFC07EE900A42
:10149000B8EEE70A10EE100A04F5B27104F5C27254
:1014A0004FF0080301F0ECFA08EE100A09F0B8FC5E
:1014B00000EE900AB8EEE01A11EE100A04F5D271AF
:1014C00004F5E2724FF0080301F0DAFA08EE900A30
:1014D00047F21070C2F2010018EE101A41F2615288
:1014E000C0F601022B4609F0CBFF47F22C70C2F286
:1014F000010078EE288A18EE901A41F21152C0F6D7
:1015000001022B4609F0BCFFBDEC028B38BD00BFC9
:1015100008B54FF0200383F31188F2F7D1FC47F6AA
:101520004C03C2F2010393ED007A47F20C70C2F251
:101530000100D0ED007AB8EEE70AC7EE000A47F2E4
:101540004071C2F20101C1ED000AF2F791FC4FF0C7
:10155000000383F3118808BDAFF30080AFF3008070
:1015600010B54FF0200383F31188F2F7A9FC47F67A
:101570004C03C2F201034FF000021A604FF0000466
:1015800047F20C70C2F201000460F2F771FC2346CE
:1015900083F3118810BD00BFAFF30080AFF300806C
:1015A00047F64803C2F2010318687047AFF30080A2
:1015B00038B52DED028B47F22473C2F201031A688D
:1015C00002F101021A6007EE900AB8EEE78AB0EE67
:1015D000080A68EE000A9FED2A1AC0EE811A41F24D
:1015E0007824C2F20004206800F53B6191ED002AE6
:1015F00021EE828A18EE100A02F002FE05462368E8
:10160000B3F94E21022A11D147F22474C2F2010427
:10161000206810F00F0F09D140F2B411C1F200019F
:10162000C86809F01DFC2946FAF7DAFA47F208748F
:10163000C2F201042068294601F072FC20604FF0DC
:10164000200383F31188F2F73BFC47F64C03C2F208
:101650000103D3ED002A32EE888A83ED008A47F237
:101660000C70C2F20100026802F101020260F2F79E
:10167000FFFB4FF0000383F31188BDEC028B38BDF4
:1016800000F07F45AFF30080AFF30080AFF3008040
:1016900008B547F24073C2F20103186802F0B0FDCA
:1016A00008BD00BFAFF30080AFF30080AFF3008050
:1016B00008B547F24470C2F2010042F2D441C0F6CC
:1016C0000201F6F735FD41F24140C0F6010042F259
:1016D000E441C0F6020109F043FA42F2F440C0F6D8
:1016E000020041F21141C0F60101F4F771FE08BD9C
:1016F00041F27823C2F200031A6847F65000C2F2A2
:10170000010002F5E361016002F5EB63436002F55D
:10171000F361816002F5FB63C36002F618010161A9
:1017200002F65803436102F69801816102F6D8037C
:10173000C36102F61811016202F65813436202F601
:101740009811816202F6D813C36202F61821016370
:1017500002F65823436302F69821816302F6D822E9
:10176000C26347F69000C2F201004FF0010303602C
:10177000704700BFAFF30080AFF30080AFF300808D
:1017800010B5044602F014FC70B941F27823C2F29D
:1017900000031A68204602F1480102F188024FF066
:1017A000100301F06DF910BD4FF07E5010BD00BF69
:1017B00010B5044602F0FCFB70B941F27823C2F286
:1017C00000031A68204602F1C80102F584724FF046
:1017D000100301F055F910BD4FF07E5010BD00BF51
:1017E00038B5044602F0E4FB68B12046F0F7ECFCA3
:1017F00002460B4642F20050C0F60200F6F770F8BF
:101800009FED0D0A14E041F27825C2F200052A6826
:10181000204602F1080102F128024FF0080301F00E
:101820002FF92B68D3ED007A07EE100A37EE270A5E
:1018300010EE100A38BD00BF00000000AFF30080BA
:10184000E0B584B006460F4647F69002C2F20102A8
:10185000106858B942F20C50C0F6020042F228510A
:10186000C0F602014FF05502F2F742FA41F2782138
:10187000C2F200010B6803F6583500954FF01002D4
:10188000019247F65005C2F201050295384603F66B
:10189000183107EE906AB8EEE70A10EE103A01F040
:1018A0001FF904B0E0BD00BFAFF30080AFF30080CC
:1018B00008B52DED048BFFF7C3FF09EE100A02F007
:1018C0003FFFFFF775FF08EE100A02F079FEFFF701
:1018D00057FF08EE900A02F023FDFFF781FF69EE43
:1018E000288A07EE900A48EE887A17EE900ABDEC37
:1018F000048B08BDAFF30080AFF30080AFF300802E
:1019000000B52DED028B83B008EE100A02F050FBFB
:1019100058B941F27823C2F200031868D0ED547A26
:10192000B4EEE78AF1EE10FA07D541F27821C2F25F
:1019300000010A68D2F8580115E090ED557AB4EE2E
:10194000C78AF1EE10FA02DDD0F85C010BE0D0F8A6
:101950005811D0F85C318DED008A17EE900A17EE21
:10196000102A01F025F803B0BDEC028B00BD00BFCA
:1019700008B502F025FEFFF7C3FF08BDAFF30080F6
:1019800010B5044609F05CFA10B1FFF7F1FF10BD85
:1019900041F27823C2F20003186802F0B1F901465F
:1019A0002046FFF785FF10BDAFF30080AFF3008046
:1019B00038B505460C4603290BD941F23820C0F64C
:1019C000020042F22851C0F602014FF09702F2F7EE
:1019D0008FF92DB15CB1022C14BF0020012038BD5D
:1019E000012C07D0032C14BF0020012038BD4FF07C
:1019F000010038BD4FF0010038BD00BFAFF30080DB
:101A0000E0B584B006460F4647F6D402C2F20102A2
:101A1000106858B942F25050C0F6020042F26851C4
:101A2000C0F602014FF02402F2F762F941F2782188
:101A3000C2F200010B6803F2C46500954FF010027A
:101A4000019247F69405C2F201050295384603F269
:101A5000846107EE906AB8EEE70A10EE103A01F0E2
:101A60003FF804B0E0BD00BFAFF30080AFF30080EB
:101A700038B504460D4641F27823C2F200031868D7
:101A8000214602F065F948B141F27820C2F2000027
:101A9000016801F5E16292ED000A10E02046294656
:101AA000FFF7AEFF41F27821C2F200010A6802F2AC
:101AB0000473D3ED007A07EE100A37EE270A10EE12
:101AC000100A38BDAFF30080AFF30080AFF30080A1
:101AD00041F27823C2F200031A6847F69400C2F27A
:101AE000010002F5E361016002F5EB63436002F57A
:101AF000F361816002F5FB63C36002F618010161C6
:101B000002F65803436102F69801816102F6D80398
:101B1000C36102F61811016202F65813436202F61D
:101B20009811816202F6D813C36202F6182101638C
:101B300002F65823436302F69821816302F6D82205
:101B4000C26347F6D400C2F201004FF00103036004
:101B5000704700BFAFF30080AFF30080AFF30080A9
:101B600047F6D803C2F2010318687047AFF300804C
:101B700047F6D803C2F201031A6802F101021A60A3
:101B8000704700BFAFF30080AFF30080AFF3008079
:101B90004FF00003C0F84432C0F864124FF0000266
:101BA000C4F27A42C0F84822C0F868124FF000032D
:101BB000C4F2FA43C0F84C32C0F86C124FF4004241
:101BC000C4F23B52C0F85022C0F870124FF000032C
:101BD000C4F27A53C0F85432C0F874124FF4804201
:101BE000C4F29C52C0F85822C0F878124FF4004357
:101BF000C4F2BB53C0F85C32C0F87C124FF44042D0
